 LenRCClient

 Timestamp is 54265c36 (Sat Sep 27 14:41:58 2014)

 Preferred load address is 00400000

 Start         Length     Name                   Class
 0001:00000000 00021e98H .text                   CODE
 0001:00021ea0 00002721H .text$x                 CODE
 0001:000245d0 000001beH .text$yc                CODE
 0001:00024790 000000ccH .text$yd                CODE
 0002:00000000 000009dcH .idata$5                DATA
 0002:000009dc 00000004H .CRT$XCA                DATA
 0002:000009e0 00000004H .CRT$XCAA               DATA
 0002:000009e4 00000004H .CRT$XCL                DATA
 0002:000009e8 00000034H .CRT$XCU                DATA
 0002:00000a1c 00000004H .CRT$XCZ                DATA
 0002:00000a20 00000004H .CRT$XIA                DATA
 0002:00000a24 00000004H .CRT$XIAA               DATA
 0002:00000a28 00000004H .CRT$XIC                DATA
 0002:00000a2c 00000004H .CRT$XIY                DATA
 0002:00000a30 00000004H .CRT$XIZ                DATA
 0002:00000a40 00006170H .rdata                  DATA
 0002:00006bb0 0000004aH .rdata$debug            DATA
 0002:00006bfc 00000d4cH .rdata$r                DATA
 0002:00007950 000001c0H .rdata$sxdata           DATA
 0002:00007b10 00000004H .rtc$IAA                DATA
 0002:00007b14 00000004H .rtc$IZZ                DATA
 0002:00007b18 00000004H .rtc$TAA                DATA
 0002:00007b1c 00000004H .rtc$TZZ                DATA
 0002:00007b20 00002168H .xdata$x                DATA
 0002:00009c88 00000000H ATL$__a                 DATA
 0002:00009c88 00000000H ATL$__z                 DATA
 0002:00009c88 00000020H .didat$2                DATA
 0002:00009ca8 00000020H .didat$3                DATA
 0002:00009cc8 00000008H .didat$4                DATA
 0002:00009cd0 00000008H .didat$7                DATA
 0002:00009cd8 000001ccH .idata$2                DATA
 0002:00009ea4 00000014H .idata$3                DATA
 0002:00009eb8 000009dcH .idata$4                DATA
 0002:0000a894 00000ff0H .idata$6                DATA
 0002:0000b890 00000182H .edata                  DATA
 0003:00000000 00000910H .data                   DATA
 0003:00000910 00000008H .didat$5                DATA
 0003:00000918 00002bd4H .bss                    DATA
 0004:00000000 00000c40H .rsrc$01                DATA
 0004:00000c40 00032728H .rsrc$02                DATA

  Address         Publics by Value              Rva+Base       Lib:Object

 0000:00000000       __except_list              00000000     <absolute>
 0000:00000070       ___safe_se_handler_count   00000070     <absolute>
 0000:00009876       __fltused                  00009876     <absolute>
 0000:00009876       __ldused                   00009876     <absolute>
 0000:00000000       ___ImageBase               00400000     <linker-defined>
 0001:00000000       ??0CBootModuleManager@@QAE@XZ 00401000 f   BootModuleManager.obj
 0001:00000090       ??_ECBootModuleManager@@UAEPAXI@Z 00401090 f i BootModuleManager.obj
 0001:00000090       ??_GCBootModuleManager@@UAEPAXI@Z 00401090 f i BootModuleManager.obj
 0001:000000c0       ??1?$CTypedPtrList@VCPtrList@@PAK@@UAE@XZ 004010c0 f i BootModuleManager.obj
 0001:000000c0       ??1?$CTypedPtrList@VCPtrList@@PAUtagPROPERTY_REQUEST@@@@UAE@XZ 004010c0 f i PropertyManager.obj
 0001:000000c0       ??1?$CTypedPtrList@VCPtrList@@PAUtagRECVREQUEST@@@@UAE@XZ 004010c0 f i MainFrm.obj
 0001:000000e0       ??1CBootModuleManager@@UAE@XZ 004010e0 f   BootModuleManager.obj
 0001:00000170       ?GetBootParamInfo@CBootModuleManager@@QAEHXZ 00401170 f   BootModuleManager.obj
 0001:000002d0       ?SetBootParamInfo@CBootModuleManager@@QAEHXZ 004012d0 f   BootModuleManager.obj
 0001:000003b0       ?ClearCommand@CBootModuleManager@@QAEXXZ 004013b0 f   BootModuleManager.obj
 0001:00000400       ?GetPartitionProtectType@CBootModuleManager@@QAEEE@Z 00401400 f   BootModuleManager.obj
 0001:000004b0       ??0?$CTypedPtrList@VCPtrList@@PAK@@QAE@H@Z 004014b0 f i BootModuleManager.obj
 0001:000004e0       ??_G?$CTypedPtrList@VCPtrList@@PAUtagRECVREQUEST@@@@UAEPAXI@Z 004014e0 f i MainFrm.obj
 0001:000004e0       ??_E?$CTypedPtrList@VCPtrList@@PAK@@UAEPAXI@Z 004014e0 f i BootModuleManager.obj
 0001:000004e0       ??_E?$CTypedPtrList@VCPtrList@@PAUtagPROPERTY_REQUEST@@@@UAEPAXI@Z 004014e0 f i PropertyManager.obj
 0001:000004e0       ??_E?$CTypedPtrList@VCPtrList@@PAUtagRECVREQUEST@@@@UAEPAXI@Z 004014e0 f i MainFrm.obj
 0001:000004e0       ??_G?$CTypedPtrList@VCPtrList@@PAUtagPROPERTY_REQUEST@@@@UAEPAXI@Z 004014e0 f i PropertyManager.obj
 0001:000004e0       ??_G?$CTypedPtrList@VCPtrList@@PAK@@UAEPAXI@Z 004014e0 f i BootModuleManager.obj
 0001:00000510       ??0?$_CTypedPtrList@VCPtrList@@PAK@@QAE@H@Z 00401510 f i BootModuleManager.obj
 0001:00000540       ??_E?$_CTypedPtrList@VCPtrList@@PAK@@UAEPAXI@Z 00401540 f i BootModuleManager.obj
 0001:00000540       ??_G?$_CTypedPtrList@VCPtrList@@PAK@@UAEPAXI@Z 00401540 f i BootModuleManager.obj
 0001:00000540       ??_E?$_CTypedPtrList@VCPtrList@@PAUtagRECVREQUEST@@@@UAEPAXI@Z 00401540 f i MainFrm.obj
 0001:00000540       ??_G?$_CTypedPtrList@VCPtrList@@PAUtagPROPERTY_REQUEST@@@@UAEPAXI@Z 00401540 f i PropertyManager.obj
 0001:00000540       ??_G?$_CTypedPtrList@VCPtrList@@PAUtagRECVREQUEST@@@@UAEPAXI@Z 00401540 f i MainFrm.obj
 0001:00000540       ??_E?$_CTypedPtrList@VCPtrList@@PAUtagPROPERTY_REQUEST@@@@UAEPAXI@Z 00401540 f i PropertyManager.obj
 0001:00000570       ?DoDataExchange@CWnd@@MAEXPAVCDataExchange@@@Z 00401570 f i ChatDlg.obj
 0001:00000570       ?Dump@CObject@@UBEXAAVCDumpContext@@@Z 00401570 f i BootModuleManager.obj
 0001:00000570       ?Serialize@CObject@@UAEXAAVCArchive@@@Z 00401570 f i BootModuleManager.obj
 0001:00000580       ??3CObject@@SGXPAX@Z       00401580 f i BootModuleManager.obj
 0001:000005a0       ??0CCriticalSection@@QAE@XZ 004015a0 f i BootModuleManager.obj
 0001:00000620       ?Unlock@CSyncObject@@UAEHJPAJ@Z 00401620 f i BootModuleManager.obj
 0001:00000620       ?OnTearOffMenu@CFrameWndEx@@UAEHPAVCMFCPopupMenu@@PAVCPane@@@Z 00401620 f i MainFrm.obj
 0001:00000640       ?Init@CCriticalSection@@AAEHXZ 00401640 f i BootModuleManager.obj
 0001:000006e0       ??_GCCriticalSection@@UAEPAXI@Z 004016e0 f i BootModuleManager.obj
 0001:000006e0       ??_ECCriticalSection@@UAEPAXI@Z 004016e0 f i BootModuleManager.obj
 0001:00000710       ??BCCriticalSection@@QAEPAU_RTL_CRITICAL_SECTION@@XZ 00401710 f i BootModuleManager.obj
 0001:00000730       ??1CCriticalSection@@UAE@XZ 00401730 f i BootModuleManager.obj
 0001:00000760       ?Lock@CCriticalSection@@UAEHK@Z 00401760 f i BootModuleManager.obj
 0001:00000780       ?Lock@CCriticalSection@@QAEHXZ 00401780 f i BootModuleManager.obj
 0001:00000820       ?Unlock@CCriticalSection@@UAEHXZ 00401820 f i BootModuleManager.obj
 0001:00000840       ??0CErrorMessage@@QAE@ABV0@@Z 00401840 f i ChatDlg.obj
 0001:00000870       ??4CErrorMessage@@QAEAAV0@ABV0@@Z 00401870 f i ChatDlg.obj
 0001:00000890       ??_ECErrorMessage@@UAEPAXI@Z 00401890 f i ChatDlg.obj
 0001:00000900       ??0CErrorTable@@QAE@ABV0@@Z 00401900 f i ChatDlg.obj
 0001:00000930       ??4CErrorTable@@QAEAAV0@ABV0@@Z 00401930 f i ChatDlg.obj
 0001:00000960       ??_ECErrorTable@@UAEPAXI@Z 00401960 f i ChatDlg.obj
 0001:000009d0       ??0CInstall@@QAE@ABV0@@Z   004019d0 f i ChatDlg.obj
 0001:00000a30       ??4CInstall@@QAEAAV0@ABV0@@Z 00401a30 f i ChatDlg.obj
 0001:00000a90       ??_ECInstall@@UAEPAXI@Z    00401a90 f i ChatDlg.obj
 0001:00000b00       ??0CChatDlg@@QAE@PAVCWnd@@@Z 00401b00 f   ChatDlg.obj
 0001:00000be0       ??_ECChatDlg@@UAEPAXI@Z    00401be0 f i ChatDlg.obj
 0001:00000be0       ??_GCChatDlg@@UAEPAXI@Z    00401be0 f i ChatDlg.obj
 0001:00000c10       ??1CChatDlg@@UAE@XZ        00401c10 f i ChatDlg.obj
 0001:00000cc0       ?DoDataExchange@CChatDlg@@MAEXPAVCDataExchange@@@Z 00401cc0 f   ChatDlg.obj
 0001:00000d20       ?GetMessageMap@CChatDlg@@MBEPBUAFX_MSGMAP@@XZ 00401d20 f   ChatDlg.obj
 0001:00000d30       ?GetThisMessageMap@CChatDlg@@KGPBUAFX_MSGMAP@@XZ 00401d30 f   ChatDlg.obj
 0001:00000d50       ?OnSendButton@CChatDlg@@IAEXXZ 00401d50 f   ChatDlg.obj
 0001:00001390       ?OnInitDialog@CChatDlg@@MAEHXZ 00402390 f   ChatDlg.obj
 0001:00002050       ?OnCommand@CChatDlg@@MAEHIJ@Z 00403050 f   ChatDlg.obj
 0001:000025b0       ?PreTranslateMessage@CChatDlg@@UAEHPAUtagMSG@@@Z 004035b0 f   ChatDlg.obj
 0001:00002620       ?OnClose@CChatDlg@@IAEXXZ  00403620 f   ChatDlg.obj
 0001:00002660       ?OnCancel@CChatDlg@@MAEXXZ 00403660 f   ChatDlg.obj
 0001:000026a0       ??HATL@@YA?AV?$CStringT@DV?$StrTraitMFC_DLL@DV?$ChTraitsCRT@D@ATL@@@@@0@ABV10@0@Z 004036a0 f i ChatDlg.obj
 0001:00002760       ?GetCount@CPtrList@@QBEHXZ 00403760 f i MainFrm.obj
 0001:00002760       ?GetCount@CStringList@@QBEHXZ 00403760 f i ChatDlg.obj
 0001:00002780       ?GetHeadPosition@CStringList@@QBEPAU__POSITION@@XZ 00403780 f i ChatDlg.obj
 0001:000027a0       ?GetNext@CStringList@@QAEAAV?$CStringT@DV?$StrTraitMFC_DLL@DV?$ChTraitsCRT@D@ATL@@@@@ATL@@AAPAU__POSITION@@@Z 004037a0 f i ChatDlg.obj
 0001:000027e0       ?PostMessageA@CWnd@@QAEHIIJ@Z 004037e0 f i ChatDlg.obj
 0001:00002810       ?OnClose@CWnd@@IAEXXZ      00403810 f i ChatDlg.obj
 0001:00002830       ?BeginModalState@CWnd@@UAEXXZ 00403830 f i ChatDlg.obj
 0001:00002850       ?EndModalState@CWnd@@UAEXXZ 00403850 f i ChatDlg.obj
 0001:00002870       ?Create@CDialog@@UAEHIPAVCWnd@@@Z 00403870 f i ChatDlg.obj
 0001:00002890       ??0CStatic@@QAE@XZ         00403890 f i ChatDlg.obj
 0001:000028b0       ??_GCStatic@@UAEPAXI@Z     004038b0 f i ChatDlg.obj
 0001:000028b0       ??_ECStatic@@UAEPAXI@Z     004038b0 f i ChatDlg.obj
 0001:000028e0       ?ReplaceSel@CRichEditCtrl@@QAEXPBDH@Z 004038e0 f i ChatDlg.obj
 0001:00002910       ??HATL@@YA?AV?$CStringT@DV?$StrTraitMFC_DLL@DV?$ChTraitsCRT@D@ATL@@@@@0@ABV10@PBD@Z 00403910 f i ChatDlg.obj
 0001:000029d0       ??0CCheckPasswordDlg@@QAE@PAVCWnd@@@Z 004039d0 f   CheckPasswordDlg.obj
 0001:00002a80       ??_ECCheckPasswordDlg@@UAEPAXI@Z 00403a80 f i CheckPasswordDlg.obj
 0001:00002a80       ??_GCCheckPasswordDlg@@UAEPAXI@Z 00403a80 f i CheckPasswordDlg.obj
 0001:00002ab0       ??1CCheckPasswordDlg@@UAE@XZ 00403ab0 f i CheckPasswordDlg.obj
 0001:00002b30       ?DoDataExchange@CCheckPasswordDlg@@MAEXPAVCDataExchange@@@Z 00403b30 f   CheckPasswordDlg.obj
 0001:00002bb0       ?GetMessageMap@CCheckPasswordDlg@@MBEPBUAFX_MSGMAP@@XZ 00403bb0 f   CheckPasswordDlg.obj
 0001:00002bc0       ?GetThisMessageMap@CCheckPasswordDlg@@KGPBUAFX_MSGMAP@@XZ 00403bc0 f   CheckPasswordDlg.obj
 0001:00002bd0       ?OnInitDialog@CCheckPasswordDlg@@MAEHXZ 00403bd0 f   CheckPasswordDlg.obj
 0001:00002e00       ?OnOK@CCheckPasswordDlg@@MAEXXZ 00403e00 f   CheckPasswordDlg.obj
 0001:00002f00       ?OnCtlColor@CCheckPasswordDlg@@IAEPAUHBRUSH__@@PAVCDC@@PAVCWnd@@I@Z 00403f00 f   CheckPasswordDlg.obj
 0001:00002f70       ?OnBnClickedCancel@CCheckPasswordDlg@@QAEXXZ 00403f70 f   CheckPasswordDlg.obj
 0001:00002f90       ??0CEdit@@QAE@XZ           00403f90 f i CheckPasswordDlg.obj
 0001:00002fb0       ??_ECEdit@@UAEPAXI@Z       00403fb0 f i CheckPasswordDlg.obj
 0001:00002fb0       ??_GCEdit@@UAEPAXI@Z       00403fb0 f i CheckPasswordDlg.obj
 0001:00002ff0       ?SetSel@CEdit@@QAEXHHH@Z   00403ff0 f i CheckPasswordDlg.obj
 0001:00003040       ?IsPhysicalLocalMac@@YAHABV?$CStringT@DV?$StrTraitMFC_DLL@DV?$ChTraitsCRT@D@ATL@@@@@ATL@@@Z 00404040 f   CommonFunc.obj
 0001:00003380       ?GetLocalComputerInfo@@YAHPAD0@Z 00404380 f   CommonFunc.obj
 0001:00004540       ?ReadParttionMACInfo@@YAHAAUUpdateprotect@@@Z 00405540 f   CommonFunc.obj
 0001:000045f0       ?WriteParttionMACInfo@@YAHPAD@Z 004055f0 f   CommonFunc.obj
 0001:00004780       ?NICLinknumber@@YAHXZ      00405780 f   CommonFunc.obj
 0001:00004a70       ?ReadParttionPara@@YAHAAUPartion_para_sector_s@@@Z 00405a70 f   CommonFunc.obj
 0001:00004f20       ?WriteParttionPara@@YAHUPartion_para_sector_s@@H@Z 00405f20 f   CommonFunc.obj
 0001:000054f0       ?MyStringToDWORD@@YAKPAD@Z 004064f0 f   CommonFunc.obj
 0001:00005560       ?OpenOrCloseAero@@YAHH@Z   00406560 f   CommonFunc.obj
 0001:000055c0       ?GetfileVersion@@YAHV?$CStringT@DV?$StrTraitMFC_DLL@DV?$ChTraitsCRT@D@ATL@@@@@ATL@@AAV12@@Z 004065c0 f   CommonFunc.obj
 0001:000057b0       ??$strcpy_s@$0BB@@@YAHAAY0BB@DPBD@Z 004067b0 f i CommonFunc.obj
 0001:000057d0       ??8ATL@@YA_NABV?$CStringT@DV?$StrTraitMFC_DLL@DV?$ChTraitsCRT@D@ATL@@@@@0@PBD@Z 004067d0 f i CommonFunc.obj
 0001:000057f0       ?GetRuntimeClass@CDialogInputname@@UBEPAUCRuntimeClass@@XZ 004067f0 f   DialogInputname.obj
 0001:00005800       ??0CDialogInputname@@QAE@PAVCWnd@@@Z 00406800 f   DialogInputname.obj
 0001:000058a0       ??_ECDialogInputname@@UAEPAXI@Z 004068a0 f i DialogInputname.obj
 0001:000058a0       ??_GCDialogInputname@@UAEPAXI@Z 004068a0 f i DialogInputname.obj
 0001:000058d0       ??1CDialogInputname@@UAE@XZ 004068d0 f   DialogInputname.obj
 0001:00005950       ?DoDataExchange@CDialogInputname@@MAEXPAVCDataExchange@@@Z 00406950 f   DialogInputname.obj
 0001:000059d0       ?GetMessageMap@CDialogInputname@@MBEPBUAFX_MSGMAP@@XZ 004069d0 f   DialogInputname.obj
 0001:000059e0       ?GetThisMessageMap@CDialogInputname@@KGPBUAFX_MSGMAP@@XZ 004069e0 f   DialogInputname.obj
 0001:000059f0       ?OnInitDialog@CDialogInputname@@MAEHXZ 004069f0 f   DialogInputname.obj
 0001:00005b80       ?OnBnClickedOk@CDialogInputname@@QAEXXZ 00406b80 f   DialogInputname.obj
 0001:00006230       ?IsCNOrEN@CDialogInputname@@QAE_NV?$CStringT@DV?$StrTraitMFC_DLL@DV?$ChTraitsCRT@D@ATL@@@@@ATL@@@Z 00407230 f   DialogInputname.obj
 0001:000063f0       ?_GetBaseClass@CFtpClientDlg@@KGPAUCRuntimeClass@@XZ 004073f0 f   FtpClientDlg.obj
 0001:000063f0       ?_GetBaseClass@CPortChannelDlg@@KGPAUCRuntimeClass@@XZ 004073f0 f   PortChannelDlg.obj
 0001:000063f0       ?_GetBaseClass@CSetDrfaultNICDlg@@KGPAUCRuntimeClass@@XZ 004073f0 f   SetDrfaultNICDlg.obj
 0001:000063f0       ?_GetBaseClass@CDialogInputname@@KGPAUCRuntimeClass@@XZ 004073f0 f   DialogInputname.obj
 0001:00006400       ?GetRuntimeClass@CFtpClientDlg@@UBEPAUCRuntimeClass@@XZ 00407400 f   FtpClientDlg.obj
 0001:00006410       ??0CFtpClientDlg@@QAE@PAVCWnd@@@Z 00407410 f   FtpClientDlg.obj
 0001:000064d0       ??_GCFtpClientDlg@@UAEPAXI@Z 004074d0 f i FtpClientDlg.obj
 0001:000064d0       ??_ECFtpClientDlg@@UAEPAXI@Z 004074d0 f i FtpClientDlg.obj
 0001:00006500       ??1CFtpClientDlg@@UAE@XZ   00407500 f   FtpClientDlg.obj
 0001:00006540       ?DoDataExchange@CFtpClientDlg@@MAEXPAVCDataExchange@@@Z 00407540 f   FtpClientDlg.obj
 0001:00006590       ?GetMessageMap@CFtpClientDlg@@MBEPBUAFX_MSGMAP@@XZ 00407590 f   FtpClientDlg.obj
 0001:000065a0       ?GetThisMessageMap@CFtpClientDlg@@KGPBUAFX_MSGMAP@@XZ 004075a0 f   FtpClientDlg.obj
 0001:000065b0       ?OnInitDialog@CFtpClientDlg@@MAEHXZ 004075b0 f   FtpClientDlg.obj
 0001:000067c0       ?GetFtpPara@CFtpClientDlg@@QAEXXZ 004077c0 f   FtpClientDlg.obj
 0001:00006970       ?BeginFindServFile@CFtpClientDlg@@QAEHXZ 00407970 f   FtpClientDlg.obj
 0001:00006a20       ?OnConnect@CFtpClientDlg@@QAEHXZ 00407a20 f   FtpClientDlg.obj
 0001:00006b00       ?BeginSendFile@CFtpClientDlg@@QAEHXZ 00407b00 f   FtpClientDlg.obj
 0001:00006bb0       ?OnBnClickedOk@CFtpClientDlg@@QAEXXZ 00407bb0 f   FtpClientDlg.obj
 0001:000070c0       ?FindServFileThread@CMyAppThread@@SAIPAX@Z 004080c0 f   FtpClientDlg.obj
 0001:00007420       ?SendFileThread@CMyAppThread@@SAIPAX@Z 00408420 f   FtpClientDlg.obj
 0001:00007ea0       ?OnBnClickedBrowse@CFtpClientDlg@@QAEXXZ 00408ea0 f   FtpClientDlg.obj
 0001:00008170       ?OnFtp@CFtpClientDlg@@QAEJIJ@Z 00409170 f   FtpClientDlg.obj
 0001:00008550       ?OnClose@CFtpClientDlg@@QAEXXZ 00409550 f   FtpClientDlg.obj
 0001:00008630       ?OnBnClickedCancel@CFtpClientDlg@@QAEXXZ 00409630 f   FtpClientDlg.obj
 0001:00008710       ?OnTimer@CFtpClientDlg@@QAEXI@Z 00409710 f   FtpClientDlg.obj
 0001:00008730       ?OnBnClickedChkDefaultclient@CFtpClientDlg@@QAEXXZ 00409730 f   FtpClientDlg.obj
 0001:00008760       ??2CObject@@SGPAXI@Z       00409760 f i FtpClientDlg.obj
 0001:00008780       ?AfxGetAppName@@YGPBDXZ    00409780 f i FtpClientDlg.obj
 0001:00008790       ?AfxGetMainWnd@@YGPAVCWnd@@XZ 00409790 f i FtpClientDlg.obj
 0001:000087d0       ?GetSafeHwnd@CWnd@@QBEPAUHWND__@@XZ 004097d0 f i FtpClientDlg.obj
 0001:00008800       ?OnTimer@CWnd@@IAEXI@Z     00409800 f i FtpClientDlg.obj
 0001:00008820       ?GetCheck@CButton@@QBEHXZ  00409820 f i FtpClientDlg.obj
 0001:00008850       ?ResumeThread@CWinThread@@QAEKXZ 00409850 f i FtpClientDlg.obj
 0001:00008870       ?GetStartPosition@CFileDialog@@QBEPAU__POSITION@@XZ 00409870 f i FtpClientDlg.obj
 0001:00008890       ??HATL@@YA?AV?$CStringT@DV?$StrTraitMFC_DLL@DV?$ChTraitsCRT@D@ATL@@@@@0@PBDABV10@@Z 00409890 f i FtpClientDlg.obj
 0001:00008950       ??8ATL@@YA_NABV?$CStringT@DV?$StrTraitMFC_DLL@DV?$ChTraitsCRT@D@ATL@@@@@0@0@Z 00409950 f i FtpClientDlg.obj
 0001:00008970       ?GetMessageMap@CKiboClientApp@@MBEPBUAFX_MSGMAP@@XZ 00409970 f   KiboClient.obj
 0001:00008980       ?GetThisMessageMap@CKiboClientApp@@KGPBUAFX_MSGMAP@@XZ 00409980 f   KiboClient.obj
 0001:00008990       ??0CKiboClientApp@@QAE@XZ  00409990 f   KiboClient.obj
 0001:000089c0       ??_ECKiboClientApp@@UAEPAXI@Z 004099c0 f i KiboClient.obj
 0001:000089c0       ??_GCKiboClientApp@@UAEPAXI@Z 004099c0 f i KiboClient.obj
 0001:000089f0       ??1CKiboClientApp@@UAE@XZ  004099f0 f i KiboClient.obj
 0001:00008a10       ?InitInstance@CKiboClientApp@@UAEHXZ 00409a10 f   KiboClient.obj
 0001:00008db0       ??0CAboutDlg@@QAE@XZ       00409db0 f   KiboClient.obj
 0001:00008e70       ??_GCAboutDlg@@UAEPAXI@Z   00409e70 f i KiboClient.obj
 0001:00008e70       ??_ECAboutDlg@@UAEPAXI@Z   00409e70 f i KiboClient.obj
 0001:00008ea0       ??1CAboutDlg@@UAE@XZ       00409ea0 f i KiboClient.obj
 0001:00008f40       ?DoDataExchange@CAboutDlg@@MAEXPAVCDataExchange@@@Z 00409f40 f   KiboClient.obj
 0001:00008fd0       ?GetMessageMap@CAboutDlg@@MBEPBUAFX_MSGMAP@@XZ 00409fd0 f   KiboClient.obj
 0001:00008fe0       ?GetThisMessageMap@CAboutDlg@@KGPBUAFX_MSGMAP@@XZ 00409fe0 f   KiboClient.obj
 0001:00008ff0       ?OnAppAbout@CKiboClientApp@@QAEXXZ 00409ff0 f   KiboClient.obj
 0001:000090b0       ?PreLoadState@CKiboClientApp@@UAEXXZ 0040a0b0 f   KiboClient.obj
 0001:00009140       ?ExitInstance@CKiboClientApp@@MAEHXZ 0040a140 f   KiboClient.obj
 0001:00009160       ?OnInitDialog@CAboutDlg@@UAEHXZ 0040a160 f   KiboClient.obj
 0001:00009720       ?SetTitle@CAboutDlg@@QAEXXZ 0040a720 f   KiboClient.obj
 0001:000097f0       ?WMIGetHardInfo@CKiboClientApp@@QAEXV?$CStringT@DV?$StrTraitMFC_DLL@DV?$ChTraitsCRT@D@ATL@@@@@ATL@@AAH@Z 0040a7f0 f   KiboClient.obj
 0001:0000a140       ?OnBnClickedOk@CCheckPasswordDlg@@QAEXXZ 0040b140 f   CheckPasswordDlg.obj
 0001:0000a140       ?OnBnClickedOk@CAboutDlg@@QAEXXZ 0040b140 f   KiboClient.obj
 0001:0000a160       ?OnBnClickedButtonRegister@CAboutDlg@@QAEXXZ 0040b160 f   KiboClient.obj
 0001:0000a360       ?WindowProc@CAboutDlg@@MAEJIIJ@Z 0040b360 f   KiboClient.obj
 0001:0000a390       ??$wcscpy_s@$0BAE@@@YAHAAY0BAE@_WPB_W@Z 0040b390 f i KiboClient.obj
 0001:0000a3b0       ??$strncpy_s@$0BE@@@YAHAAY0BE@DPBDI@Z 0040b3b0 f i KiboClient.obj
 0001:0000a3d0       ??$strcpy_s@$0BE@@@YAHAAY0BE@DPBD@Z 0040b3d0 f i KiboClient.obj
 0001:0000a3f0       ?UpdateWindow@CWnd@@QAEXXZ 0040b3f0 f i KiboClient.obj
 0001:0000a410       ??1COleVariant@@QAE@XZ     0040b410 f i KiboClient.obj
 0001:0000a430       ?OnWorkspaceIdle@CWinAppEx@@UAEHPAVCWnd@@@Z 0040b430 f i KiboClient.obj
 0001:0000a440       ?PreSaveState@CWinAppEx@@MAEXXZ 0040b440 f i KiboClient.obj
 0001:0000a440       ?LoadCustomState@CKiboClientApp@@UAEXXZ 0040b440 f i KiboClient.obj
 0001:0000a440       ??1CObject@@UAE@XZ         0040b440 f i MainFrm.obj
 0001:0000a440       ?OnOK@CChatDlg@@MAEXXZ     0040b440 f i ChatDlg.obj
 0001:0000a440       ?SaveCustomState@CKiboClientApp@@UAEXXZ 0040b440 f i KiboClient.obj
 0001:0000a440       ?AssertValid@CObject@@UBEXXZ 0040b440 f i BootModuleManager.obj
 0001:0000a450       ??0CMFCToolTipInfo@@QAE@XZ 0040b450 f i KiboClient.obj
 0001:0000a4e0       ??0_bstr_t@@QAE@PBD@Z      0040b4e0 f i KiboClient.obj
 0001:0000a580       ??0_bstr_t@@QAE@PB_W@Z     0040b580 f i KiboClient.obj
 0001:0000a620       ??1_bstr_t@@QAE@XZ         0040b620 f i KiboClient.obj
 0001:0000a640       ??B_bstr_t@@QBEPA_WXZ      0040b640 f i KiboClient.obj
 0001:0000a670       ?_Free@_bstr_t@@AAEXXZ     0040b670 f i KiboClient.obj
 0001:0000a6a0       ??0Data_t@_bstr_t@@QAE@PBD@Z 0040b6a0 f i KiboClient.obj
 0001:0000a6e0       ??0Data_t@_bstr_t@@QAE@PB_W@Z 0040b6e0 f i KiboClient.obj
 0001:0000a730       ?Release@Data_t@_bstr_t@@QAEKXZ 0040b730 f i KiboClient.obj
 0001:0000a780       ??_GData_t@_bstr_t@@AAEPAXI@Z 0040b780 f i KiboClient.obj
 0001:0000a7b0       ??2Data_t@_bstr_t@@SAPAXI@Z 0040b7b0 f i KiboClient.obj
 0001:0000a7d0       ??1Data_t@_bstr_t@@AAE@XZ  0040b7d0 f i KiboClient.obj
 0001:0000a7f0       ?_Free@Data_t@_bstr_t@@AAEXXZ 0040b7f0 f i KiboClient.obj
 0001:0000a830       ?CreateObject@CMainFrame@@SGPAVCObject@@XZ 0040b830 f   MainFrm.obj
 0001:0000a8b0       ?_GetBaseClass@CMainFrame@@KGPAUCRuntimeClass@@XZ 0040b8b0 f   MainFrm.obj
 0001:0000a8c0       ?GetRuntimeClass@CMainFrame@@UBEPAUCRuntimeClass@@XZ 0040b8c0 f   MainFrm.obj
 0001:0000a8d0       ?GetMessageMap@CMainFrame@@MBEPBUAFX_MSGMAP@@XZ 0040b8d0 f   MainFrm.obj
 0001:0000a8e0       ?GetThisMessageMap@CMainFrame@@KGPBUAFX_MSGMAP@@XZ 0040b8e0 f   MainFrm.obj
 0001:0000ad20       ??0CMainFrame@@QAE@XZ      0040bd20 f   MainFrm.obj
 0001:0000b0c0       ??_GCMainFrame@@UAEPAXI@Z  0040c0c0 f i MainFrm.obj
 0001:0000b0c0       ??_ECMainFrame@@UAEPAXI@Z  0040c0c0 f i MainFrm.obj
 0001:0000b0f0       ??1CMainFrame@@UAE@XZ      0040c0f0 f   MainFrm.obj
 0001:0000b230       ?OnCreate@CMainFrame@@IAEHPAUtagCREATESTRUCTA@@@Z 0040c230 f   MainFrm.obj
 0001:0000b990       ?PreCreateWindow@CMainFrame@@UAEHAAUtagCREATESTRUCTA@@@Z 0040c990 f   MainFrm.obj
 0001:0000b9e0       ?OnViewCustomize@CMainFrame@@IAEXXZ 0040c9e0 f   MainFrm.obj
 0001:0000ba80       ?OnToolbarCreateNew@CMainFrame@@IAEJIJ@Z 0040ca80 f   MainFrm.obj
 0001:0000bb30       ?OnApplicationLook@CMainFrame@@IAEXI@Z 0040cb30 f   MainFrm.obj
 0001:0000bcd0       ?OnUpdateApplicationLook@CMainFrame@@IAEXPAVCCmdUI@@@Z 0040ccd0 f   MainFrm.obj
 0001:0000bd00       ?LoadFrame@CMainFrame@@UAEHIKPAVCWnd@@PAUCCreateContext@@@Z 0040cd00 f   MainFrm.obj
 0001:0000bde0       ?AddRemoveTray@CMainFrame@@QAEHH@Z 0040cde0 f   MainFrm.obj
 0001:0000bf90       ?OnWM_NOTIFYICON@CMainFrame@@IAEJIJ@Z 0040cf90 f   MainFrm.obj
 0001:0000c000       ?DisplayMenu@CMainFrame@@QAEXXZ 0040d000 f   MainFrm.obj
 0001:0000c0f0       ?OnExit@CMainFrame@@QAEXXZ 0040d0f0 f   MainFrm.obj
 0001:0000c230       ?GetGroupParameterSector@CMainFrame@@QAEHXZ 0040d230 f   MainFrm.obj
 0001:0000c5c0       ?DriverExit@CMainFrame@@QAEHXZ 0040d5c0 f   MainFrm.obj
 0001:0000c860       ?GetHostBasicIPInfo@CMainFrame@@QAEHAAUstruct_ipsetting_param@@@Z 0040d860 f   MainFrm.obj
 0001:0000dc50       ?InitNetworkComponent@CMainFrame@@QAEHXZ 0040ec50 f   MainFrm.obj
 0001:0000dde0       ?MyTrayTip@CMainFrame@@SA?AV?$CStringT@DV?$StrTraitMFC_DLL@DV?$ChTraitsCRT@D@ATL@@@@@ATL@@H@Z 0040ede0 f   MainFrm.obj
 0001:0000e110       ?ModifyTrayTip@CMainFrame@@QAEXXZ 0040f110 f   MainFrm.obj
 0001:0000e180       ?RequestHandleThread@CMainFrame@@SAIPAX@Z 0040f180 f   MainFrm.obj
 0001:0000e670       ?SetGroupParameterSector@CMainFrame@@QAEHV?$CStringT@DV?$StrTraitMFC_DLL@DV?$ChTraitsCRT@D@ATL@@@@@ATL@@@Z 0040f670 f   MainFrm.obj
 0001:0000e870       ?SendLoginRequest@CMainFrame@@QAEXXZ 0040f870 f   MainFrm.obj
 0001:0000ee30       ?_NoMessageBox@@YAIPAX@Z   0040fe30 f   MainFrm.obj
 0001:0000eee0       ?ReInitNetwrokComponent@CMainFrame@@QAEXXZ 0040fee0 f   MainFrm.obj
 0001:0000eff0       ?HandleRemoteControlCmd@CMainFrame@@QAEXPAUtagRECVREQUEST@@@Z 0040fff0 f   MainFrm.obj
 0001:00012350       ?GetDisksProperty@@YAHPAXPAU_STORAGE_DEVICE_DESCRIPTOR@@@Z 00413350 f   MainFrm.obj
 0001:000123b0       ?RejectUSBDevice@CMainFrame@@QAEXXZ 004133b0 f   MainFrm.obj
 0001:000125d0       ?SendPropertyInfoThread@CMainFrame@@SAIPAX@Z 004135d0 f   MainFrm.obj
 0001:00012a80       ?AutoSendPropertyInfoThread@CMainFrame@@SAIPAX@Z 00413a80 f   MainFrm.obj
 0001:00012ef0       ?SendBootInfoThread@CMainFrame@@SAIPAX@Z 00413ef0 f   MainFrm.obj
 0001:00013490       ?GetalldayEx@CMainFrame@@QAEGXZ 00414490 f   MainFrm.obj
 0001:00013690       ?SendPortInfoThread@CMainFrame@@SAIPAX@Z 00414690 f   MainFrm.obj
 0001:00013e60       ?OnRecvC@CMainFrame@@IAEJIJ@Z 00414e60 f   MainFrm.obj
 0001:00013f50       ?OnTimer@CMainFrame@@IAEXI@Z 00414f50 f   MainFrm.obj
 0001:00014480       ?DecreaseLifeValue@CMainFrame@@QAEXXZ 00415480 f   MainFrm.obj
 0001:00014530       ?InitSamingFilter@CMainFrame@@QAEHXZ 00415530 f   MainFrm.obj
 0001:00014920       ?OnClose@CMainFrame@@IAEXXZ 00415920 f   MainFrm.obj
 0001:00014bb0       ?_ChatHandleThread@CMainFrame@@SAIPAX@Z 00415bb0 f   MainFrm.obj
 0001:00014c40       ?SendMsg@CMainFrame@@QAEXPAU_charformat@@V?$CStringT@DV?$StrTraitMFC_DLL@DV?$ChTraitsCRT@D@ATL@@@@@ATL@@1@Z 00415c40 f   MainFrm.obj
 0001:00014ea0       ?OnChat@CMainFrame@@QAEXXZ 00415ea0 f   MainFrm.obj
 0001:00014fa0       ?OnAbout@CMainFrame@@QAEXXZ 00415fa0 f   MainFrm.obj
 0001:00014fc0       ?OnDestroy@CMainFrame@@IAEXXZ 00415fc0 f   MainFrm.obj
 0001:00014ff0       ?WindowProc@CMainFrame@@MAEJIIJ@Z 00415ff0 f   MainFrm.obj
 0001:00015e60       ?OnHand@CMainFrame@@QAEXXZ 00416e60 f   MainFrm.obj
 0001:00015fb0       ?OnUpfile@CMainFrame@@QAEXXZ 00416fb0 f   MainFrm.obj
 0001:00016110       ?ReadParttionID@CMainFrame@@QAEHAAUPara_SamEDU_Mod_Head@@@Z 00417110 f   MainFrm.obj
 0001:000163b0       ?DeleteDnsTxt@CMainFrame@@QAEXXZ 004173b0 f   MainFrm.obj
 0001:00016540       ?SendFtpFileComplete@CMainFrame@@QAEXV?$CStringT@DV?$StrTraitMFC_DLL@DV?$ChTraitsCRT@D@ATL@@@@@ATL@@0@Z 00417540 f   MainFrm.obj
 0001:00016810       ?SetInternetExplorerStartPage@CMainFrame@@QAE_NV?$CStringT@DV?$StrTraitMFC_DLL@DV?$ChTraitsCRT@D@ATL@@@@@ATL@@@Z 00417810 f   MainFrm.obj
 0001:00016930       ?AddProtect@CMainFrame@@QAEXXZ 00417930 f   MainFrm.obj
 0001:00016990       ?DelProtect@CMainFrame@@QAEXXZ 00417990 f   MainFrm.obj
 0001:000169e0       ?InitPortAndCode@CMainFrame@@QAEXXZ 004179e0 f   MainFrm.obj
 0001:00016b30       ?OnSetPort@CMainFrame@@QAEXXZ 00417b30 f   MainFrm.obj
 0001:00016d80       ?OnNetworkSet@CMainFrame@@QAEXXZ 00417d80 f   MainFrm.obj
 0001:00016eb0       ?ShowBalloonTip@CMainFrame@@QAEHPBD0K@Z 00417eb0 f   MainFrm.obj
 0001:00016f50       ?StartEClassServer@CMainFrame@@QAEXKH@Z 00417f50 f   MainFrm.obj
 0001:000171f0       ?CloseEClassServer@CMainFrame@@QAEXXZ 004181f0 f   MainFrm.obj
 0001:00017220       ?StartEClassClient@CMainFrame@@QAEXH@Z 00418220 f   MainFrm.obj
 0001:00017510       ?CloseEClassClient@CMainFrame@@QAEXXZ 00418510 f   MainFrm.obj
 0001:00017670       ?LockCDRom@CMainFrame@@QAEX_N@Z 00418670 f   MainFrm.obj
 0001:00017990       ?ModifyFirewallRule@CMainFrame@@QAEHHH@Z 00418990 f   MainFrm.obj
 0001:00018170       ?MyCreateProcess@CMainFrame@@QAEHPBDHHAAK@Z 00419170 f   MainFrm.obj
 0001:00018280       ?GetTickCount@CTime@ATL@@SG?AV12@XZ 00419280 f i MainFrm.obj
 0001:000182a0       ??0CTime@ATL@@QAE@_J@Z     004192a0 f i MainFrm.obj
 0001:000182c0       ?OnHotKey@CMainFrame@@QAEXIII@Z 004192c0 f   MainFrm.obj
 0001:00018320       ?OnShoworhide@CMainFrame@@QAEXXZ 00419320 f   MainFrm.obj
 0001:00018350       ?OnUpdateShoworhide@CMainFrame@@QAEXPAVCCmdUI@@@Z 00419350 f   MainFrm.obj
 0001:00018380       ??9ATL@@YA_NABV?$CStringT@DV?$StrTraitMFC_DLL@DV?$ChTraitsCRT@D@ATL@@@@@0@0@Z 00419380 f i MainFrm.obj
 0001:000183a0       ?RemoveHead@?$_CTypedPtrList@VCPtrList@@PAUtagRECVREQUEST@@@@QAEPAUtagRECVREQUEST@@XZ 004193a0 f i MainFrm.obj
 0001:000183a0       ?RemoveHead@?$_CTypedPtrList@VCPtrList@@PAUtagUDPRECV@@@@QAEPAUtagUDPRECV@@XZ 004193a0 f i MainFrm.obj
 0001:000183a0       ?RemoveHead@?$_CTypedPtrList@VCPtrList@@PAK@@QAEPAKXZ 004193a0 f i MainFrm.obj
 0001:000183a0       ?RemoveHead@?$_CTypedPtrList@VCPtrList@@PAUtagPROPERTY_REQUEST@@@@QAEPAUtagPROPERTY_REQUEST@@XZ 004193a0 f i MainFrm.obj
 0001:000183c0       ??0?$CTypedPtrList@VCPtrList@@PAUtagRECVREQUEST@@@@QAE@H@Z 004193c0 f i MainFrm.obj
 0001:000183f0       ?AddTail@?$CTypedPtrList@VCPtrList@@PAUtagPROPERTY_REQUEST@@@@QAEPAU__POSITION@@PAUtagPROPERTY_REQUEST@@@Z 004193f0 f i MainFrm.obj
 0001:000183f0       ?AddTail@?$CTypedPtrList@VCPtrList@@PAK@@QAEPAU__POSITION@@PAK@Z 004193f0 f i MainFrm.obj
 0001:000183f0       ?AddTail@?$CTypedPtrList@VCPtrList@@PAUtagRECVREQUEST@@@@QAEPAU__POSITION@@PAUtagRECVREQUEST@@@Z 004193f0 f i MainFrm.obj
 0001:00018410       ?GetYear@CTime@ATL@@QBEHXZ 00419410 f i MainFrm.obj
 0001:00018450       ?GetLocalTm@CTime@ATL@@QBEPAUtm@@PAU3@@Z 00419450 f i MainFrm.obj
 0001:000184c0       ?AtlThrowImpl@ATL@@YGXJ@Z  004194c0 f i MainFrm.obj
 0001:000184e0       ?GetMonth@CTime@ATL@@QBEHXZ 004194e0 f i MainFrm.obj
 0001:00018520       ?GetDay@CTime@ATL@@QBEHXZ  00419520 f i MainFrm.obj
 0001:00018560       ??0?$_CTypedPtrList@VCPtrList@@PAUtagRECVREQUEST@@@@QAE@H@Z 00419560 f i MainFrm.obj
 0001:00018590       ??$strcat_s@$0BAE@@@YAHAAY0BAE@DPBD@Z 00419590 f i MainFrm.obj
 0001:000185b0       ??$strcpy_s@$0BK@@@YAHAAY0BK@DPBD@Z 004195b0 f i MainFrm.obj
 0001:000185d0       ??$strcpy_s@$03@@YAHAAY03DPBD@Z 004195d0 f i MainFrm.obj
 0001:000185f0       ??$strcpy_s@$0EA@@@YAHAAY0EA@DPBD@Z 004195f0 f i MainFrm.obj
 0001:00018610       ??$strcpy_s@$0BAA@@@YAHAAY0BAA@DPBD@Z 00419610 f i MainFrm.obj
 0001:00018630       ??$strcpy_s@$0IA@@@YAHAAY0IA@DPBD@Z 00419630 f i MainFrm.obj
 0001:00018650       ??$strcpy_s@$0BA@@@YAHAAY0BA@DPBD@Z 00419650 f i MainFrm.obj
 0001:00018670       ??$strcpy_s@$0BD@@@YAHAAY0BD@DPBD@Z 00419670 f i MainFrm.obj
 0001:00018690       ??$sprintf_s@$09@@YAHAAY09DPBDZZ 00419690 f i MainFrm.obj
 0001:000186c0       ??$strcpy_s@$0BO@@@YAHAAY0BO@DPBD@Z 004196c0 f i MainFrm.obj
 0001:000186e0       ?Offset@CPoint@@QAEXHH@Z   004196e0 f i MainFrm.obj
 0001:00018710       ??0CPoint@@QAE@XZ          00419710 f i MainFrm.obj
 0001:00018710       ??BCRect@@QAEPAUtagRECT@@XZ 00419710 f i MainFrm.obj
 0001:00018710       ??0CObject@@IAE@XZ         00419710 f i MainFrm.obj
 0001:00018710       ?TopLeft@CRect@@QAEAAVCPoint@@XZ 00419710 f i MainFrm.obj
 0001:00018710       ?GetWString@Data_t@_bstr_t@@QAEAAPA_WXZ 00419710 f i KiboClient.obj
 0001:00018710       ??0CRect@@QAE@XZ           00419710 f i MainFrm.obj
 0001:00018720       ?IsEmpty@CPtrList@@QBEHXZ  00419720 f i MainFrm.obj
 0001:00018740       ?AfxGetInstanceHandle@@YGPAUHINSTANCE__@@XZ 00419740 f i MainFrm.obj
 0001:00018750       ??0CMenu@@QAE@XZ           00419750 f i MainFrm.obj
 0001:00018780       ??_ECMenu@@UAEPAXI@Z       00419780 f i MainFrm.obj
 0001:00018780       ??_GCMenu@@UAEPAXI@Z       00419780 f i MainFrm.obj
 0001:000187b0       ??1CMenu@@UAE@XZ           004197b0 f i MainFrm.obj
 0001:00018810       ?GetSubMenu@CMenu@@QBEPAV1@H@Z 00419810 f i MainFrm.obj
 0001:00018840       ?LoadMenuA@CMenu@@QAEHI@Z  00419840 f i MainFrm.obj
 0001:00018870       ?SendMessageA@CWnd@@QBEJIIJ@Z 00419870 f i MainFrm.obj
 0001:000188a0       ?GetClientRect@CWnd@@QBEXPAUtagRECT@@@Z 004198a0 f i MainFrm.obj
 0001:000188c0       ?RedrawWindow@CWnd@@QAEHPBUtagRECT@@PAVCRgn@@I@Z 004198c0 f i MainFrm.obj
 0001:000188f0       ?GetSafeHandle@CGdiObject@@QBEPAXXZ 004198f0 f i MainFrm.obj
 0001:00018920       ?SetTimer@CWnd@@QAEIIIP6GXPAUHWND__@@IIK@Z@Z 00419920 f i MainFrm.obj
 0001:00018950       ?KillTimer@CWnd@@QAEHI@Z   00419950 f i MainFrm.obj
 0001:00018970       ?GetFocus@CWnd@@SGPAV1@XZ  00419970 f i MainFrm.obj
 0001:00018990       ?FindWindowA@CWnd@@SGPAV1@PBD0@Z 00419990 f i MainFrm.obj
 0001:000189b0       ?OnRButtonDown@CWnd@@IAEXIVCPoint@@@Z 004199b0 f i MyRichEdit.obj
 0001:000189b0       ?OnHotKey@CWnd@@IAEXIII@Z  004199b0 f i MainFrm.obj
 0001:000189d0       ??0CWaitCursor@@QAE@XZ     004199d0 f i MainFrm.obj
 0001:000189f0       ?AfxGetApp@@YGPAVCWinApp@@XZ 004199f0 f i MainFrm.obj
 0001:00018a00       ??1CWaitCursor@@QAE@XZ     00419a00 f i MainFrm.obj
 0001:00018b90       ?GetUserToolBarByIndex@CFrameWndEx@@IBEPAVCMFCToolBar@@H@Z 00419b90 f i MainFrm.obj
 0001:00018bb0       ?OnShowCustomizePane@CFrameWndEx@@UAEHPAVCMFCPopupMenu@@I@Z 00419bb0 f i MainFrm.obj
 0001:00018be0       ?OnMenuButtonToolHitTest@CFrameWndEx@@UAEHPAVCMFCToolBarButton@@PAUtagTOOLINFOA@@@Z 00419be0 f i MainFrm.obj
 0001:00018be0       ?GetToolbarButtonToolTipText@CFrameWndEx@@UAEHPAVCMFCToolBarButton@@AAV?$CStringT@DV?$StrTraitMFC_DLL@DV?$ChTraitsCRT@D@ATL@@@@@ATL@@@Z 00419be0 f i MainFrm.obj
 0001:00018bf0       ?OnDrawMenuLogo@CFrameWndEx@@UAEXPAVCDC@@PAVCMFCPopupMenu@@ABVCRect@@@Z 00419bf0 f i MainFrm.obj
 0001:00018c00       ?OnCloseMiniFrame@CFrameWndEx@@UAEHPAVCPaneFrameWnd@@@Z 00419c00 f i MainFrm.obj
 0001:00018c00       ?OnCloseDockingPane@CFrameWndEx@@UAEHPAVCDockablePane@@@Z 00419c00 f i MainFrm.obj
 0001:00018c20       ??0CMyRichEdit@@QAE@XZ     00419c20 f   MyRichEdit.obj
 0001:00018c40       ??_ECMyRichEdit@@UAEPAXI@Z 00419c40 f i MyRichEdit.obj
 0001:00018c40       ??_GCMyRichEdit@@UAEPAXI@Z 00419c40 f i MyRichEdit.obj
 0001:00018c70       ??1CMyRichEdit@@UAE@XZ     00419c70 f   MyRichEdit.obj
 0001:00018c90       ?GetMessageMap@CMyRichEdit@@MBEPBUAFX_MSGMAP@@XZ 00419c90 f   MyRichEdit.obj
 0001:00018ca0       ?GetThisMessageMap@CMyRichEdit@@KGPBUAFX_MSGMAP@@XZ 00419ca0 f   MyRichEdit.obj
 0001:00018cb0       ?OnCopy@CMyRichEdit@@QAEXXZ 00419cb0 f i MyRichEdit.obj
 0001:00018cd0       ?OnCut@CMyRichEdit@@QAEXXZ 00419cd0 f i MyRichEdit.obj
 0001:00018cf0       ?OnPaste@CMyRichEdit@@QAEXXZ 00419cf0 f i MyRichEdit.obj
 0001:00018d10       ?OnSelectall@CMyRichEdit@@QAEXXZ 00419d10 f i MyRichEdit.obj
 0001:00018d30       ?OnUndo@CMyRichEdit@@QAEXXZ 00419d30 f i MyRichEdit.obj
 0001:00018d50       ?OnClear@CMyRichEdit@@QAEXXZ 00419d50 f i MyRichEdit.obj
 0001:00018d80       ?OnRButtonDown@CMyRichEdit@@QAEXIVCPoint@@@Z 00419d80 f   MyRichEdit.obj
 0001:000190b0       ?CreatePopupMenu@CMenu@@QAEHXZ 0041a0b0 f i MyRichEdit.obj
 0001:000190d0       ?AppendMenuA@CMenu@@QAEHIIPBD@Z 0041a0d0 f i MyRichEdit.obj
 0001:00019100       ?EnableMenuItem@CMenu@@QAEIII@Z 0041a100 f i MyRichEdit.obj
 0001:00019130       ??0CRichEditCtrl@@QAE@XZ   0041a130 f i MyRichEdit.obj
 0001:00019150       ??_ECRichEditCtrl@@UAEPAXI@Z 0041a150 f i MyRichEdit.obj
 0001:00019150       ??_GCRichEditCtrl@@UAEPAXI@Z 0041a150 f i MyRichEdit.obj
 0001:00019180       ?CanUndo@CRichEditCtrl@@QBEHXZ 0041a180 f i MyRichEdit.obj
 0001:000191b0       ?Undo@CRichEditCtrl@@QAEHXZ 0041a1b0 f i MyRichEdit.obj
 0001:000191e0       ?Copy@CRichEditCtrl@@QAEXXZ 0041a1e0 f i MyRichEdit.obj
 0001:00019210       ?Cut@CRichEditCtrl@@QAEXXZ 0041a210 f i MyRichEdit.obj
 0001:00019240       ?Paste@CRichEditCtrl@@QAEXXZ 0041a240 f i MyRichEdit.obj
 0001:00019270       ?GetSelectionType@CRichEditCtrl@@QBEGXZ 0041a270 f i MyRichEdit.obj
 0001:000192a0       ?GetTextLength@CRichEditCtrl@@QBEJXZ 0041a2a0 f i MyRichEdit.obj
 0001:000192c0       ?GetRuntimeClass@CPortChannelDlg@@UBEPAUCRuntimeClass@@XZ 0041a2c0 f   PortChannelDlg.obj
 0001:000192d0       ??0CPortChannelDlg@@QAE@PAVCWnd@@@Z 0041a2d0 f   PortChannelDlg.obj
 0001:00019310       ??_GCPortChannelDlg@@UAEPAXI@Z 0041a310 f i PortChannelDlg.obj
 0001:00019310       ??_ECPortChannelDlg@@UAEPAXI@Z 0041a310 f i PortChannelDlg.obj
 0001:00019340       ??1CPortChannelDlg@@UAE@XZ 0041a340 f   PortChannelDlg.obj
 0001:00019360       ?DoDataExchange@CPortChannelDlg@@MAEXPAVCDataExchange@@@Z 0041a360 f   PortChannelDlg.obj
 0001:00019390       ?GetMessageMap@CPortChannelDlg@@MBEPBUAFX_MSGMAP@@XZ 0041a390 f   PortChannelDlg.obj
 0001:000193a0       ?GetThisMessageMap@CPortChannelDlg@@KGPBUAFX_MSGMAP@@XZ 0041a3a0 f   PortChannelDlg.obj
 0001:000193b0       ?OnBnClickedOk@CPortChannelDlg@@QAEXXZ 0041a3b0 f   PortChannelDlg.obj
 0001:00019480       ?OnInitDialog@CPortChannelDlg@@UAEHXZ 0041a480 f   PortChannelDlg.obj
 0001:000195e0       ?SetTitle@CPortChannelDlg@@QAEXXZ 0041a5e0 f   PortChannelDlg.obj
 0001:000197b0       ??0CPropertyManager@@QAE@XZ 0041a7b0 f   PropertyManager.obj
 0001:00019840       ??_ECPropertyManager@@UAEPAXI@Z 0041a840 f i PropertyManager.obj
 0001:00019840       ??_GCPropertyManager@@UAEPAXI@Z 0041a840 f i PropertyManager.obj
 0001:00019870       ??1?$_CTypedPtrList@VCPtrList@@PAUtagRECVREQUEST@@@@UAE@XZ 0041a870 f i MainFrm.obj
 0001:00019870       ??1?$_CTypedPtrList@VCPtrList@@PAK@@UAE@XZ 0041a870 f i BootModuleManager.obj
 0001:00019870       ??1?$_CTypedPtrList@VCPtrList@@PAUtagPROPERTY_REQUEST@@@@UAE@XZ 0041a870 f i PropertyManager.obj
 0001:00019890       ??1CPropertyManager@@UAE@XZ 0041a890 f   PropertyManager.obj
 0001:00019920       ?GetCurrentPropertyInfo@CPropertyManager@@QAEPAUPropertyInfo@@XZ 0041a920 f   PropertyManager.obj
 0001:00019a80       ?GetCurrentHardwareInfo@CPropertyManager@@QAEXXZ 0041aa80 f   PropertyManager.obj
 0001:00019be0       ?GetCurrentSoftwareInfo@CPropertyManager@@QAEXXZ 0041abe0 f   PropertyManager.obj
 0001:0001ae30       ?strstr@@YAPADPADPBD@Z     0041be30 f i PropertyManager.obj
 0001:0001ae50       ?FilerIllegalCharacters@CPropertyManager@@QAEXXZ 0041be50 f   PropertyManager.obj
 0001:0001aeb0       ?GethardInfo@CPropertyManager@@QAEHV?$CStringT@DV?$StrTraitMFC_DLL@DV?$ChTraitsCRT@D@ATL@@@@@ATL@@0H@Z 0041beb0 f   PropertyManager.obj
 0001:0001b330       ?WMIGetHardInfo@CPropertyManager@@QAEXV?$CStringT@DV?$StrTraitMFC_DLL@DV?$ChTraitsCRT@D@ATL@@@@@ATL@@@Z 0041c330 f   PropertyManager.obj
 0001:0001c340       ??0?$CTypedPtrList@VCPtrList@@PAUtagPROPERTY_REQUEST@@@@QAE@H@Z 0041d340 f i PropertyManager.obj
 0001:0001c370       ??0?$_CTypedPtrList@VCPtrList@@PAUtagPROPERTY_REQUEST@@@@QAE@H@Z 0041d370 f i PropertyManager.obj
 0001:0001c3a0       ??$strcpy_s@$0N@@@YAHAAY0N@DPBD@Z 0041d3a0 f i PropertyManager.obj
 0001:0001c3c0       ??$strcpy_s@$0FA@@@YAHAAY0FA@DPBD@Z 0041d3c0 f i PropertyManager.obj
 0001:0001c3e0       ??$strcpy_s@$0HM@@@YAHAAY0HM@DPBD@Z 0041d3e0 f i PropertyManager.obj
 0001:0001c400       ?SetAt@CMapStringToString@@QAEXPBD0@Z 0041d400 f i PropertyManager.obj
 0001:0001c430       ?GetStartPosition@CMapStringToString@@QBEPAU__POSITION@@XZ 0041d430 f i PropertyManager.obj
 0001:0001c450       ?GetRuntimeClass@CSetDrfaultNICDlg@@UBEPAUCRuntimeClass@@XZ 0041d450 f   SetDrfaultNICDlg.obj
 0001:0001c460       ??0CSetDrfaultNICDlg@@QAE@PAVCWnd@@@Z 0041d460 f   SetDrfaultNICDlg.obj
 0001:0001c510       ??_ECSetDrfaultNICDlg@@UAEPAXI@Z 0041d510 f i SetDrfaultNICDlg.obj
 0001:0001c510       ??_GCSetDrfaultNICDlg@@UAEPAXI@Z 0041d510 f i SetDrfaultNICDlg.obj
 0001:0001c540       ??1CSetDrfaultNICDlg@@UAE@XZ 0041d540 f   SetDrfaultNICDlg.obj
 0001:0001c5d0       ?DoDataExchange@CSetDrfaultNICDlg@@MAEXPAVCDataExchange@@@Z 0041d5d0 f   SetDrfaultNICDlg.obj
 0001:0001c630       ?GetMessageMap@CSetDrfaultNICDlg@@MBEPBUAFX_MSGMAP@@XZ 0041d630 f   SetDrfaultNICDlg.obj
 0001:0001c640       ?GetThisMessageMap@CSetDrfaultNICDlg@@KGPBUAFX_MSGMAP@@XZ 0041d640 f   SetDrfaultNICDlg.obj
 0001:0001c650       ?OnBnClickedOk@CSetDrfaultNICDlg@@QAEXXZ 0041d650 f   SetDrfaultNICDlg.obj
 0001:0001c7c0       ?OnInitDialog@CSetDrfaultNICDlg@@UAEHXZ 0041d7c0 f   SetDrfaultNICDlg.obj
 0001:0001c9e0       ?GetLocalComputerInfo@CSetDrfaultNICDlg@@QAEHXZ 0041d9e0 f   SetDrfaultNICDlg.obj
 0001:0001cce0       ?SetTitle@CSetDrfaultNICDlg@@QAEXXZ 0041dce0 f   SetDrfaultNICDlg.obj
 0001:0001cf00       ??0CComboBox@@QAE@XZ       0041df00 f i SetDrfaultNICDlg.obj
 0001:0001cf20       ??_ECComboBox@@UAEPAXI@Z   0041df20 f i SetDrfaultNICDlg.obj
 0001:0001cf20       ??_GCComboBox@@UAEPAXI@Z   0041df20 f i SetDrfaultNICDlg.obj
 0001:0001cf50       ?SetCurSel@CComboBox@@QAEHH@Z 0041df50 f i SetDrfaultNICDlg.obj
 0001:0001cf80       ?AddString@CComboBox@@QAEHPBD@Z 0041df80 f i SetDrfaultNICDlg.obj
 0001:0001cfb0       ?GetCurrentPath@@YAHXZ     0041dfb0 f   comfunc:comfunc.obj
 0001:0001d080       ?SetLogFile@@YAHPBD@Z      0041e080 f   comfunc:comfunc.obj
 0001:0001d130       _AlreadyRunning            0041e130 f   comfunc:comfunc.obj
 0001:0001d170       _ExReBoot                  0041e170 f   comfunc:comfunc.obj
 0001:0001d260       ?SetPrivilege@@YAHPAXPBDH@Z 0041e260 f   comfunc:comfunc.obj
 0001:0001d2d0       _KillPS                    0041e2d0 f   comfunc:comfunc.obj
 0001:0001d3f0       _IsWow64                   0041e3f0 f   comfunc:comfunc.obj
 0001:0001d440       _ExIsVista                 0041e440 f   comfunc:comfunc.obj
 0001:0001d4b0       _WriteRunLog               0041e4b0 f   comfunc:comfunc.obj
 0001:0001d6d0       ?IsNtSys@@YAHXZ            0041e6d0 f   comfunc:comfunc.obj
 0001:0001d780       _GetWindowsVersion         0041e780 f   comfunc:comfunc.obj
 0001:0001d950       _InitComFunc               0041e950 f   comfunc:comfunc.obj
 0001:0001d9d0       ?ExtractProcessName@@YA?AV?$CStringT@DV?$StrTraitMFC_DLL@DV?$ChTraitsCRT@D@ATL@@@@@ATL@@PAD@Z 0041e9d0 f   comfunc:comfunc.obj
 0001:0001da10       _GetProcessIdFromName      0041ea10 f   comfunc:comfunc.obj
 0001:0001daf0       ??0CRegistry@@QAE@XZ       0041eaf0 f   comfunc:Registry.obj
 0001:0001db20       ?ClearKey@CRegistry@@QAEHXZ 0041eb20 f   comfunc:Registry.obj
 0001:0001db40       ?SetRootKey@CRegistry@@QAEHPAUHKEY__@@@Z 0041eb40 f   comfunc:Registry.obj
 0001:0001db70       ?GetDataType@CRegistry@@QAEKV?$CStringT@DV?$StrTraitMFC_DLL@DV?$ChTraitsCRT@D@ATL@@@@@ATL@@@Z 0041eb70 f   comfunc:Registry.obj
 0001:0001dc00       ?KeyExists@CRegistry@@QAEHV?$CStringT@DV?$StrTraitMFC_DLL@DV?$ChTraitsCRT@D@ATL@@@@@ATL@@PAUHKEY__@@@Z 0041ec00 f   comfunc:Registry.obj
 0001:0001dc60       ?SetKey@CRegistry@@QAEHV?$CStringT@DV?$StrTraitMFC_DLL@DV?$ChTraitsCRT@D@ATL@@@@@ATL@@H@Z 0041ec60 f   comfunc:Registry.obj
 0001:0001ddb0       ?ReadString@CRegistry@@QAE?AV?$CStringT@DV?$StrTraitMFC_DLL@DV?$ChTraitsCRT@D@ATL@@@@@ATL@@V23@0@Z 0041edb0 f   comfunc:Registry.obj
 0001:0001df10       ?ReadDword@CRegistry@@QAEKV?$CStringT@DV?$StrTraitMFC_DLL@DV?$ChTraitsCRT@D@ATL@@@@@ATL@@K@Z 0041ef10 f   comfunc:Registry.obj
 0001:0001dfc0       ?ReadBool@CRegistry@@QAEHV?$CStringT@DV?$StrTraitMFC_DLL@DV?$ChTraitsCRT@D@ATL@@@@@ATL@@H@Z 0041efc0 f   comfunc:Registry.obj
 0001:0001e070       ?WriteBool@CRegistry@@QAEHV?$CStringT@DV?$StrTraitMFC_DLL@DV?$ChTraitsCRT@D@ATL@@@@@ATL@@H@Z 0041f070 f   comfunc:Registry.obj
 0001:0001e110       ?WriteString@CRegistry@@QAEHV?$CStringT@DV?$StrTraitMFC_DLL@DV?$ChTraitsCRT@D@ATL@@@@@ATL@@0@Z 0041f110 f   comfunc:Registry.obj
 0001:0001e230       ?WriteDword@CRegistry@@QAEHV?$CStringT@DV?$StrTraitMFC_DLL@DV?$ChTraitsCRT@D@ATL@@@@@ATL@@K@Z 0041f230 f   comfunc:Registry.obj
 0001:0001e2d0       ?ReadBinary@CRegistry@@QAEHV?$CStringT@DV?$StrTraitMFC_DLL@DV?$ChTraitsCRT@D@ATL@@@@@ATL@@PAEK@Z 0041f2d0 f   comfunc:Registry.obj
 0001:0001e370       ?WriteMSZString@CRegistry@@QAEHV?$CStringT@DV?$StrTraitMFC_DLL@DV?$ChTraitsCRT@D@ATL@@@@@ATL@@0@Z 0041f370 f   comfunc:Registry.obj
 0001:0001e500       ?ReadMSZString@CRegistry@@QAEHV?$CStringT@DV?$StrTraitMFC_DLL@DV?$ChTraitsCRT@D@ATL@@@@@ATL@@PAD@Z 0041f500 f   comfunc:Registry.obj
 0001:0001e650       ??1CRegistry@@QAE@XZ       0041f650 f   comfunc:Registry.obj
 0001:0001e662       _ExRWDisk                  0041f662 f   windisk:windisk.dll
 0001:0001e668       _ExRWDiskAbs               0041f668 f   windisk:windisk.dll
 0001:0001e66e       _ExDetectProtect           0041f66e f   windisk:windisk.dll
 0001:0001e680       ?TranNodeToStr@@YAHPAE0@Z  0041f680 f   helpful:helpful.obj
 0001:0001e6c0       ?SetTTL@CMulticastSocket@@QAEHI@Z 0041f6c0 f   commod2:MulticastSocket.obj
 0001:0001e6f0       ?SetLoopBack@CMulticastSocket@@QAEHH@Z 0041f6f0 f   commod2:MulticastSocket.obj
 0001:0001e720       ?JoinGroup@CMulticastSocket@@QAEHV?$CStringT@DV?$StrTraitMFC_DLL@DV?$ChTraitsCRT@D@ATL@@@@@ATL@@PBD@Z 0041f720 f   commod2:MulticastSocket.obj
 0001:0001e790       ?LeaveGroup@CMulticastSocket@@QAEHXZ 0041f790 f   commod2:MulticastSocket.obj
 0001:0001e7b0       ?CommSecrect@CMulticastSocket@@QAEXPAEG@Z 0041f7b0 f   commod2:MulticastSocket.obj
 0001:0001e7d0       ?SendToSingle@CMulticastSocket@@QAEHPAD0GK@Z 0041f7d0 f   commod2:MulticastSocket.obj
 0001:0001e8a0       ??1?$CTypedPtrList@VCPtrList@@PAUtagUDPRECV@@@@UAE@XZ 0041f8a0 f i commod2:MulticastSocket.obj
 0001:0001e8a0       ??1?$CTypedPtrList@VCPtrList@@PAUSTRUCT_PROTECTITEM@@@@UAE@XZ 0041f8a0 f i kibokern:kibokern.obj
 0001:0001e8b0       ?CreateReceivingSocket@CMulticastSocket@@QAEHPAVCWnd@@PBDG1@Z 0041f8b0 f   commod2:MulticastSocket.obj
 0001:0001ea10       ?CreateSendingSocket@CMulticastSocket@@QAEHIHPBD@Z 0041fa10 f   commod2:MulticastSocket.obj
 0001:0001eb30       ?Receive@CMulticastSocket@@QAEHXZ 0041fb30 f   commod2:MulticastSocket.obj
 0001:0001ebe0       ?Initial@CMulticastSocket@@QAEHPAVCWnd@@V?$CStringT@DV?$StrTraitMFC_DLL@DV?$ChTraitsCRT@D@ATL@@@@@ATL@@GPBDIHH@Z 0041fbe0 f   commod2:MulticastSocket.obj
 0001:0001eca0       ??0CMulticastSocket@@QAE@XZ 0041fca0 f   commod2:MulticastSocket.obj
 0001:0001ed60       ?CloseSocket@CMulticastSocket@@QAEXXZ 0041fd60 f   commod2:MulticastSocket.obj
 0001:0001edc0       ??1CMulticastSocket@@UAE@XZ 0041fdc0 f   commod2:MulticastSocket.obj
 0001:0001ee30       ??_GCMulticastSocket@@UAEPAXI@Z 0041fe30 f i commod2:MulticastSocket.obj
 0001:0001ee30       ??_ECMulticastSocket@@UAEPAXI@Z 0041fe30 f i commod2:MulticastSocket.obj
 0001:0001ee50       ?descryptparasector@CKiboKern@@AAEXXZ 0041fe50 f   kibokern:kibokern.obj
 0001:0001ef10       ?encryptparasector@CKiboKern@@AAEXXZ 0041ff10 f   kibokern:kibokern.obj
 0001:0001efd0       ?WriteParaSector@CKiboKern@@QAEXXZ 0041ffd0 f   kibokern:kibokern.obj
 0001:0001f050       ?LoadParaSector@CKiboKern@@QAEHXZ 00420050 f   kibokern:kibokern.obj
 0001:0001f130       ?InitKern@CKiboKern@@QAEHXZ 00420130 f   kibokern:kibokern.obj
 0001:0001f3b0       ??_G?$CTypedPtrList@VCPtrList@@PAUSTRUCT_PROTECTITEM@@@@UAEPAXI@Z 004203b0 f i kibokern:kibokern.obj
 0001:0001f3b0       ??_E?$CTypedPtrList@VCPtrList@@PAUSTRUCT_PROTECTITEM@@@@UAEPAXI@Z 004203b0 f i kibokern:kibokern.obj
 0001:0001f3b0       ??_G?$CTypedPtrList@VCPtrList@@PAUtagUDPRECV@@@@UAEPAXI@Z 004203b0 f i commod2:MulticastSocket.obj
 0001:0001f3b0       ??_E?$CTypedPtrList@VCPtrList@@PAUtagUDPRECV@@@@UAEPAXI@Z 004203b0 f i commod2:MulticastSocket.obj
 0001:0001f3d0       ??0CKiboKern@@QAE@XZ       004203d0 f   kibokern:kibokern.obj
 0001:0001f400       ??1CKiboKern@@UAE@XZ       00420400 f   kibokern:kibokern.obj
 0001:0001f4b0       ??_ECKiboKern@@UAEPAXI@Z   004204b0 f i kibokern:kibokern.obj
 0001:0001f4b0       ??_GCKiboKern@@UAEPAXI@Z   004204b0 f i kibokern:kibokern.obj
 0001:0001f4ce       ??1CErrorMessage@@UAE@XZ   004204ce f   SPIFilter:SPIFilter.dll
 0001:0001f4d4       ??1CErrorTable@@UAE@XZ     004204d4 f   SPIFilter:SPIFilter.dll
 0001:0001f4da       ??1CInstall@@UAE@XZ        004204da f   SPIFilter:SPIFilter.dll
 0001:0001f4e0       ??0CInstall@@QAE@XZ        004204e0 f   SPIFilter:SPIFilter.dll
 0001:0001f4f0       ?SetBasicPath@@YAXPBD@Z    004204f0 f   loadres:exloadres.obj
 0001:0001f510       ?ExGetResString@@YA?AV?$CStringT@DV?$StrTraitMFC_DLL@DV?$ChTraitsCRT@D@ATL@@@@@ATL@@PAD0@Z 00420510 f   loadres:exloadres.obj
 0001:0001f620       ?ExGetResBmp@@YA?AV?$CStringT@DV?$StrTraitMFC_DLL@DV?$ChTraitsCRT@D@ATL@@@@@ATL@@PAD0@Z 00420620 f   loadres:exloadres.obj
 0001:0001f7b0       ?ExCheckAllRes@@YAHPBD@Z   004207b0 f   loadres:exloadres.obj
 0001:0001fce0       ??0CIniStruct@@QAE@XZ      00420ce0 f   loadres:initwork.obj
 0001:0001fcf0       ?addsection@CIniStruct@@QAEHPAD@Z 00420cf0 f   loadres:initwork.obj
 0001:0001fe20       ?sectionkey@CIniStruct@@QAEPADH@Z 00420e20 f   loadres:initwork.obj
 0001:0001fe30       ?sectionvalue@CIniStruct@@QAEPADH@Z 00420e30 f   loadres:initwork.obj
 0001:0001fe40       ?GetCount@CIniStruct@@QAEHXZ 00420e40 f   loadres:initwork.obj
 0001:0001fe50       ?Release@CIniStruct@@QAEHXZ 00420e50 f   loadres:initwork.obj
 0001:0001feb0       ??1CIniStruct@@QAE@XZ      00420eb0 f   loadres:initwork.obj
 0001:0001fec0       ?ReadProfileSection@@YAKPBD0AAVCIniStruct@@@Z 00420ec0 f   loadres:initwork.obj
 0001:0001fff0       ?replacestr@@YAXPAD00@Z    00420ff0 f   loadres:initwork.obj
 0001:00020170       ?ReadProfileReplace@@YAKPBDAAVCIniStruct@@@Z 00421170 f   loadres:initwork.obj
 0001:000202b0       ?ReadIniFileKey@@YAAAV?$CStringT@DV?$StrTraitMFC_DLL@DV?$ChTraitsCRT@D@ATL@@@@@ATL@@PBD0PADAAV12@@Z 004212b0 f   loadres:initwork.obj
 0001:000204ab       __imp_load__DwmEnableComposition@4 004214ab     dwmapi:dwmapi.dll
 0001:000204b5       __tailMerge_dwmapi_dll     004214b5     dwmapi:dwmapi.dll
 0001:000204c6       ___delayLoadHelper2@8      004214c6 f   DelayImp:delayhlp.obj
 0001:00020704       ??3@YAXPAX@Z               00421704 f   mfc90:mfc90.dll
 0001:0002070a       ??1CPtrList@@UAE@XZ        0042170a f   mfc90:mfc90.dll
 0001:00020710       ?GetRuntimeClass@CPtrList@@UBEPAUCRuntimeClass@@XZ 00421710 f   mfc90:mfc90.dll
 0001:00020716       ??0CPtrList@@QAE@H@Z       00421716 f   mfc90:mfc90.dll
 0001:0002071c       ??1CSyncObject@@UAE@XZ     0042171c f   mfc90:mfc90.dll
 0001:00020722       ?AfxThrowMemoryException@@YGXXZ 00421722 f   mfc90:mfc90.dll
 0001:00020728       ??0CSyncObject@@QAE@PBD@Z  00421728 f   mfc90:mfc90.dll
 0001:0002072e       ?GetRuntimeClass@CCriticalSection@@UBEPAUCRuntimeClass@@XZ 0042172e f   mfc90:mfc90.dll
 0001:00020734       ??_V@YAXPAX@Z              00421734 f   mfc90:mfc90.dll
 0001:0002073a       ??1CDialog@@UAE@XZ         0042173a f   mfc90:mfc90.dll
 0001:00020740       ??0CDialog@@QAE@IPAVCWnd@@@Z 00421740 f   mfc90:mfc90.dll
 0001:00020746       ?GetRuntimeClass@CDialog@@UBEPAUCRuntimeClass@@XZ 00421746 f   mfc90:mfc90.dll
 0001:0002074c       ?OnCmdMsg@CDialog@@UAEHIHPAXPAUAFX_CMDHANDLERINFO@@@Z 0042174c f   mfc90:mfc90.dll
 0001:00020752       ?OnFinalRelease@CWnd@@UAEXXZ 00421752 f   mfc90:mfc90.dll
 0001:00020758       ?IsInvokeAllowed@CCmdTarget@@UAEHJ@Z 00421758 f   mfc90:mfc90.dll
 0001:0002075e       ?GetDispatchIID@CCmdTarget@@UAEHPAU_GUID@@@Z 0042175e f   mfc90:mfc90.dll
 0001:00020764       ?GetTypeInfoCount@CCmdTarget@@UAEIXZ 00421764 f   mfc90:mfc90.dll
 0001:0002076a       ?GetTypeLibCache@CCmdTarget@@UAEPAVCTypeLibCache@@XZ 0042176a f   mfc90:mfc90.dll
 0001:00020770       ?GetTypeLib@CCmdTarget@@UAEJKPAPAUITypeLib@@@Z 00421770 f   mfc90:mfc90.dll
 0001:00020776       ?GetCommandMap@CCmdTarget@@MBEPBUAFX_OLECMDMAP@@XZ 00421776 f   mfc90:mfc90.dll
 0001:0002077c       ?GetDispatchMap@CCmdTarget@@MBEPBUAFX_DISPMAP@@XZ 0042177c f   mfc90:mfc90.dll
 0001:00020782       ?GetConnectionMap@CCmdTarget@@MBEPBUAFX_CONNECTIONMAP@@XZ 00421782 f   mfc90:mfc90.dll
 0001:00020788       ?GetInterfaceMap@CWnd@@MBEPBUAFX_INTERFACEMAP@@XZ 00421788 f   mfc90:mfc90.dll
 0001:0002078e       ?GetEventSinkMap@CCmdTarget@@MBEPBUAFX_EVENTSINKMAP@@XZ 0042178e f   mfc90:mfc90.dll
 0001:00020794       ?OnCreateAggregates@CCmdTarget@@UAEHXZ 00421794 f   mfc90:mfc90.dll
 0001:0002079a       ?GetInterfaceHook@CCmdTarget@@UAEPAUIUnknown@@PBX@Z 0042179a f   mfc90:mfc90.dll
 0001:000207a0       ?GetExtraConnectionPoints@CCmdTarget@@MAEHPAVCPtrArray@@@Z 004217a0 f   mfc90:mfc90.dll
 0001:000207a6       ?GetConnectionHook@CCmdTarget@@MAEPAUIConnectionPoint@@ABU_GUID@@@Z 004217a6 f   mfc90:mfc90.dll
 0001:000207ac       ?PreSubclassWindow@CWnd@@UAEXXZ 004217ac f   mfc90:mfc90.dll
 0001:000207b2       ?Create@CWnd@@UAEHPBD0KABUtagRECT@@PAV1@IPAUCCreateContext@@@Z 004217b2 f   mfc90:mfc90.dll
 0001:000207b8       ?CreateEx@CWnd@@UAEHKPBD0KABUtagRECT@@PAV1@IPAX@Z 004217b8 f   mfc90:mfc90.dll
 0001:000207be       ?CreateEx@CWnd@@UAEHKPBD0KHHHHPAUHWND__@@PAUHMENU__@@PAX@Z 004217be f   mfc90:mfc90.dll
 0001:000207c4       ?DestroyWindow@CWnd@@UAEHXZ 004217c4 f   mfc90:mfc90.dll
 0001:000207ca       ?PreCreateWindow@CWnd@@UAEHAAUtagCREATESTRUCTA@@@Z 004217ca f   mfc90:mfc90.dll
 0001:000207d0       ?CalcWindowRect@CWnd@@UAEXPAUtagRECT@@I@Z 004217d0 f   mfc90:mfc90.dll
 0001:000207d6       ?GetMenu@CWnd@@UBEPAVCMenu@@XZ 004217d6 f   mfc90:mfc90.dll
 0001:000207dc       ?SetMenu@CWnd@@UAEHPAVCMenu@@@Z 004217dc f   mfc90:mfc90.dll
 0001:000207e2       ?OnToolHitTest@CWnd@@UBEHVCPoint@@PAUtagTOOLINFOA@@@Z 004217e2 f   mfc90:mfc90.dll
 0001:000207e8       ?GetScrollBarCtrl@CWnd@@UBEPAVCScrollBar@@H@Z 004217e8 f   mfc90:mfc90.dll
 0001:000207ee       ?WinHelpA@CWnd@@UAEXKI@Z   004217ee f   mfc90:mfc90.dll
 0001:000207f4       ?HtmlHelpA@CWnd@@UAEXKI@Z  004217f4 f   mfc90:mfc90.dll
 0001:000207fa       ?WinHelpInternal@CWnd@@UAEXKI@Z 004217fa f   mfc90:mfc90.dll
 0001:00020800       ?ContinueModal@CWnd@@UAEHXZ 00421800 f   mfc90:mfc90.dll
 0001:00020806       ?EndModalLoop@CWnd@@UAEXH@Z 00421806 f   mfc90:mfc90.dll
 0001:0002080c       ?EnsureStdObj@CWnd@@UAEJXZ 0042180c f   mfc90:mfc90.dll
 0001:00020812       ?get_accParent@CWnd@@UAEJPAPAUIDispatch@@@Z 00421812 f   mfc90:mfc90.dll
 0001:00020818       ?get_accChildCount@CWnd@@UAEJPAJ@Z 00421818 f   mfc90:mfc90.dll
 0001:0002081e       ?get_accChild@CWnd@@UAEJUtagVARIANT@@PAPAUIDispatch@@@Z 0042181e f   mfc90:mfc90.dll
 0001:00020824       ?get_accName@CWnd@@UAEJUtagVARIANT@@PAPA_W@Z 00421824 f   mfc90:mfc90.dll
 0001:0002082a       ?get_accValue@CWnd@@UAEJUtagVARIANT@@PAPA_W@Z 0042182a f   mfc90:mfc90.dll
 0001:00020830       ?get_accDescription@CWnd@@UAEJUtagVARIANT@@PAPA_W@Z 00421830 f   mfc90:mfc90.dll
 0001:00020836       ?get_accRole@CWnd@@UAEJUtagVARIANT@@PAU2@@Z 00421836 f   mfc90:mfc90.dll
 0001:0002083c       ?get_accState@CWnd@@UAEJUtagVARIANT@@PAU2@@Z 0042183c f   mfc90:mfc90.dll
 0001:00020842       ?get_accHelp@CWnd@@UAEJUtagVARIANT@@PAPA_W@Z 00421842 f   mfc90:mfc90.dll
 0001:00020848       ?get_accHelpTopic@CWnd@@UAEJPAPA_WUtagVARIANT@@PAJ@Z 00421848 f   mfc90:mfc90.dll
 0001:0002084e       ?get_accKeyboardShortcut@CWnd@@UAEJUtagVARIANT@@PAPA_W@Z 0042184e f   mfc90:mfc90.dll
 0001:00020854       ?get_accFocus@CWnd@@UAEJPAUtagVARIANT@@@Z 00421854 f   mfc90:mfc90.dll
 0001:0002085a       ?get_accSelection@CWnd@@UAEJPAUtagVARIANT@@@Z 0042185a f   mfc90:mfc90.dll
 0001:00020860       ?get_accDefaultAction@CWnd@@UAEJUtagVARIANT@@PAPA_W@Z 00421860 f   mfc90:mfc90.dll
 0001:00020866       ?accSelect@CWnd@@UAEJJUtagVARIANT@@@Z 00421866 f   mfc90:mfc90.dll
 0001:0002086c       ?accLocation@CWnd@@UAEJPAJ000UtagVARIANT@@@Z 0042186c f   mfc90:mfc90.dll
 0001:00020872       ?accNavigate@CWnd@@UAEJJUtagVARIANT@@PAU2@@Z 00421872 f   mfc90:mfc90.dll
 0001:00020878       ?accHitTest@CWnd@@UAEJJJPAUtagVARIANT@@@Z 00421878 f   mfc90:mfc90.dll
 0001:0002087e       ?accDoDefaultAction@CWnd@@UAEJUtagVARIANT@@@Z 0042187e f   mfc90:mfc90.dll
 0001:00020884       ?put_accName@CWnd@@UAEJUtagVARIANT@@PA_W@Z 00421884 f   mfc90:mfc90.dll
 0001:0002088a       ?put_accValue@CWnd@@UAEJUtagVARIANT@@PA_W@Z 0042188a f   mfc90:mfc90.dll
 0001:00020890       ?SetProxy@CWnd@@UAEJPAUIAccessibleProxy@@@Z 00421890 f   mfc90:mfc90.dll
 0001:00020896       ?CreateAccessibleProxy@CWnd@@UAEJIJPAJ@Z 00421896 f   mfc90:mfc90.dll
 0001:0002089c       ?OnNotify@CWnd@@MAEHIJPAJ@Z 0042189c f   mfc90:mfc90.dll
 0001:000208a2       ?GetSuperWndProcAddr@CWnd@@MAEPAP6GJPAUHWND__@@IIJ@ZXZ 004218a2 f   mfc90:mfc90.dll
 0001:000208a8       ?OnAmbientProperty@CWnd@@UAEHPAVCOleControlSite@@JPAUtagVARIANT@@@Z 004218a8 f   mfc90:mfc90.dll
 0001:000208ae       ?WindowProc@CWnd@@MAEJIIJ@Z 004218ae f   mfc90:mfc90.dll
 0001:000208b4       ?OnWndMsg@CWnd@@MAEHIIJPAJ@Z 004218b4 f   mfc90:mfc90.dll
 0001:000208ba       ?DefWindowProcA@CWnd@@MAEJIIJ@Z 004218ba f   mfc90:mfc90.dll
 0001:000208c0       ?PostNcDestroy@CWnd@@MAEXXZ 004218c0 f   mfc90:mfc90.dll
 0001:000208c6       ?OnChildNotify@CWnd@@MAEHIIJPAJ@Z 004218c6 f   mfc90:mfc90.dll
 0001:000208cc       ?CheckAutoCenter@CDialog@@UAEHXZ 004218cc f   mfc90:mfc90.dll
 0001:000208d2       ?IsFrameWnd@CWnd@@UBEHXZ   004218d2 f   mfc90:mfc90.dll
 0001:000208d8       ?CreateControlContainer@CWnd@@MAEHPAPAVCOleControlContainer@@@Z 004218d8 f   mfc90:mfc90.dll
 0001:000208de       ?CreateControlSite@CWnd@@MAEHPAVCOleControlContainer@@PAPAVCOleControlSite@@IABU_GUID@@@Z 004218de f   mfc90:mfc90.dll
 0001:000208e4       ?SetOccDialogInfo@CDialog@@MAEHPAU_AFX_OCC_DIALOG_INFO@@@Z 004218e4 f   mfc90:mfc90.dll
 0001:000208ea       ?GetOccDialogInfo@CDialog@@MAEPAU_AFX_OCC_DIALOG_INFO@@XZ 004218ea f   mfc90:mfc90.dll
 0001:000208f0       ?Create@CDialog@@UAEHPBDPAVCWnd@@@Z 004218f0 f   mfc90:mfc90.dll
 0001:000208f6       ?CreateIndirect@CDialog@@UAEHPAXPAVCWnd@@@Z 004218f6 f   mfc90:mfc90.dll
 0001:000208fc       ?CreateIndirect@CDialog@@UAEHPBUDLGTEMPLATE@@PAVCWnd@@PAX@Z 004218fc f   mfc90:mfc90.dll
 0001:00020902       ?DoModal@CDialog@@UAEHXZ   00421902 f   mfc90:mfc90.dll
 0001:00020908       ?OnSetFont@CDialog@@UAEXPAVCFont@@@Z 00421908 f   mfc90:mfc90.dll
 0001:0002090e       ?PreInitDialog@CDialog@@MAEXXZ 0042190e f   mfc90:mfc90.dll
 0001:00020914       ??1CStatic@@UAE@XZ         00421914 f   mfc90:mfc90.dll
 0001:0002091a       ?DDX_Control@@YGXPAVCDataExchange@@HAAVCWnd@@@Z 0042191a f   mfc90:mfc90.dll
 0001:00020920       ?GetThisMessageMap@CDialog@@KGPBUAFX_MSGMAP@@XZ 00421920 f   mfc90:mfc90.dll
 0001:00020926       ?SetWindowTextA@CWnd@@QAEXPBD@Z 00421926 f   mfc90:mfc90.dll
 0001:0002092c       ?SetWordCharFormat@CRichEditCtrl@@QAEHAAU_charformat@@@Z 0042192c f   mfc90:mfc90.dll
 0001:00020932       ?SetSel@CRichEditCtrl@@QAEXJJ@Z 00421932 f   mfc90:mfc90.dll
 0001:00020938       ?AddTail@CStringList@@QAEPAU__POSITION@@ABV?$CStringT@DV?$StrTraitMFC_DLL@DV?$ChTraitsCRT@D@ATL@@@@@ATL@@@Z 00421938 f   mfc90:mfc90.dll
 0001:0002093e       ?GetWindowTextLengthA@CWnd@@QBEHXZ 0042193e f   mfc90:mfc90.dll
 0001:00020944       ?GetWindowTextA@CWnd@@QBEXAAV?$CStringT@DV?$StrTraitMFC_DLL@DV?$ChTraitsCRT@D@ATL@@@@@ATL@@@Z 00421944 f   mfc90:mfc90.dll
 0001:0002094a       ?SetFocus@CWnd@@QAEPAV1@XZ 0042194a f   mfc90:mfc90.dll
 0001:00020950       ?GetDlgItem@CWnd@@QBEPAV1@H@Z 00421950 f   mfc90:mfc90.dll
 0001:00020956       ?AfxMessageBox@@YGHPBDII@Z 00421956 f   mfc90:mfc90.dll
 0001:0002095c       ?SetWindowPos@CWnd@@QAEHPBV1@HHHHI@Z 0042195c f   mfc90:mfc90.dll
 0001:00020962       ?OnInitDialog@CDialog@@UAEHXZ 00421962 f   mfc90:mfc90.dll
 0001:00020968       ?OnCommand@CWnd@@MAEHIJ@Z  00421968 f   mfc90:mfc90.dll
 0001:0002096e       ?EndDialog@CDialog@@QAEXH@Z 0042196e f   mfc90:mfc90.dll
 0001:00020974       ?PreTranslateMessage@CDialog@@UAEHPAUtagMSG@@@Z 00421974 f   mfc90:mfc90.dll
 0001:0002097a       ?RemoveAll@CStringList@@QAEXXZ 0042197a f   mfc90:mfc90.dll
 0001:00020980       ?OnCancel@CDialog@@MAEXXZ  00421980 f   mfc90:mfc90.dll
 0001:00020986       ?AfxThrowInvalidArgException@@YGXXZ 00421986 f   mfc90:mfc90.dll
 0001:0002098c       ?Default@CWnd@@IAEJXZ      0042198c f   mfc90:mfc90.dll
 0001:00020992       ??0CWnd@@QAE@XZ            00421992 f   mfc90:mfc90.dll
 0001:00020998       ?GetRuntimeClass@CStatic@@UBEPAUCRuntimeClass@@XZ 00421998 f   mfc90:mfc90.dll
 0001:0002099e       ?OnCmdMsg@CCmdTarget@@UAEHIHPAXPAUAFX_CMDHANDLERINFO@@@Z 0042199e f   mfc90:mfc90.dll
 0001:000209a4       ?GetMessageMap@CWnd@@MBEPBUAFX_MSGMAP@@XZ 004219a4 f   mfc90:mfc90.dll
 0001:000209aa       ?PreTranslateMessage@CWnd@@UAEHPAUtagMSG@@@Z 004219aa f   mfc90:mfc90.dll
 0001:000209b0       ?OnChildNotify@CStatic@@MAEHIIJPAJ@Z 004219b0 f   mfc90:mfc90.dll
 0001:000209b6       ?CheckAutoCenter@CWnd@@UAEHXZ 004219b6 f   mfc90:mfc90.dll
 0001:000209bc       ?SetOccDialogInfo@CWnd@@MAEHPAU_AFX_OCC_DIALOG_INFO@@@Z 004219bc f   mfc90:mfc90.dll
 0001:000209c2       ?GetOccDialogInfo@CWnd@@MAEPAU_AFX_OCC_DIALOG_INFO@@XZ 004219c2 f   mfc90:mfc90.dll
 0001:000209c8       ?Create@CStatic@@UAEHPBDKABUtagRECT@@PAVCWnd@@I@Z 004219c8 f   mfc90:mfc90.dll
 0001:000209ce       ?DrawItem@CStatic@@UAEXPAUtagDRAWITEMSTRUCT@@@Z 004219ce f   mfc90:mfc90.dll
 0001:000209d4       ??1CEdit@@UAE@XZ           004219d4 f   mfc90:mfc90.dll
 0001:000209da       ?DDV_MaxChars@@YGXPAVCDataExchange@@ABV?$CStringT@DV?$StrTraitMFC_DLL@DV?$ChTraitsCRT@D@ATL@@@@@ATL@@H@Z 004219da f   mfc90:mfc90.dll
 0001:000209e0       ?DDX_Text@@YGXPAVCDataExchange@@HAAV?$CStringT@DV?$StrTraitMFC_DLL@DV?$ChTraitsCRT@D@ATL@@@@@ATL@@@Z 004219e0 f   mfc90:mfc90.dll
 0001:000209e6       ?ShowWindow@CWnd@@QAEHH@Z  004219e6 f   mfc90:mfc90.dll
 0001:000209ec       ?UpdateData@CWnd@@QAEHH@Z  004219ec f   mfc90:mfc90.dll
 0001:000209f2       ?OnOK@CDialog@@MAEXXZ      004219f2 f   mfc90:mfc90.dll
 0001:000209f8       ?SetBkMode@CDC@@QAEHH@Z    004219f8 f   mfc90:mfc90.dll
 0001:000209fe       ?GetDlgCtrlID@CWnd@@QBEHXZ 004219fe f   mfc90:mfc90.dll
 0001:00020a04       ?OnCtlColor@CWnd@@IAEPAUHBRUSH__@@PAVCDC@@PAV1@I@Z 00421a04 f   mfc90:mfc90.dll
 0001:00020a0a       ?GetRuntimeClass@CEdit@@UBEPAUCRuntimeClass@@XZ 00421a0a f   mfc90:mfc90.dll
 0001:00020a10       ??_U@YAPAXI@Z              00421a10 f   mfc90:mfc90.dll
 0001:00020a16       ?GetThisClass@CDialog@@SGPAUCRuntimeClass@@XZ 00421a16 f   mfc90:mfc90.dll
 0001:00020a1c       ?DDX_Check@@YGXPAVCDataExchange@@HAAH@Z 00421a1c f   mfc90:mfc90.dll
 0001:00020a22       ?AfxBeginThread@@YGPAVCWinThread@@P6AIPAX@Z0HIKPAU_SECURITY_ATTRIBUTES@@@Z 00421a22 f   mfc90:mfc90.dll
 0001:00020a28       ?MessageBoxA@CWnd@@QAEHPBD0I@Z 00421a28 f   mfc90:mfc90.dll
 0001:00020a2e       ??1CFileFind@@UAE@XZ       00421a2e f   mfc90:mfc90.dll
 0001:00020a34       ?FindFile@CFileFind@@UAEHPBDK@Z 00421a34 f   mfc90:mfc90.dll
 0001:00020a3a       ??0CFileFind@@QAE@XZ       00421a3a f   mfc90:mfc90.dll
 0001:00020a40       ?OnFinalRelease@CCmdTarget@@UAEXXZ 00421a40 f   mfc90:mfc90.dll
 0001:00020a46       ?GetInterfaceMap@CCmdTarget@@MBEPBUAFX_INTERFACEMAP@@XZ 00421a46 f   mfc90:mfc90.dll
 0001:00020a4c       ?PreTranslateMessage@CWinThread@@UAEHPAUtagMSG@@@Z 00421a4c f   mfc90:mfc90.dll
 0001:00020a52       ?PumpMessage@CWinThread@@UAEHXZ 00421a52 f   mfc90:mfc90.dll
 0001:00020a58       ?IsIdleMessage@CWinThread@@UAEHPAUtagMSG@@@Z 00421a58 f   mfc90:mfc90.dll
 0001:00020a5e       ?ProcessMessageFilter@CWinThread@@UAEHHPAUtagMSG@@@Z 00421a5e f   mfc90:mfc90.dll
 0001:00020a64       ?GetMainWnd@CWinThread@@UAEPAVCWnd@@XZ 00421a64 f   mfc90:mfc90.dll
 0001:00020a6a       ?Delete@CWinThread@@UAEXXZ 00421a6a f   mfc90:mfc90.dll
 0001:00020a70       ?PutFile@CFtpConnection@@QAEHPBD0KK@Z 00421a70 f   mfc90:mfc90.dll
 0001:00020a76       ??1CFtpFileFind@@UAE@XZ    00421a76 f   mfc90:mfc90.dll
 0001:00020a7c       ?GetFileName@CFileFind@@UBE?AV?$CStringT@DV?$StrTraitMFC_DLL@DV?$ChTraitsCRT@D@ATL@@@@@ATL@@XZ 00421a7c f   mfc90:mfc90.dll
 0001:00020a82       ?FindNextFileA@CFtpFileFind@@UAEHXZ 00421a82 f   mfc90:mfc90.dll
 0001:00020a88       ?FindFile@CFtpFileFind@@UAEHPBDK@Z 00421a88 f   mfc90:mfc90.dll
 0001:00020a8e       ??0CFtpFileFind@@QAE@PAVCFtpConnection@@K@Z 00421a8e f   mfc90:mfc90.dll
 0001:00020a94       ?SetCurrentDirectoryA@CFtpConnection@@QAEHPBD@Z 00421a94 f   mfc90:mfc90.dll
 0001:00020a9a       ?CreateDirectoryA@CFtpConnection@@QAEHPBD@Z 00421a9a f   mfc90:mfc90.dll
 0001:00020aa0       ?GetFtpConnection@CInternetSession@@QAEPAVCFtpConnection@@PBD00GH@Z 00421aa0 f   mfc90:mfc90.dll
 0001:00020aa6       ??0CInternetSession@@QAE@PBDKK00K@Z 00421aa6 f   mfc90:mfc90.dll
 0001:00020aac       ?GetNextPathName@CFileDialog@@QBE?AV?$CStringT@DV?$StrTraitMFC_DLL@DV?$ChTraitsCRT@D@ATL@@@@@ATL@@AAPAU__POSITION@@@Z 00421aac f   mfc90:mfc90.dll
 0001:00020ab2       ??1CFileDialog@@UAE@XZ     00421ab2 f   mfc90:mfc90.dll
 0001:00020ab8       ?DoModal@CFileDialog@@UAEHXZ 00421ab8 f   mfc90:mfc90.dll
 0001:00020abe       ?GetOFN@CFileDialog@@QAEAAUtagOFNA@@XZ 00421abe f   mfc90:mfc90.dll
 0001:00020ac4       ??0CFileDialog@@QAE@HPBD0K0PAVCWnd@@KH@Z 00421ac4 f   mfc90:mfc90.dll
 0001:00020aca       ?EnableWindow@CWnd@@QAEHH@Z 00421aca f   mfc90:mfc90.dll
 0001:00020ad0       ??2@YAPAXI@Z               00421ad0 f   mfc90:mfc90.dll
 0001:00020ad6       ?AfxGetModuleState@@YGPAVAFX_MODULE_STATE@@XZ 00421ad6 f   mfc90:mfc90.dll
 0001:00020adc       ?AfxGetThread@@YGPAVCWinThread@@XZ 00421adc f   mfc90:mfc90.dll
 0001:00020ae2       ?GetOFN@CFileDialog@@QBEABUtagOFNA@@XZ 00421ae2 f   mfc90:mfc90.dll
 0001:00020ae8       ?GetThisMessageMap@CWinApp@@KGPBUAFX_MSGMAP@@XZ 00421ae8 f   mfc90:mfc90.dll
 0001:00020aee       ?OnFileNew@CWinApp@@IAEXXZ 00421aee f   mfc90:mfc90.dll
 0001:00020af4       ?OnFileOpen@CWinApp@@IAEXXZ 00421af4 f   mfc90:mfc90.dll
 0001:00020afa       ?OnFilePrintSetup@CWinApp@@IAEXXZ 00421afa f   mfc90:mfc90.dll
 0001:00020b00       ??0CWinAppEx@@QAE@H@Z      00421b00 f   mfc90:mfc90.dll
 0001:00020b06       ?GetRuntimeClass@CWinAppEx@@UBEPAUCRuntimeClass@@XZ 00421b06 f   mfc90:mfc90.dll
 0001:00020b0c       ?Run@CWinApp@@UAEHXZ       00421b0c f   mfc90:mfc90.dll
 0001:00020b12       ?OnIdle@CWinApp@@UAEHJ@Z   00421b12 f   mfc90:mfc90.dll
 0001:00020b18       ?ProcessWndProcException@CWinApp@@UAEJPAVCException@@PBUtagMSG@@@Z 00421b18 f   mfc90:mfc90.dll
 0001:00020b1e       ?InitLibId@CWinApp@@UAEXXZ 00421b1e f   mfc90:mfc90.dll
 0001:00020b24       ?Register@CWinApp@@UAEHXZ  00421b24 f   mfc90:mfc90.dll
 0001:00020b2a       ?Unregister@CWinApp@@UAEHXZ 00421b2a f   mfc90:mfc90.dll
 0001:00020b30       ?OpenDocumentFile@CWinApp@@UAEPAVCDocument@@PBD@Z 00421b30 f   mfc90:mfc90.dll
 0001:00020b36       ?AddToRecentFileList@CWinApp@@UAEXPBD@Z 00421b36 f   mfc90:mfc90.dll
 0001:00020b3c       ?InitApplication@CWinApp@@UAEHXZ 00421b3c f   mfc90:mfc90.dll
 0001:00020b42       ?SaveAllModified@CWinApp@@UAEHXZ 00421b42 f   mfc90:mfc90.dll
 0001:00020b48       ?DoMessageBox@CWinApp@@UAEHPBDII@Z 00421b48 f   mfc90:mfc90.dll
 0001:00020b4e       ?DoWaitCursor@CWinApp@@UAEXH@Z 00421b4e f   mfc90:mfc90.dll
 0001:00020b54       ?OnDDECommand@CWinApp@@UAEHPAD@Z 00421b54 f   mfc90:mfc90.dll
 0001:00020b5a       ?WinHelpA@CWinApp@@UAEXKI@Z 00421b5a f   mfc90:mfc90.dll
 0001:00020b60       ?HtmlHelpA@CWinApp@@UAEXKI@Z 00421b60 f   mfc90:mfc90.dll
 0001:00020b66       ?WinHelpInternal@CWinApp@@UAEXKI@Z 00421b66 f   mfc90:mfc90.dll
 0001:00020b6c       ?LoadAppLangResourceDLL@CWinApp@@UAEPAUHINSTANCE__@@XZ 00421b6c f   mfc90:mfc90.dll
 0001:00020b72       ?LoadSysPolicies@CWinApp@@UAEHXZ 00421b72 f   mfc90:mfc90.dll
 0001:00020b78       ?LoadState@CWinAppEx@@UAEHPBDPAVCFrameImpl@@@Z 00421b78 f   mfc90:mfc90.dll
 0001:00020b7e       ?CleanState@CWinAppEx@@UAEHPBD@Z 00421b7e f   mfc90:mfc90.dll
 0001:00020b84       ?SaveState@CWinAppEx@@UAEHPBDPAVCFrameImpl@@@Z 00421b84 f   mfc90:mfc90.dll
 0001:00020b8a       ?OnViewDoubleClick@CWinAppEx@@UAEHPAVCWnd@@H@Z 00421b8a f   mfc90:mfc90.dll
 0001:00020b90       ?ShowPopupMenu@CWinAppEx@@UAEHIABVCPoint@@PAVCWnd@@@Z 00421b90 f   mfc90:mfc90.dll
 0001:00020b96       ?OnAppContextHelp@CWinAppEx@@UAEXPAVCWnd@@QBK@Z 00421b96 f   mfc90:mfc90.dll
 0001:00020b9c       ?OnClosingMainFrame@CWinAppEx@@MAEXPAVCFrameImpl@@@Z 00421b9c f   mfc90:mfc90.dll
 0001:00020ba2       ?LoadWindowPlacement@CWinAppEx@@MAEHAAVCRect@@AAH1@Z 00421ba2 f   mfc90:mfc90.dll
 0001:00020ba8       ?StoreWindowPlacement@CWinAppEx@@MAEHABVCRect@@HH@Z 00421ba8 f   mfc90:mfc90.dll
 0001:00020bae       ?ReloadWindowPlacement@CWinAppEx@@MAEHPAVCFrameWnd@@@Z 00421bae f   mfc90:mfc90.dll
 0001:00020bb4       ??1CWinAppEx@@UAE@XZ       00421bb4 f   mfc90:mfc90.dll
 0001:00020bba       ??1CCommandLineInfo@@UAE@XZ 00421bba f   mfc90:mfc90.dll
 0001:00020bc0       ?ProcessShellCommand@CWinApp@@QAEHAAVCCommandLineInfo@@@Z 00421bc0 f   mfc90:mfc90.dll
 0001:00020bc6       ?ParseCommandLine@CWinApp@@QAEXAAVCCommandLineInfo@@@Z 00421bc6 f   mfc90:mfc90.dll
 0001:00020bcc       ??0CCommandLineInfo@@QAE@XZ 00421bcc f   mfc90:mfc90.dll
 0001:00020bd2       ?SetTooltipParams@CTooltipManager@@QAEXIPAUCRuntimeClass@@PAVCMFCToolTipInfo@@@Z 00421bd2 f   mfc90:mfc90.dll
 0001:00020bd8       ?GetTooltipManager@CWinAppEx@@QAEPAVCTooltipManager@@XZ 00421bd8 f   mfc90:mfc90.dll
 0001:00020bde       ?GetThisClass@CMFCToolTipCtrl@@SGPAUCRuntimeClass@@XZ 00421bde f   mfc90:mfc90.dll
 0001:00020be4       ?InitTooltipManager@CWinAppEx@@QAEHXZ 00421be4 f   mfc90:mfc90.dll
 0001:00020bea       ?InitKeyboardManager@CWinAppEx@@QAEHXZ 00421bea f   mfc90:mfc90.dll
 0001:00020bf0       ?InitContextMenuManager@CWinAppEx@@QAEHXZ 00421bf0 f   mfc90:mfc90.dll
 0001:00020bf6       ?LoadStdProfileSettings@CWinApp@@IAEXI@Z 00421bf6 f   mfc90:mfc90.dll
 0001:00020bfc       ?SetRegistryKey@CWinApp@@IAEXPBD@Z 00421bfc f   mfc90:mfc90.dll
 0001:00020c02       ?AfxEnableControlContainer@@YAXPAVCOccManager@@@Z 00421c02 f   mfc90:mfc90.dll
 0001:00020c08       ?AfxMessageBox@@YGHIII@Z   00421c08 f   mfc90:mfc90.dll
 0001:00020c0e       ?AfxOleInit@@YGHXZ         00421c0e f   mfc90:mfc90.dll
 0001:00020c14       ?InitInstance@CWinApp@@UAEHXZ 00421c14 f   mfc90:mfc90.dll
 0001:00020c1a       ?AfxInitRichEdit@@YGHXZ    00421c1a f   mfc90:mfc90.dll
 0001:00020c20       ?AddMenu@CContextMenuManager@@QAEHPBDI@Z 00421c20 f   mfc90:mfc90.dll
 0001:00020c26       ?GetContextMenuManager@CWinAppEx@@QAEPAVCContextMenuManager@@XZ 00421c26 f   mfc90:mfc90.dll
 0001:00020c2c       ?ExitInstance@CWinAppEx@@UAEHXZ 00421c2c f   mfc90:mfc90.dll
 0001:00020c32       ??0COleVariant@@QAE@ABUtagVARIANT@@@Z 00421c32 f   mfc90:mfc90.dll
 0001:00020c38       ?GetThisClass@CFrameWndEx@@SGPAUCRuntimeClass@@XZ 00421c38 f   mfc90:mfc90.dll
 0001:00020c3e       ?GetThisMessageMap@CFrameWndEx@@KGPBUAFX_MSGMAP@@XZ 00421c3e f   mfc90:mfc90.dll
 0001:00020c44       ??1CMFCToolBarImages@@UAE@XZ 00421c44 f   mfc90:mfc90.dll
 0001:00020c4a       ??1CMFCStatusBar@@UAE@XZ   00421c4a f   mfc90:mfc90.dll
 0001:00020c50       ??1CMFCToolBar@@UAE@XZ     00421c50 f   mfc90:mfc90.dll
 0001:00020c56       ??1CMFCMenuBar@@UAE@XZ     00421c56 f   mfc90:mfc90.dll
 0001:00020c5c       ??1CFrameWndEx@@MAE@XZ     00421c5c f   mfc90:mfc90.dll
 0001:00020c62       ?GetInt@CWinAppEx@@QAEHPBDH@Z 00421c62 f   mfc90:mfc90.dll
 0001:00020c68       ??0CMFCToolBarImages@@QAE@XZ 00421c68 f   mfc90:mfc90.dll
 0001:00020c6e       ??0CMFCStatusBar@@QAE@XZ   00421c6e f   mfc90:mfc90.dll
 0001:00020c74       ??0CMFCToolBar@@QAE@XZ     00421c74 f   mfc90:mfc90.dll
 0001:00020c7a       ??0CMFCMenuBar@@QAE@XZ     00421c7a f   mfc90:mfc90.dll
 0001:00020c80       ??0CFrameWndEx@@IAE@XZ     00421c80 f   mfc90:mfc90.dll
 0001:00020c86       ?OnCmdMsg@CFrameWndEx@@UAEHIHPAXPAUAFX_CMDHANDLERINFO@@@Z 00421c86 f   mfc90:mfc90.dll
 0001:00020c8c       ?GetMenu@CFrameWnd@@UBEPAVCMenu@@XZ 00421c8c f   mfc90:mfc90.dll
 0001:00020c92       ?SetMenu@CFrameWnd@@UAEHPAVCMenu@@@Z 00421c92 f   mfc90:mfc90.dll
 0001:00020c98       ?WinHelpA@CFrameWndEx@@UAEXKI@Z 00421c98 f   mfc90:mfc90.dll
 0001:00020c9e       ?HtmlHelpA@CFrameWndEx@@MAEXKI@Z 00421c9e f   mfc90:mfc90.dll
 0001:00020ca4       ?OnCommand@CFrameWndEx@@MAEHIJ@Z 00421ca4 f   mfc90:mfc90.dll
 0001:00020caa       ?BeginModalState@CFrameWnd@@UAEXXZ 00421caa f   mfc90:mfc90.dll
 0001:00020cb0       ?EndModalState@CFrameWnd@@UAEXXZ 00421cb0 f   mfc90:mfc90.dll
 0001:00020cb6       ?PreTranslateMessage@CFrameWndEx@@UAEHPAUtagMSG@@@Z 00421cb6 f   mfc90:mfc90.dll
 0001:00020cbc       ?PostNcDestroy@CFrameWnd@@MAEXXZ 00421cbc f   mfc90:mfc90.dll
 0001:00020cc2       ?IsFrameWnd@CFrameWnd@@UBEHXZ 00421cc2 f   mfc90:mfc90.dll
 0001:00020cc8       ?Create@CFrameWnd@@UAEHPBD0KABUtagRECT@@PAVCWnd@@0KPAUCCreateContext@@@Z 00421cc8 f   mfc90:mfc90.dll
 0001:00020cce       ?GetActiveDocument@CFrameWnd@@UAEPAVCDocument@@XZ 00421cce f   mfc90:mfc90.dll
 0001:00020cd4       ?GetActiveFrame@CFrameWnd@@UAEPAV1@XZ 00421cd4 f   mfc90:mfc90.dll
 0001:00020cda       ?GetMessageString@CFrameWnd@@UBEXIAAV?$CStringT@DV?$StrTraitMFC_DLL@DV?$ChTraitsCRT@D@ATL@@@@@ATL@@@Z 00421cda f   mfc90:mfc90.dll
 0001:00020ce0       ?RecalcLayout@CFrameWndEx@@UAEXH@Z 00421ce0 f   mfc90:mfc90.dll
 0001:00020ce6       ?ActivateFrame@CFrameWnd@@UAEXH@Z 00421ce6 f   mfc90:mfc90.dll
 0001:00020cec       ?SetMenuBarVisibility@CFrameWnd@@UAEXK@Z 00421cec f   mfc90:mfc90.dll
 0001:00020cf2       ?GetMenuBarVisibility@CFrameWnd@@UBEKXZ 00421cf2 f   mfc90:mfc90.dll
 0001:00020cf8       ?SetMenuBarState@CFrameWnd@@UAEHK@Z 00421cf8 f   mfc90:mfc90.dll
 0001:00020cfe       ?GetMenuBarState@CFrameWnd@@UBEKXZ 00421cfe f   mfc90:mfc90.dll
 0001:00020d04       ?OnSetPreviewMode@CFrameWndEx@@UAEXHPAUCPrintPreviewState@@@Z 00421d04 f   mfc90:mfc90.dll
 0001:00020d0a       ?GetMessageBar@CFrameWnd@@UAEPAVCWnd@@XZ 00421d0a f   mfc90:mfc90.dll
 0001:00020d10       ?NegotiateBorderSpace@CFrameWndEx@@UAEHIPAUtagRECT@@@Z 00421d10 f   mfc90:mfc90.dll
 0001:00020d16       ?OnCreateClient@CFrameWnd@@MAEHPAUtagCREATESTRUCTA@@PAUCCreateContext@@@Z 00421d16 f   mfc90:mfc90.dll
 0001:00020d1c       ?OnUpdateFrameTitle@CFrameWndEx@@UAEXH@Z 00421d1c f   mfc90:mfc90.dll
 0001:00020d22       ?OnUpdateFrameMenu@CFrameWndEx@@UAEXPAUHMENU__@@@Z 00421d22 f   mfc90:mfc90.dll
 0001:00020d28       ?GetDefaultAccelerator@CFrameWnd@@UAEPAUHACCEL__@@XZ 00421d28 f   mfc90:mfc90.dll
 0001:00020d2e       ?DelayUpdateFrameMenu@CFrameWndEx@@UAEXPAUHMENU__@@@Z 00421d2e f   mfc90:mfc90.dll
 0001:00020d34       ?ExitHelpMode@CFrameWnd@@UAEXXZ 00421d34 f   mfc90:mfc90.dll
 0001:00020d3a       ?OnShowMenuBar@CFrameWnd@@MAEXXZ 00421d3a f   mfc90:mfc90.dll
 0001:00020d40       ?OnHideMenuBar@CFrameWnd@@MAEXXZ 00421d40 f   mfc90:mfc90.dll
 0001:00020d46       ?AdjustDockingLayout@CFrameWndEx@@UAEXPAX@Z 00421d46 f   mfc90:mfc90.dll
 0001:00020d4c       ?OnMoveMiniFrame@CFrameWndEx@@UAEHPAVCWnd@@@Z 00421d4c f   mfc90:mfc90.dll
 0001:00020d52       ?AdjustClientArea@CFrameWndEx@@MAEXXZ 00421d52 f   mfc90:mfc90.dll
 0001:00020d58       ?GetInPlaceActiveItem@CFrameWndEx@@MAEPAVCOleClientItem@@XZ 00421d58 f   mfc90:mfc90.dll
 0001:00020d5e       ?OnShowPopupMenu@CFrameWndEx@@UAEHPAVCMFCPopupMenu@@@Z 00421d5e f   mfc90:mfc90.dll
 0001:00020d64       ?OnClosePopupMenu@CFrameWndEx@@UAEXPAVCMFCPopupMenu@@@Z 00421d64 f   mfc90:mfc90.dll
 0001:00020d6a       ?OnDrawMenuImage@CFrameWndEx@@UAEHPAVCDC@@PBVCMFCToolBarMenuButton@@ABVCRect@@@Z 00421d6a f   mfc90:mfc90.dll
 0001:00020d70       ?OnShowPanes@CFrameWndEx@@UAEHH@Z 00421d70 f   mfc90:mfc90.dll
 0001:00020d76       ?OnCreate@CFrameWndEx@@QAEHPAUtagCREATESTRUCTA@@@Z 00421d76 f   mfc90:mfc90.dll
 0001:00020d7c       ?AfxRegisterWndClass@@YGPBDIPAUHICON__@@PAUHBRUSH__@@0@Z 00421d7c f   mfc90:mfc90.dll
 0001:00020d82       ?PreCreateWindow@CFrameWndEx@@MAEHAAUtagCREATESTRUCTA@@@Z 00421d82 f   mfc90:mfc90.dll
 0001:00020d88       ?EnableUserDefinedToolbars@CMFCToolBarsCustomizeDialog@@QAEXH@Z 00421d88 f   mfc90:mfc90.dll
 0001:00020d8e       ??0CMFCToolBarsCustomizeDialog@@QAE@PAVCFrameWnd@@HIPAV?$CList@PAUCRuntimeClass@@PAU1@@@@Z 00421d8e f   mfc90:mfc90.dll
 0001:00020d94       ?EnableCustomizeButton@CMFCToolBar@@QAEXHHABV?$CStringT@DV?$StrTraitMFC_DLL@DV?$ChTraitsCRT@D@ATL@@@@@ATL@@H@Z 00421d94 f   mfc90:mfc90.dll
 0001:00020d9a       ?OnToolbarCreateNew@CFrameWndEx@@QAEJIJ@Z 00421d9a f   mfc90:mfc90.dll
 0001:00020da0       ?WriteInt@CWinAppEx@@QAEHPBDH@Z 00421da0 f   mfc90:mfc90.dll
 0001:00020da6       ?GetThisClass@CMFCVisualManagerOffice2007@@SGPAUCRuntimeClass@@XZ 00421da6 f   mfc90:mfc90.dll
 0001:00020dac       ?SetStyle@CMFCVisualManagerOffice2007@@SGHW4Style@1@PBD@Z 00421dac f   mfc90:mfc90.dll
 0001:00020db2       ?GetThisClass@CMFCVisualManagerVS2005@@SGPAUCRuntimeClass@@XZ 00421db2 f   mfc90:mfc90.dll
 0001:00020db8       ?SetDockingMode@CDockingManager@@SGXW4AFX_DOCK_TYPE@@@Z 00421db8 f   mfc90:mfc90.dll
 0001:00020dbe       ?GetThisClass@CMFCVisualManagerOffice2003@@SGPAUCRuntimeClass@@XZ 00421dbe f   mfc90:mfc90.dll
 0001:00020dc4       ?GetThisClass@CMFCVisualManagerWindows@@SGPAUCRuntimeClass@@XZ 00421dc4 f   mfc90:mfc90.dll
 0001:00020dca       ?GetThisClass@CMFCVisualManagerOfficeXP@@SGPAUCRuntimeClass@@XZ 00421dca f   mfc90:mfc90.dll
 0001:00020dd0       ?SetDefaultManager@CMFCVisualManager@@SGXPAUCRuntimeClass@@@Z 00421dd0 f   mfc90:mfc90.dll
 0001:00020dd6       ?GetThisClass@CMFCVisualManager@@SGPAUCRuntimeClass@@XZ 00421dd6 f   mfc90:mfc90.dll
 0001:00020ddc       ?LoadFrame@CFrameWndEx@@UAEHIKPAVCWnd@@PAUCCreateContext@@@Z 00421ddc f   mfc90:mfc90.dll
 0001:00020de2       ?TrackPopupMenu@CMenu@@QAEHIHHPAVCWnd@@PBUtagRECT@@@Z 00421de2 f   mfc90:mfc90.dll
 0001:00020de8       ?ClientToScreen@CWnd@@QBEXPAUtagRECT@@@Z 00421de8 f   mfc90:mfc90.dll
 0001:00020dee       ??1CStringArray@@UAE@XZ    00421dee f   mfc90:mfc90.dll
 0001:00020df4       ??0CStringArray@@QAE@XZ    00421df4 f   mfc90:mfc90.dll
 0001:00020dfa       ?OnClose@CFrameWnd@@IAEXXZ 00421dfa f   mfc90:mfc90.dll
 0001:00020e00       ?OnDestroy@CFrameWnd@@IAEXXZ 00421e00 f   mfc90:mfc90.dll
 0001:00020e06       ?AddTail@CStringList@@QAEPAU__POSITION@@PBD@Z 00421e06 f   mfc90:mfc90.dll
 0001:00020e0c       ?RemoveHead@CPtrList@@QAEPAXXZ 00421e0c f   mfc90:mfc90.dll
 0001:00020e12       ?AddTail@CPtrList@@QAEPAU__POSITION@@PAX@Z 00421e12 f   mfc90:mfc90.dll
 0001:00020e18       ?AfxThrowOleException@@YGXJ@Z 00421e18 f   mfc90:mfc90.dll
 0001:00020e1e       ?GetRuntimeClass@CMenu@@UBEPAUCRuntimeClass@@XZ 00421e1e f   mfc90:mfc90.dll
 0001:00020e24       ?DrawItem@CMenu@@UAEXPAUtagDRAWITEMSTRUCT@@@Z 00421e24 f   mfc90:mfc90.dll
 0001:00020e2a       ?MeasureItem@CMenu@@UAEXPAUtagMEASUREITEMSTRUCT@@@Z 00421e2a f   mfc90:mfc90.dll
 0001:00020e30       ?DestroyMenu@CMenu@@QAEHXZ 00421e30 f   mfc90:mfc90.dll
 0001:00020e36       ?FromHandle@CMenu@@SGPAV1@PAUHMENU__@@@Z 00421e36 f   mfc90:mfc90.dll
 0001:00020e3c       ?Attach@CMenu@@QAEHPAUHMENU__@@@Z 00421e3c f   mfc90:mfc90.dll
 0001:00020e42       ?AfxFindResourceHandle@@YGPAUHINSTANCE__@@PBD0@Z 00421e42 f   mfc90:mfc90.dll
 0001:00020e48       ?FromHandle@CWnd@@SGPAV1@PAUHWND__@@@Z 00421e48 f   mfc90:mfc90.dll
 0001:00020e4e       ?BeginWaitCursor@CCmdTarget@@QAEXXZ 00421e4e f   mfc90:mfc90.dll
 0001:00020e54       ?EndWaitCursor@CCmdTarget@@QAEXXZ 00421e54 f   mfc90:mfc90.dll
 0001:00020e5a       ?GetUserToolBarByIndex@CFrameImpl@@IBEPAVCMFCToolBar@@H@Z 00421e5a f   mfc90:mfc90.dll
 0001:00020e60       ?AddDefaultButtonsToCustomizePane@CFrameImpl@@IAEXPAVCMFCPopupMenu@@I@Z 00421e60 f   mfc90:mfc90.dll
 0001:00020e66       ??0CStringList@@QAE@H@Z    00421e66 f   mfc90:mfc90.dll
 0001:00020e6c       ??1CStringList@@UAE@XZ     00421e6c f   mfc90:mfc90.dll
 0001:00020e72       ?GetRuntimeClass@CRichEditCtrl@@UBEPAUCRuntimeClass@@XZ 00421e72 f   mfc90:mfc90.dll
 0001:00020e78       ??1CRichEditCtrl@@UAE@XZ   00421e78 f   mfc90:mfc90.dll
 0001:00020e7e       ?GetThisMessageMap@CWnd@@KGPBUAFX_MSGMAP@@XZ 00421e7e f   mfc90:mfc90.dll
 0001:00020e84       ?CanPaste@CRichEditCtrl@@QBEHI@Z 00421e84 f   mfc90:mfc90.dll
 0001:00020e8a       ?GetStyle@CWnd@@QBEKXZ     00421e8a f   mfc90:mfc90.dll
 0001:00020e90       ?DDX_Text@@YGXPAVCDataExchange@@HAAH@Z 00421e90 f   mfc90:mfc90.dll
 0001:00020e96       ??1CMapStringToString@@UAE@XZ 00421e96 f   mfc90:mfc90.dll
 0001:00020e9c       ?GetNextAssoc@CMapStringToString@@QBEXAAPAU__POSITION@@AAV?$CStringT@DV?$StrTraitMFC_DLL@DV?$ChTraitsCRT@D@ATL@@@@@ATL@@1@Z 00421e9c f   mfc90:mfc90.dll
 0001:00020ea2       ?Lookup@CMapStringToString@@QBEHPBDAAV?$CStringT@DV?$StrTraitMFC_DLL@DV?$ChTraitsCRT@D@ATL@@@@@ATL@@@Z 00421ea2 f   mfc90:mfc90.dll
 0001:00020ea8       ??0CMapStringToString@@QAE@H@Z 00421ea8 f   mfc90:mfc90.dll
 0001:00020eae       ??ACMapStringToString@@QAEAAV?$CStringT@DV?$StrTraitMFC_DLL@DV?$ChTraitsCRT@D@ATL@@@@@ATL@@PBD@Z 00421eae f   mfc90:mfc90.dll
 0001:00020eb4       ??1CComboBox@@UAE@XZ       00421eb4 f   mfc90:mfc90.dll
 0001:00020eba       ?DDX_CBString@@YGXPAVCDataExchange@@HAAV?$CStringT@DV?$StrTraitMFC_DLL@DV?$ChTraitsCRT@D@ATL@@@@@ATL@@@Z 00421eba f   mfc90:mfc90.dll
 0001:00020ec0       ?GetRuntimeClass@CComboBox@@UBEPAUCRuntimeClass@@XZ 00421ec0 f   mfc90:mfc90.dll
 0001:00020ec6       ?OnChildNotify@CComboBox@@MAEHIIJPAJ@Z 00421ec6 f   mfc90:mfc90.dll
 0001:00020ecc       ?Create@CComboBox@@UAEHKABUtagRECT@@PAVCWnd@@I@Z 00421ecc f   mfc90:mfc90.dll
 0001:00020ed2       ?DrawItem@CComboBox@@UAEXPAUtagDRAWITEMSTRUCT@@@Z 00421ed2 f   mfc90:mfc90.dll
 0001:00020ed8       ?MeasureItem@CComboBox@@UAEXPAUtagMEASUREITEMSTRUCT@@@Z 00421ed8 f   mfc90:mfc90.dll
 0001:00020ede       ?CompareItem@CComboBox@@UAEHPAUtagCOMPAREITEMSTRUCT@@@Z 00421ede f   mfc90:mfc90.dll
 0001:00020ee4       ?DeleteItem@CComboBox@@UAEXPAUtagDELETEITEMSTRUCT@@@Z 00421ee4 f   mfc90:mfc90.dll
 0001:00020eea       ?Close@CStdioFile@@UAEXXZ  00421eea f   mfc90:mfc90.dll
 0001:00020ef0       ?Flush@CStdioFile@@UAEXXZ  00421ef0 f   mfc90:mfc90.dll
 0001:00020ef6       ?WriteString@CStdioFile@@UAEXPBD@Z 00421ef6 f   mfc90:mfc90.dll
 0001:00020efc       ??1CStdioFile@@UAE@XZ      00421efc f   mfc90:mfc90.dll
 0001:00020f02       ?Open@CStdioFile@@UAEHPBDIPAVCFileException@@@Z 00421f02 f   mfc90:mfc90.dll
 0001:00020f08       ??0CStdioFile@@QAE@XZ      00421f08 f   mfc90:mfc90.dll
 0001:00020f0e       ?AddHead@CPtrList@@QAEPAU__POSITION@@PAX@Z 00421f0e f   mfc90:mfc90.dll
 0001:00020f14       ?RemoveAt@CPtrList@@QAEXPAU__POSITION@@@Z 00421f14 f   mfc90:mfc90.dll
 0001:00020f1a       ?ReadString@CStdioFile@@UAEHAAV?$CStringT@DV?$StrTraitMFC_DLL@DV?$ChTraitsCRT@D@ATL@@@@@ATL@@@Z 00421f1a f   mfc90:mfc90.dll
 0001:00020f20       ___CxxFrameHandler3        00421f20 f   msvcrt:MSVCR90.dll
 0001:00020f26       @__security_check_cookie@4 00421f26 f   msvcrt:secchk.obj
 0001:00020f35       ??_Etype_info@@UAEPAXI@Z   00421f35 f i msvcrt:ti_inst.obj
 0001:00020f82       _memset                    00421f82 f   msvcrt:MSVCR90.dll
 0001:00020f88       __except_handler4          00421f88 f   msvcrt:chandler4gs.obj
 0001:00020fad       ?__ArrayUnwind@@YGXPAXIHP6EX0@Z@Z 00421fad f   msvcrt:ehvecdtr.obj
 0001:0002100b       ??_M@YGXPAXIHP6EX0@Z@Z     0042200b f   msvcrt:ehvecdtr.obj
 0001:00021070       __alloca_probe             00422070     msvcrt:chkstk.obj
 0001:00021070       __chkstk                   00422070 f   msvcrt:chkstk.obj
 0001:0002109b       __onexit                   0042209b f   msvcrt:atonexit.obj
 0001:00021140       _atexit                    00422140 f   msvcrt:atonexit.obj
 0001:00021160       __alldiv                   00422160 f   msvcrt:lldiv.obj
 0001:0002120a       _free                      0042220a f   msvcrt:MSVCR90.dll
 0001:00021210       _malloc                    00422210 f   msvcrt:MSVCR90.dll
 0001:00021216       _memcpy                    00422216 f   msvcrt:MSVCR90.dll
 0001:00021527       _WinMainCRTStartup         00422527 f   msvcrt:crtexew.obj
 0001:00021540       __ftol2_sse                00422540 f   msvcrt:ftol2.obj
 0001:00021549       __ftol2_pentium4           00422549 f   msvcrt:ftol2.obj
 0001:0002155c       __ftol2_sse_excpt          0042255c f   msvcrt:ftol2.obj
 0001:00021576       __ftol2                    00422576 f   msvcrt:ftol2.obj
 0001:000215eb       ___report_gsfailure        004225eb f   msvcrt:gs_report.obj
 0001:000216f2       __except_handler4_common   004226f2 f   msvcrt:MSVCR90.dll
 0001:000216f8       ?terminate@@YAXXZ          004226f8 f   msvcrt:MSVCR90.dll
 0001:00021700       __SEH_prolog4              00422700 f   msvcrt:sehprolg4.obj
 0001:00021745       __SEH_epilog4              00422745 f   msvcrt:sehprolg4.obj
 0001:0002175a       __unlock                   0042275a f   msvcrt:MSVCR90.dll
 0001:00021760       ___dllonexit               00422760 f   msvcrt:MSVCR90.dll
 0001:00021766       __lock                     00422766 f   msvcrt:MSVCR90.dll
 0001:0002176c       ?__CxxUnhandledExceptionFilter@@YGJPAU_EXCEPTION_POINTERS@@@Z 0042276c f   msvcrt:unhandld.obj
 0001:000217ae       ___CxxSetUnhandledExceptionFilter 004227ae f   msvcrt:unhandld.obj
 0001:000217bc       __amsg_exit                004227bc f   msvcrt:MSVCR90.dll
 0001:000217c2       __RTC_Initialize           004227c2 f   msvcrt:_initsect_.obj
 0001:000217e8       __RTC_Terminate            004227e8 f   msvcrt:_initsect_.obj
 0001:0002180e       __XcptFilter               0042280e f   msvcrt:MSVCR90.dll
 0001:00021820       __ValidateImageBase        00422820 f   msvcrt:pesect.obj
 0001:00021860       __FindPESection            00422860 f   msvcrt:pesect.obj
 0001:000218b0       __IsNonwritableInCurrentImage 004228b0 f   msvcrt:pesect.obj
 0001:0002196e       __initterm                 0042296e f   msvcrt:MSVCR90.dll
 0001:00021974       __initterm_e               00422974 f   msvcrt:MSVCR90.dll
 0001:0002197a       __setdefaultprecision      0042297a f   msvcrt:fp8.obj
 0001:000219a5       __matherr                  004229a5 f   msvcrt:merr.obj
 0001:000219a5       __setargv                  004229a5 f   msvcrt:dllargv.obj
 0001:000219a8       ___security_init_cookie    004229a8 f   msvcrt:gs_support.obj
 0001:00021a8e       __get_sse2_info            00422a8e f   msvcrt:cpu_disp.obj
 0001:00021af0       ___sse2_available_init     00422af0 f   msvcrt:cpu_disp.obj
 0001:00021afe       __crt_debugger_hook        00422afe f   msvcrt:MSVCR90.dll
 0001:00021b04       ?_type_info_dtor_internal_method@type_info@@QAEXXZ 00422b04 f   msvcrt:MSVCR90.dll
 0001:00021b04       ??1type_info@@UAE@XZ       00422b04 f   msvcrt:MSVCR90.dll
 0001:00021b0a       __invoke_watson            00422b0a f   msvcrt:MSVCR90.dll
 0001:00021b10       __controlfp_s              00422b10 f   msvcrt:MSVCR90.dll
 0001:00021b16       _Process32Next@8           00422b16 f   kernel32:KERNEL32.dll
 0001:00021b1c       _Process32First@8          00422b1c f   kernel32:KERNEL32.dll
 0001:00021b22       _CreateToolhelp32Snapshot@8 00422b22 f   kernel32:KERNEL32.dll
 0001:00021b30       ?_com_issue_error@@YGXJ@Z  00422b30 f   comsuppw:comsupp.obj
 0001:00021b50       ?ConvertStringToBSTR@_com_util@@YGPA_WPBD@Z 00422b50 f   comsuppw:comutil.obj
 0001:00021cd0       ??1_com_error@@UAE@XZ      00422cd0 f i comsuppw:comraise.obj
 0001:00021d10       ?_com_raise_error@@YGXJPAUIErrorInfo@@@Z 00422d10 f   comsuppw:comraise.obj
 0001:00021d50       ??0_com_error@@QAE@ABV0@@Z 00422d50 f i comsuppw:comraise.obj
 0001:00021d90       ??_G_com_error@@UAEPAXI@Z  00422d90 f i comsuppw:comraise.obj
 0001:00021d90       ??_E_com_error@@UAEPAXI@Z  00422d90 f i comsuppw:comraise.obj
 0001:00021de0       _VerQueryValueA@16         00422de0 f   Version:VERSION.dll
 0001:00021de6       _GetFileVersionInfoA@16    00422de6 f   Version:VERSION.dll
 0001:00021dec       _GetFileVersionInfoSizeA@8 00422dec f   Version:VERSION.dll
 0001:00021df2       _CtlUsb                    00422df2 f   UsbControl:UsbControl.dll
 0001:00021df8       _WTSRegisterSessionNotification@8 00422df8 f   Wtsapi32:WTSAPI32.dll
 0001:00021dfe       _WTSUnRegisterSessionNotification@4 00422dfe f   Wtsapi32:WTSAPI32.dll
 0001:00021e04       ?HTS_LiveStart@@YGKPAKKHHH@Z 00422e04 f   htsapi:HTSAPI.dll
 0001:00021e0a       ?HTS_Init@@YGKHKKKKPADH@Z  00422e0a f   htsapi:HTSAPI.dll
 0001:00021e10       ?HTS_Uninit@@YGKXZ         00422e10 f   htsapi:HTSAPI.dll
 0001:00021e16       ?HTS_LiveStop@@YGKXZ       00422e16 f   htsapi:HTSAPI.dll
 0001:00021e1c       ?HTS_SetWindowText@@YGKPAD@Z 00422e1c f   htsapi:HTSAPI.dll
 0001:00021e22       _GetAdaptersInfo@8         00422e22 f   Iphlpapi:IPHLPAPI.DLL
 0001:00021e28       _WinMain@16                00422e28 f   mfcs90:appmodul.obj
 0001:00021e33       ?AfxInitialize@@YGHHK@Z    00422e33 f   mfcs90:appmodul.obj
 0001:00021e60       __alloca_probe_16          00422e60 f   msvcrt:alloca16.obj
 0001:00021e76       __alloca_probe_8           00422e76     msvcrt:alloca16.obj
 0001:00021e8c       __CxxThrowException@8      00422e8c f   msvcrt:MSVCR90.dll
 0001:00021e92       ?AfxWinMain@@YGHPAUHINSTANCE__@@0PADH@Z 00422e92 f   mfc90:mfc90.dll
 0002:00000000       __imp__RegCloseKey@4       00426000     advapi32:ADVAPI32.dll
 0002:00000004       __imp__RegQueryValueExA@24 00426004     advapi32:ADVAPI32.dll
 0002:00000008       __imp__RegOpenKeyExA@20    00426008     advapi32:ADVAPI32.dll
 0002:0000000c       __imp__RegEnumKeyExA@32    0042600c     advapi32:ADVAPI32.dll
 0002:00000010       __imp__RegQueryInfoKeyA@48 00426010     advapi32:ADVAPI32.dll
 0002:00000014       __imp__AdjustTokenPrivileges@24 00426014     advapi32:ADVAPI32.dll
 0002:00000018       __imp__LookupPrivilegeValueA@12 00426018     advapi32:ADVAPI32.dll
 0002:0000001c       __imp__OpenProcessToken@12 0042601c     advapi32:ADVAPI32.dll
 0002:00000020       __imp__RegFlushKey@4       00426020     advapi32:ADVAPI32.dll
 0002:00000024       __imp__RegSetValueExA@24   00426024     advapi32:ADVAPI32.dll
 0002:00000028       __imp__RegCreateKeyExA@36  00426028     advapi32:ADVAPI32.dll
 0002:0000002c       \177ADVAPI32_NULL_THUNK_DATA 0042602c     advapi32:ADVAPI32.dll
 0002:00000030       __imp__InitCommonControlsEx@4 00426030     comctl32:COMCTL32.dll
 0002:00000034       \177COMCTL32_NULL_THUNK_DATA 00426034     comctl32:COMCTL32.dll
 0002:00000038       __imp_?HTS_Init@@YGKHKKKKPADH@Z 00426038     htsapi:HTSAPI.dll
 0002:0000003c       __imp_?HTS_SetWindowText@@YGKPAD@Z 0042603c     htsapi:HTSAPI.dll
 0002:00000040       __imp_?HTS_LiveStop@@YGKXZ 00426040     htsapi:HTSAPI.dll
 0002:00000044       __imp_?HTS_Uninit@@YGKXZ   00426044     htsapi:HTSAPI.dll
 0002:00000048       __imp_?HTS_LiveStart@@YGKPAKKHHH@Z 00426048     htsapi:HTSAPI.dll
 0002:0000004c       \177HTSAPI_NULL_THUNK_DATA 0042604c     htsapi:HTSAPI.dll
 0002:00000050       __imp_??1CKeyboradLock@@UAE@XZ 00426050     hook:Hook.dll
 0002:00000054       __imp_?CtrlAltDel_Enable_Disable@CKeyboradLock@@QAEHH@Z 00426054     hook:Hook.dll
 0002:00000058       __imp_?StopHook@CKeyboradLock@@QAEHXZ 00426058     hook:Hook.dll
 0002:0000005c       __imp_?StartHook@CKeyboradLock@@QAEHXZ 0042605c     hook:Hook.dll
 0002:00000060       __imp_??0CKeyboradLock@@QAE@XZ 00426060     hook:Hook.dll
 0002:00000064       __imp_??0CMouseLock@@QAE@XZ 00426064     hook:Hook.dll
 0002:00000068       __imp_?StartHook@CMouseLock@@QAEHXZ 00426068     hook:Hook.dll
 0002:0000006c       __imp_?StopHook@CMouseLock@@QAEHXZ 0042606c     hook:Hook.dll
 0002:00000070       __imp_??1CMouseLock@@UAE@XZ 00426070     hook:Hook.dll
 0002:00000074       __imp_?LockAll@CKeyboradLock@@QAEXH@Z 00426074     hook:Hook.dll
 0002:00000078       __imp_?LockAll@CMouseLock@@QAEXH@Z 00426078     hook:Hook.dll
 0002:0000007c       \177Hook_NULL_THUNK_DATA   0042607c     hook:Hook.dll
 0002:00000080       __imp__GetAdaptersInfo@8   00426080     Iphlpapi:IPHLPAPI.DLL
 0002:00000084       \177IPHLPAPI_NULL_THUNK_DATA 00426084     Iphlpapi:IPHLPAPI.DLL
 0002:00000088       __imp__DeviceIoControl@32  00426088     kernel32:KERNEL32.dll
 0002:0000008c       __imp__GetCurrentProcessId@0 0042608c     kernel32:KERNEL32.dll
 0002:00000090       __imp__OpenProcess@12      00426090     kernel32:KERNEL32.dll
 0002:00000094       __imp__CreateProcessA@40   00426094     kernel32:KERNEL32.dll
 0002:00000098       __imp__SetLocalTime@4      00426098     kernel32:KERNEL32.dll
 0002:0000009c       __imp__GetSystemDirectoryA@8 0042609c     kernel32:KERNEL32.dll
 0002:000000a0       __imp__WTSGetActiveConsoleSessionId@0 004260a0     kernel32:KERNEL32.dll
 0002:000000a4       __imp__GetComputerNameA@8  004260a4     kernel32:KERNEL32.dll
 0002:000000a8       __imp__CreateEventA@16     004260a8     kernel32:KERNEL32.dll
 0002:000000ac       __imp__DefineDosDeviceA@12 004260ac     kernel32:KERNEL32.dll
 0002:000000b0       __imp__InterlockedDecrement@4 004260b0     kernel32:KERNEL32.dll
 0002:000000b4       __imp__lstrcatA@8          004260b4     kernel32:KERNEL32.dll
 0002:000000b8       __imp__WideCharToMultiByte@32 004260b8     kernel32:KERNEL32.dll
 0002:000000bc       __imp__ResumeThread@4      004260bc     kernel32:KERNEL32.dll
 0002:000000c0       __imp__GetModuleFileNameA@12 004260c0     kernel32:KERNEL32.dll
 0002:000000c4       __imp__GetProcessHeap@0    004260c4     kernel32:KERNEL32.dll
 0002:000000c8       __imp__HeapFree@12         004260c8     kernel32:KERNEL32.dll
 0002:000000cc       __imp__SetCurrentDirectoryA@4 004260cc     kernel32:KERNEL32.dll
 0002:000000d0       __imp__CreateFileA@28      004260d0     kernel32:KERNEL32.dll
 0002:000000d4       __imp__InitializeCriticalSection@4 004260d4     kernel32:KERNEL32.dll
 0002:000000d8       __imp__DeleteCriticalSection@4 004260d8     kernel32:KERNEL32.dll
 0002:000000dc       __imp__EnterCriticalSection@4 004260dc     kernel32:KERNEL32.dll
 0002:000000e0       __imp__LeaveCriticalSection@4 004260e0     kernel32:KERNEL32.dll
 0002:000000e4       __imp__GetLocalTime@4      004260e4     kernel32:KERNEL32.dll
 0002:000000e8       __imp__lstrcpyA@8          004260e8     kernel32:KERNEL32.dll
 0002:000000ec       __imp__FreeLibrary@4       004260ec     kernel32:KERNEL32.dll
 0002:000000f0       __imp__GetProcAddress@8    004260f0     kernel32:KERNEL32.dll
 0002:000000f4       __imp__LoadLibraryA@4      004260f4     kernel32:KERNEL32.dll
 0002:000000f8       __imp__GetModuleHandleA@4  004260f8     kernel32:KERNEL32.dll
 0002:000000fc       __imp__SetEvent@4          004260fc     kernel32:KERNEL32.dll
 0002:00000100       __imp__lstrcmpA@8          00426100     kernel32:KERNEL32.dll
 0002:00000104       __imp__MultiByteToWideChar@24 00426104     kernel32:KERNEL32.dll
 0002:00000108       __imp__lstrlenA@4          00426108     kernel32:KERNEL32.dll
 0002:0000010c       __imp__GetSystemTimeAsFileTime@4 0042610c     kernel32:KERNEL32.dll
 0002:00000110       __imp__GetVersionExA@4     00426110     kernel32:KERNEL32.dll
 0002:00000114       __imp__WaitForSingleObject@8 00426114     kernel32:KERNEL32.dll
 0002:00000118       __imp__Sleep@4             00426118     kernel32:KERNEL32.dll
 0002:0000011c       __imp__GetLastError@0      0042611c     kernel32:KERNEL32.dll
 0002:00000120       __imp__GetCurrentThreadId@0 00426120     kernel32:KERNEL32.dll
 0002:00000124       __imp__GetTickCount@0      00426124     kernel32:KERNEL32.dll
 0002:00000128       __imp__IsDebuggerPresent@0 00426128     kernel32:KERNEL32.dll
 0002:0000012c       __imp__SetUnhandledExceptionFilter@4 0042612c     kernel32:KERNEL32.dll
 0002:00000130       __imp__UnhandledExceptionFilter@4 00426130     kernel32:KERNEL32.dll
 0002:00000134       __imp__GetStartupInfoA@4   00426134     kernel32:KERNEL32.dll
 0002:00000138       __imp__InterlockedCompareExchange@12 00426138     kernel32:KERNEL32.dll
 0002:0000013c       __imp__RaiseException@16   0042613c     kernel32:KERNEL32.dll
 0002:00000140       __imp__InterlockedExchange@8 00426140     kernel32:KERNEL32.dll
 0002:00000144       __imp__QueryPerformanceCounter@4 00426144     kernel32:KERNEL32.dll
 0002:00000148       __imp__CreateToolhelp32Snapshot@8 00426148     kernel32:KERNEL32.dll
 0002:0000014c       __imp__Process32First@8    0042614c     kernel32:KERNEL32.dll
 0002:00000150       __imp__Process32Next@8     00426150     kernel32:KERNEL32.dll
 0002:00000154       __imp__TerminateProcess@8  00426154     kernel32:KERNEL32.dll
 0002:00000158       __imp__LocalAlloc@8        00426158     kernel32:KERNEL32.dll
 0002:0000015c       __imp__GetCurrentProcess@0 0042615c     kernel32:KERNEL32.dll
 0002:00000160       __imp__CreateMutexA@12     00426160     kernel32:KERNEL32.dll
 0002:00000164       __imp__ReleaseMutex@4      00426164     kernel32:KERNEL32.dll
 0002:00000168       __imp__GetPrivateProfileSectionA@16 00426168     kernel32:KERNEL32.dll
 0002:0000016c       __imp__GetPrivateProfileStringA@24 0042616c     kernel32:KERNEL32.dll
 0002:00000170       __imp__GetExitCodeProcess@8 00426170     kernel32:KERNEL32.dll
 0002:00000174       __imp__CloseHandle@4       00426174     kernel32:KERNEL32.dll
 0002:00000178       __imp__DeleteFileA@4       00426178     kernel32:KERNEL32.dll
 0002:0000017c       \177KERNEL32_NULL_THUNK_DATA 0042617c     kernel32:KERNEL32.dll
 0002:00000180       __imp_?CallLock@@YAHV?$CStringT@DV?$StrTraitMFC_DLL@DV?$ChTraitsCRT@D@ATL@@@@@ATL@@@Z 00426180     LockScreen:LockScreen.dll
 0002:00000184       __imp_?CallUnlock@@YAHXZ   00426184     LockScreen:LockScreen.dll
 0002:00000188       \177LockScreen_NULL_THUNK_DATA 00426188     LockScreen:LockScreen.dll
 0002:0000018c       __imp_?_type_info_dtor_internal_method@type_info@@QAEXXZ 0042618c     msvcrt:MSVCR90.dll
 0002:00000190       __imp___crt_debugger_hook  00426190     msvcrt:MSVCR90.dll
 0002:00000194       __imp____set_app_type      00426194     msvcrt:MSVCR90.dll
 0002:00000198       __imp____p__fmode          00426198     msvcrt:MSVCR90.dll
 0002:0000019c       __imp____p__commode        0042619c     msvcrt:MSVCR90.dll
 0002:000001a0       __imp___adjust_fdiv        004261a0     msvcrt:MSVCR90.dll
 0002:000001a4       __imp____setusermatherr    004261a4     msvcrt:MSVCR90.dll
 0002:000001a8       __imp____CxxFrameHandler3  004261a8     msvcrt:MSVCR90.dll
 0002:000001ac       __imp___configthreadlocale 004261ac     msvcrt:MSVCR90.dll
 0002:000001b0       __imp___initterm_e         004261b0     msvcrt:MSVCR90.dll
 0002:000001b4       __imp___initterm           004261b4     msvcrt:MSVCR90.dll
 0002:000001b8       __imp___acmdln             004261b8     msvcrt:MSVCR90.dll
 0002:000001bc       __imp___ismbblead          004261bc     msvcrt:MSVCR90.dll
 0002:000001c0       __imp___XcptFilter         004261c0     msvcrt:MSVCR90.dll
 0002:000001c4       __imp___invoke_watson      004261c4     msvcrt:MSVCR90.dll
 0002:000001c8       __imp___cexit              004261c8     msvcrt:MSVCR90.dll
 0002:000001cc       __imp____getmainargs       004261cc     msvcrt:MSVCR90.dll
 0002:000001d0       __imp___amsg_exit          004261d0     msvcrt:MSVCR90.dll
 0002:000001d4       __imp___decode_pointer     004261d4     msvcrt:MSVCR90.dll
 0002:000001d8       __imp___onexit             004261d8     msvcrt:MSVCR90.dll
 0002:000001dc       __imp___lock               004261dc     msvcrt:MSVCR90.dll
 0002:000001e0       __imp___encode_pointer     004261e0     msvcrt:MSVCR90.dll
 0002:000001e4       __imp____dllonexit         004261e4     msvcrt:MSVCR90.dll
 0002:000001e8       __imp___unlock             004261e8     msvcrt:MSVCR90.dll
 0002:000001ec       __imp_?terminate@@YAXXZ    004261ec     msvcrt:MSVCR90.dll
 0002:000001f0       __imp___except_handler4_common 004261f0     msvcrt:MSVCR90.dll
 0002:000001f4       __imp___mbslwr             004261f4     msvcrt:MSVCR90.dll
 0002:000001f8       __imp___mbsrchr            004261f8     msvcrt:MSVCR90.dll
 0002:000001fc       __imp___controlfp_s        004261fc     msvcrt:MSVCR90.dll
 0002:00000200       __imp___CxxThrowException@8 00426200     msvcrt:MSVCR90.dll
 0002:00000204       __imp___exit               00426204     msvcrt:MSVCR90.dll
 0002:00000208       __imp__fopen_s             00426208     msvcrt:MSVCR90.dll
 0002:0000020c       __imp__fclose              0042620c     msvcrt:MSVCR90.dll
 0002:00000210       __imp__strstr              00426210     msvcrt:MSVCR90.dll
 0002:00000214       __imp__vsprintf_s          00426214     msvcrt:MSVCR90.dll
 0002:00000218       __imp__strcat_s            00426218     msvcrt:MSVCR90.dll
 0002:0000021c       __imp___localtime64_s      0042621c     msvcrt:MSVCR90.dll
 0002:00000220       __imp___time64             00426220     msvcrt:MSVCR90.dll
 0002:00000224       __imp__memcpy              00426224     msvcrt:MSVCR90.dll
 0002:00000228       __imp__atoi                00426228     msvcrt:MSVCR90.dll
 0002:0000022c       __imp__malloc              0042622c     msvcrt:MSVCR90.dll
 0002:00000230       __imp__free                00426230     msvcrt:MSVCR90.dll
 0002:00000234       __imp__exit                00426234     msvcrt:MSVCR90.dll
 0002:00000238       __imp__strncpy_s           00426238     msvcrt:MSVCR90.dll
 0002:0000023c       __imp__wcscpy_s            0042623c     msvcrt:MSVCR90.dll
 0002:00000240       __imp___atoi64             00426240     msvcrt:MSVCR90.dll
 0002:00000244       __imp__sprintf             00426244     msvcrt:MSVCR90.dll
 0002:00000248       __imp__sscanf              00426248     msvcrt:MSVCR90.dll
 0002:0000024c       __imp__strcpy_s            0042624c     msvcrt:MSVCR90.dll
 0002:00000250       __imp__strncpy             00426250     msvcrt:MSVCR90.dll
 0002:00000254       __imp__strncmp             00426254     msvcrt:MSVCR90.dll
 0002:00000258       __imp__memset              00426258     msvcrt:MSVCR90.dll
 0002:0000025c       __imp___setmbcp            0042625c     msvcrt:MSVCR90.dll
 0002:00000260       \177MSVCR90_NULL_THUNK_DATA 00426260     msvcrt:MSVCR90.dll
 0002:00000264       __imp__SafeArrayGetUBound@12 00426264     oleaut32:OLEAUT32.dll
 0002:00000268       __imp__SafeArrayGetLBound@12 00426268     oleaut32:OLEAUT32.dll
 0002:0000026c       __imp__SysFreeString@4     0042626c     oleaut32:OLEAUT32.dll
 0002:00000270       __imp__SysAllocString@4    00426270     oleaut32:OLEAUT32.dll
 0002:00000274       __imp__SafeArrayGetElement@12 00426274     oleaut32:OLEAUT32.dll
 0002:00000278       __imp__VariantClear@4      00426278     oleaut32:OLEAUT32.dll
 0002:0000027c       __imp__VariantInit@4       0042627c     oleaut32:OLEAUT32.dll
 0002:00000280       \177OLEAUT32_NULL_THUNK_DATA 00426280     oleaut32:OLEAUT32.dll
 0002:00000284       __imp__ShutdownWinIo@0     00426284     samio:SAMIO.dll
 0002:00000288       __imp__StrongInitializeWinIo@0 00426288     samio:SAMIO.dll
 0002:0000028c       \177SAMIO_NULL_THUNK_DATA  0042628c     samio:SAMIO.dll
 0002:00000290       __imp__ShellExecuteA@24    00426290     shell32:SHELL32.dll
 0002:00000294       __imp__Shell_NotifyIconA@8 00426294     shell32:SHELL32.dll
 0002:00000298       \177SHELL32_NULL_THUNK_DATA 00426298     shell32:SHELL32.dll
 0002:0000029c       __imp_??1CInstall@@UAE@XZ  0042629c     SPIFilter:SPIFilter.dll
 0002:000002a0       __imp_??0CInstall@@QAE@XZ  004262a0     SPIFilter:SPIFilter.dll
 0002:000002a4       __imp_??1CErrorTable@@UAE@XZ 004262a4     SPIFilter:SPIFilter.dll
 0002:000002a8       __imp_??1CErrorMessage@@UAE@XZ 004262a8     SPIFilter:SPIFilter.dll
 0002:000002ac       \177SPIFilter_NULL_THUNK_DATA 004262ac     SPIFilter:SPIFilter.dll
 0002:000002b0       __imp_?ShowMsgDlg@@YAHV?$CStringT@DV?$StrTraitMFC_DLL@DV?$ChTraitsCRT@D@ATL@@@@@ATL@@0KIHKIKIPAVCWnd@@@Z 004262b0     SendMessage:SendMessage.dll
 0002:000002b4       \177SendMessage_NULL_THUNK_DATA 004262b4     SendMessage:SendMessage.dll
 0002:000002b8       __imp__ExitWindowsEx@8     004262b8     user32:USER32.dll
 0002:000002bc       __imp__EnableMenuItem@12   004262bc     user32:USER32.dll
 0002:000002c0       __imp__AppendMenuA@16      004262c0     user32:USER32.dll
 0002:000002c4       __imp__CreatePopupMenu@0   004262c4     user32:USER32.dll
 0002:000002c8       __imp__GetFocus@0          004262c8     user32:USER32.dll
 0002:000002cc       __imp__KillTimer@8         004262cc     user32:USER32.dll
 0002:000002d0       __imp__SetTimer@16         004262d0     user32:USER32.dll
 0002:000002d4       __imp__RedrawWindow@16     004262d4     user32:USER32.dll
 0002:000002d8       __imp__LoadMenuA@8         004262d8     user32:USER32.dll
 0002:000002dc       __imp__GetSubMenu@8        004262dc     user32:USER32.dll
 0002:000002e0       __imp__wsprintfA           004262e0     user32:USER32.dll
 0002:000002e4       __imp__GetCursorPos@4      004262e4     user32:USER32.dll
 0002:000002e8       __imp__SetForegroundWindow@4 004262e8     user32:USER32.dll
 0002:000002ec       __imp__LoadIconA@8         004262ec     user32:USER32.dll
 0002:000002f0       __imp__RegisterHotKey@16   004262f0     user32:USER32.dll
 0002:000002f4       __imp__UpdateWindow@4      004262f4     user32:USER32.dll
 0002:000002f8       __imp__FindWindowA@8       004262f8     user32:USER32.dll
 0002:000002fc       __imp__MessageBoxA@16      004262fc     user32:USER32.dll
 0002:00000300       __imp__SendMessageA@16     00426300     user32:USER32.dll
 0002:00000304       __imp__EnableWindow@8      00426304     user32:USER32.dll
 0002:00000308       __imp__GetClientRect@8     00426308     user32:USER32.dll
 0002:0000030c       __imp__PostMessageA@16     0042630c     user32:USER32.dll
 0002:00000310       __imp__GetKeyState@4       00426310     user32:USER32.dll
 0002:00000314       \177USER32_NULL_THUNK_DATA 00426314     user32:USER32.dll
 0002:00000318       __imp__CtlUsb              00426318     UsbControl:UsbControl.dll
 0002:0000031c       \177UsbControl_NULL_THUNK_DATA 0042631c     UsbControl:UsbControl.dll
 0002:00000320       __imp__VerQueryValueA@16   00426320     Version:VERSION.dll
 0002:00000324       __imp__GetFileVersionInfoA@16 00426324     Version:VERSION.dll
 0002:00000328       __imp__GetFileVersionInfoSizeA@8 00426328     Version:VERSION.dll
 0002:0000032c       \177VERSION_NULL_THUNK_DATA 0042632c     Version:VERSION.dll
 0002:00000330       __imp__FtpSetCurrentDirectoryA@8 00426330     wininet:WININET.dll
 0002:00000334       __imp__InternetCloseHandle@4 00426334     wininet:WININET.dll
 0002:00000338       __imp__InternetConnectA@32 00426338     wininet:WININET.dll
 0002:0000033c       __imp__InternetOpenA@20    0042633c     wininet:WININET.dll
 0002:00000340       \177WININET_NULL_THUNK_DATA 00426340     wininet:WININET.dll
 0002:00000344       __imp__recvfrom@24         00426344     WS2_32:WS2_32.dll
 0002:00000348       __imp__bind@12             00426348     WS2_32:WS2_32.dll
 0002:0000034c       __imp__WSAAsyncSelect@16   0042634c     WS2_32:WS2_32.dll
 0002:00000350       __imp__sendto@24           00426350     WS2_32:WS2_32.dll
 0002:00000354       __imp__inet_addr@4         00426354     WS2_32:WS2_32.dll
 0002:00000358       __imp__WSAStartup@8        00426358     WS2_32:WS2_32.dll
 0002:0000035c       __imp__socket@12           0042635c     WS2_32:WS2_32.dll
 0002:00000360       __imp__WSAGetLastError@0   00426360     WS2_32:WS2_32.dll
 0002:00000364       __imp__htons@4             00426364     WS2_32:WS2_32.dll
 0002:00000368       __imp__connect@12          00426368     WS2_32:WS2_32.dll
 0002:0000036c       __imp__inet_ntoa@4         0042636c     WS2_32:WS2_32.dll
 0002:00000370       __imp__closesocket@4       00426370     WS2_32:WS2_32.dll
 0002:00000374       __imp__send@16             00426374     WS2_32:WS2_32.dll
 0002:00000378       __imp__recv@16             00426378     WS2_32:WS2_32.dll
 0002:0000037c       __imp__WSACleanup@0        0042637c     WS2_32:WS2_32.dll
 0002:00000380       __imp__setsockopt@20       00426380     WS2_32:WS2_32.dll
 0002:00000384       \177WS2_32_NULL_THUNK_DATA 00426384     WS2_32:WS2_32.dll
 0002:00000388       __imp__WTSUnRegisterSessionNotification@4 00426388     Wtsapi32:WTSAPI32.dll
 0002:0000038c       __imp__WTSRegisterSessionNotification@8 0042638c     Wtsapi32:WTSAPI32.dll
 0002:00000390       \177WTSAPI32_NULL_THUNK_DATA 00426390     Wtsapi32:WTSAPI32.dll
 0002:00000394       __imp_??0CDiskIO@@QAE@H@Z  00426394     diskop:diskop.dll
 0002:00000398       __imp_??1CDiskIO@@QAE@XZ   00426398     diskop:diskop.dll
 0002:0000039c       __imp_?GetPartitionLetter@CDiskIO@@QAEXXZ 0042639c     diskop:diskop.dll
 0002:000003a0       \177diskop_NULL_THUNK_DATA 004263a0     diskop:diskop.dll
 0002:000003a4       __imp_?GetThisClass@CFrameWndEx@@SGPAUCRuntimeClass@@XZ 004263a4     mfc90:mfc90.dll
 0002:000003a8       __imp_?AFX_WM_CREATETOOLBAR@@3IA 004263a8     mfc90:mfc90.dll
 0002:000003ac       __imp_?GetThisMessageMap@CFrameWndEx@@KGPBUAFX_MSGMAP@@XZ 004263ac     mfc90:mfc90.dll
 0002:000003b0       __imp_??1CMFCToolBarImages@@UAE@XZ 004263b0     mfc90:mfc90.dll
 0002:000003b4       __imp_??1CMFCStatusBar@@UAE@XZ 004263b4     mfc90:mfc90.dll
 0002:000003b8       __imp_??1CMFCToolBar@@UAE@XZ 004263b8     mfc90:mfc90.dll
 0002:000003bc       __imp_??1CMFCMenuBar@@UAE@XZ 004263bc     mfc90:mfc90.dll
 0002:000003c0       __imp_??1CFrameWndEx@@MAE@XZ 004263c0     mfc90:mfc90.dll
 0002:000003c4       __imp_?GetInt@CWinAppEx@@QAEHPBDH@Z 004263c4     mfc90:mfc90.dll
 0002:000003c8       __imp_??0CMFCToolBarImages@@QAE@XZ 004263c8     mfc90:mfc90.dll
 0002:000003cc       __imp_??0CMFCStatusBar@@QAE@XZ 004263cc     mfc90:mfc90.dll
 0002:000003d0       __imp_??0CMFCToolBar@@QAE@XZ 004263d0     mfc90:mfc90.dll
 0002:000003d4       __imp_??0CMFCMenuBar@@QAE@XZ 004263d4     mfc90:mfc90.dll
 0002:000003d8       __imp_??0CFrameWndEx@@IAE@XZ 004263d8     mfc90:mfc90.dll
 0002:000003dc       __imp_?OnCmdMsg@CFrameWndEx@@UAEHIHPAXPAUAFX_CMDHANDLERINFO@@@Z 004263dc     mfc90:mfc90.dll
 0002:000003e0       __imp_?GetMenu@CFrameWnd@@UBEPAVCMenu@@XZ 004263e0     mfc90:mfc90.dll
 0002:000003e4       __imp_?SetMenu@CFrameWnd@@UAEHPAVCMenu@@@Z 004263e4     mfc90:mfc90.dll
 0002:000003e8       __imp_?WinHelpA@CFrameWndEx@@UAEXKI@Z 004263e8     mfc90:mfc90.dll
 0002:000003ec       __imp_?HtmlHelpA@CFrameWndEx@@MAEXKI@Z 004263ec     mfc90:mfc90.dll
 0002:000003f0       __imp_?OnCommand@CFrameWndEx@@MAEHIJ@Z 004263f0     mfc90:mfc90.dll
 0002:000003f4       __imp_?BeginModalState@CFrameWnd@@UAEXXZ 004263f4     mfc90:mfc90.dll
 0002:000003f8       __imp_?EndModalState@CFrameWnd@@UAEXXZ 004263f8     mfc90:mfc90.dll
 0002:000003fc       __imp_?PreTranslateMessage@CFrameWndEx@@UAEHPAUtagMSG@@@Z 004263fc     mfc90:mfc90.dll
 0002:00000400       __imp_?PostNcDestroy@CFrameWnd@@MAEXXZ 00426400     mfc90:mfc90.dll
 0002:00000404       __imp_?IsFrameWnd@CFrameWnd@@UBEHXZ 00426404     mfc90:mfc90.dll
 0002:00000408       __imp_?Create@CFrameWnd@@UAEHPBD0KABUtagRECT@@PAVCWnd@@0KPAUCCreateContext@@@Z 00426408     mfc90:mfc90.dll
 0002:0000040c       __imp_?GetActiveDocument@CFrameWnd@@UAEPAVCDocument@@XZ 0042640c     mfc90:mfc90.dll
 0002:00000410       __imp_?GetActiveFrame@CFrameWnd@@UAEPAV1@XZ 00426410     mfc90:mfc90.dll
 0002:00000414       __imp_?GetMessageString@CFrameWnd@@UBEXIAAV?$CStringT@DV?$StrTraitMFC_DLL@DV?$ChTraitsCRT@D@ATL@@@@@ATL@@@Z 00426414     mfc90:mfc90.dll
 0002:00000418       __imp_?RecalcLayout@CFrameWndEx@@UAEXH@Z 00426418     mfc90:mfc90.dll
 0002:0000041c       __imp_?ActivateFrame@CFrameWnd@@UAEXH@Z 0042641c     mfc90:mfc90.dll
 0002:00000420       __imp_?SetMenuBarVisibility@CFrameWnd@@UAEXK@Z 00426420     mfc90:mfc90.dll
 0002:00000424       __imp_?GetMenuBarVisibility@CFrameWnd@@UBEKXZ 00426424     mfc90:mfc90.dll
 0002:00000428       __imp_?SetMenuBarState@CFrameWnd@@UAEHK@Z 00426428     mfc90:mfc90.dll
 0002:0000042c       __imp_?GetMenuBarState@CFrameWnd@@UBEKXZ 0042642c     mfc90:mfc90.dll
 0002:00000430       __imp_?OnSetPreviewMode@CFrameWndEx@@UAEXHPAUCPrintPreviewState@@@Z 00426430     mfc90:mfc90.dll
 0002:00000434       __imp_?GetMessageBar@CFrameWnd@@UAEPAVCWnd@@XZ 00426434     mfc90:mfc90.dll
 0002:00000438       __imp_?NegotiateBorderSpace@CFrameWndEx@@UAEHIPAUtagRECT@@@Z 00426438     mfc90:mfc90.dll
 0002:0000043c       __imp_?OnCreateClient@CFrameWnd@@MAEHPAUtagCREATESTRUCTA@@PAUCCreateContext@@@Z 0042643c     mfc90:mfc90.dll
 0002:00000440       __imp_?OnUpdateFrameMenu@CFrameWndEx@@UAEXPAUHMENU__@@@Z 00426440     mfc90:mfc90.dll
 0002:00000444       __imp_?GetDefaultAccelerator@CFrameWnd@@UAEPAUHACCEL__@@XZ 00426444     mfc90:mfc90.dll
 0002:00000448       __imp_?DelayUpdateFrameMenu@CFrameWndEx@@UAEXPAUHMENU__@@@Z 00426448     mfc90:mfc90.dll
 0002:0000044c       __imp_?ExitHelpMode@CFrameWnd@@UAEXXZ 0042644c     mfc90:mfc90.dll
 0002:00000450       __imp_?OnShowMenuBar@CFrameWnd@@MAEXXZ 00426450     mfc90:mfc90.dll
 0002:00000454       __imp_?AfxWinMain@@YGHPAUHINSTANCE__@@0PADH@Z 00426454     mfc90:mfc90.dll
 0002:00000458       __imp_?AdjustDockingLayout@CFrameWndEx@@UAEXPAX@Z 00426458     mfc90:mfc90.dll
 0002:0000045c       __imp_?OnMoveMiniFrame@CFrameWndEx@@UAEHPAVCWnd@@@Z 0042645c     mfc90:mfc90.dll
 0002:00000460       __imp_?AdjustClientArea@CFrameWndEx@@MAEXXZ 00426460     mfc90:mfc90.dll
 0002:00000464       __imp_?GetInPlaceActiveItem@CFrameWndEx@@MAEPAVCOleClientItem@@XZ 00426464     mfc90:mfc90.dll
 0002:00000468       __imp_?OnShowPopupMenu@CFrameWndEx@@UAEHPAVCMFCPopupMenu@@@Z 00426468     mfc90:mfc90.dll
 0002:0000046c       __imp_?OnClosePopupMenu@CFrameWndEx@@UAEXPAVCMFCPopupMenu@@@Z 0042646c     mfc90:mfc90.dll
 0002:00000470       __imp_?OnDrawMenuImage@CFrameWndEx@@UAEHPAVCDC@@PBVCMFCToolBarMenuButton@@ABVCRect@@@Z 00426470     mfc90:mfc90.dll
 0002:00000474       __imp_?OnShowPanes@CFrameWndEx@@UAEHH@Z 00426474     mfc90:mfc90.dll
 0002:00000478       __imp_?OnCreate@CFrameWndEx@@QAEHPAUtagCREATESTRUCTA@@@Z 00426478     mfc90:mfc90.dll
 0002:0000047c       __imp_?AfxRegisterWndClass@@YGPBDIPAUHICON__@@PAUHBRUSH__@@0@Z 0042647c     mfc90:mfc90.dll
 0002:00000480       __imp_?PreCreateWindow@CFrameWndEx@@MAEHAAUtagCREATESTRUCTA@@@Z 00426480     mfc90:mfc90.dll
 0002:00000484       __imp_?EnableUserDefinedToolbars@CMFCToolBarsCustomizeDialog@@QAEXH@Z 00426484     mfc90:mfc90.dll
 0002:00000488       __imp_??0CMFCToolBarsCustomizeDialog@@QAE@PAVCFrameWnd@@HIPAV?$CList@PAUCRuntimeClass@@PAU1@@@@Z 00426488     mfc90:mfc90.dll
 0002:0000048c       __imp_?EnableCustomizeButton@CMFCToolBar@@QAEXHHABV?$CStringT@DV?$StrTraitMFC_DLL@DV?$ChTraitsCRT@D@ATL@@@@@ATL@@H@Z 0042648c     mfc90:mfc90.dll
 0002:00000490       __imp_?OnToolbarCreateNew@CFrameWndEx@@QAEJIJ@Z 00426490     mfc90:mfc90.dll
 0002:00000494       __imp_?WriteInt@CWinAppEx@@QAEHPBDH@Z 00426494     mfc90:mfc90.dll
 0002:00000498       __imp_?GetThisClass@CMFCVisualManagerOffice2007@@SGPAUCRuntimeClass@@XZ 00426498     mfc90:mfc90.dll
 0002:0000049c       __imp_?SetStyle@CMFCVisualManagerOffice2007@@SGHW4Style@1@PBD@Z 0042649c     mfc90:mfc90.dll
 0002:000004a0       __imp_?GetThisClass@CMFCVisualManagerVS2005@@SGPAUCRuntimeClass@@XZ 004264a0     mfc90:mfc90.dll
 0002:000004a4       __imp_?SetDockingMode@CDockingManager@@SGXW4AFX_DOCK_TYPE@@@Z 004264a4     mfc90:mfc90.dll
 0002:000004a8       __imp_?GetThisClass@CMFCVisualManagerOffice2003@@SGPAUCRuntimeClass@@XZ 004264a8     mfc90:mfc90.dll
 0002:000004ac       __imp_?GetThisClass@CMFCVisualManagerWindows@@SGPAUCRuntimeClass@@XZ 004264ac     mfc90:mfc90.dll
 0002:000004b0       __imp_?m_b3DTabsXPTheme@CMFCVisualManagerWindows@@2HA 004264b0     mfc90:mfc90.dll
 0002:000004b4       __imp_?GetThisClass@CMFCVisualManagerOfficeXP@@SGPAUCRuntimeClass@@XZ 004264b4     mfc90:mfc90.dll
 0002:000004b8       __imp_?SetDefaultManager@CMFCVisualManager@@SGXPAUCRuntimeClass@@@Z 004264b8     mfc90:mfc90.dll
 0002:000004bc       __imp_?GetThisClass@CMFCVisualManager@@SGPAUCRuntimeClass@@XZ 004264bc     mfc90:mfc90.dll
 0002:000004c0       __imp_?LoadFrame@CFrameWndEx@@UAEHIKPAVCWnd@@PAUCCreateContext@@@Z 004264c0     mfc90:mfc90.dll
 0002:000004c4       __imp_?TrackPopupMenu@CMenu@@QAEHIHHPAVCWnd@@PBUtagRECT@@@Z 004264c4     mfc90:mfc90.dll
 0002:000004c8       __imp_?ClientToScreen@CWnd@@QBEXPAUtagRECT@@@Z 004264c8     mfc90:mfc90.dll
 0002:000004cc       __imp_??1CStringArray@@UAE@XZ 004264cc     mfc90:mfc90.dll
 0002:000004d0       __imp_?Mid@?$CStringT@DV?$StrTraitMFC_DLL@DV?$ChTraitsCRT@D@ATL@@@@@ATL@@QBE?AV12@H@Z 004264d0     mfc90:mfc90.dll
 0002:000004d4       __imp_?Empty@?$CSimpleStringT@D$00@ATL@@QAEXXZ 004264d4     mfc90:mfc90.dll
 0002:000004d8       __imp_?Find@?$CStringT@DV?$StrTraitMFC_DLL@DV?$ChTraitsCRT@D@ATL@@@@@ATL@@QBEHPBDH@Z 004264d8     mfc90:mfc90.dll
 0002:000004dc       __imp_?Find@?$CStringT@DV?$StrTraitMFC_DLL@DV?$ChTraitsCRT@D@ATL@@@@@ATL@@QBEHDH@Z 004264dc     mfc90:mfc90.dll
 0002:000004e0       __imp_??0CStringArray@@QAE@XZ 004264e0     mfc90:mfc90.dll
 0002:000004e4       __imp_?ReleaseBuffer@?$CSimpleStringT@D$00@ATL@@QAEXH@Z 004264e4     mfc90:mfc90.dll
 0002:000004e8       __imp_??4?$CStringT@DV?$StrTraitMFC_DLL@DV?$ChTraitsCRT@D@ATL@@@@@ATL@@QAEAAV01@PBE@Z 004264e8     mfc90:mfc90.dll
 0002:000004ec       __imp_?OnClose@CFrameWnd@@IAEXXZ 004264ec     mfc90:mfc90.dll
 0002:000004f0       __imp_?OnDestroy@CFrameWnd@@IAEXXZ 004264f0     mfc90:mfc90.dll
 0002:000004f4       __imp_?AddTail@CStringList@@QAEPAU__POSITION@@PBD@Z 004264f4     mfc90:mfc90.dll
 0002:000004f8       __imp_?RemoveHead@CPtrList@@QAEPAXXZ 004264f8     mfc90:mfc90.dll
 0002:000004fc       __imp_?AddTail@CPtrList@@QAEPAU__POSITION@@PAX@Z 004264fc     mfc90:mfc90.dll
 0002:00000500       __imp_?AfxThrowOleException@@YGXJ@Z 00426500     mfc90:mfc90.dll
 0002:00000504       __imp_?GetRuntimeClass@CMenu@@UBEPAUCRuntimeClass@@XZ 00426504     mfc90:mfc90.dll
 0002:00000508       __imp_?DrawItem@CMenu@@UAEXPAUtagDRAWITEMSTRUCT@@@Z 00426508     mfc90:mfc90.dll
 0002:0000050c       __imp_?MeasureItem@CMenu@@UAEXPAUtagMEASUREITEMSTRUCT@@@Z 0042650c     mfc90:mfc90.dll
 0002:00000510       __imp_?DestroyMenu@CMenu@@QAEHXZ 00426510     mfc90:mfc90.dll
 0002:00000514       __imp_?FromHandle@CMenu@@SGPAV1@PAUHMENU__@@@Z 00426514     mfc90:mfc90.dll
 0002:00000518       __imp_?Attach@CMenu@@QAEHPAUHMENU__@@@Z 00426518     mfc90:mfc90.dll
 0002:0000051c       __imp_?AfxFindResourceHandle@@YGPAUHINSTANCE__@@PBD0@Z 0042651c     mfc90:mfc90.dll
 0002:00000520       __imp_?FromHandle@CWnd@@SGPAV1@PAUHWND__@@@Z 00426520     mfc90:mfc90.dll
 0002:00000524       __imp_?BeginWaitCursor@CCmdTarget@@QAEXXZ 00426524     mfc90:mfc90.dll
 0002:00000528       __imp_?EndWaitCursor@CCmdTarget@@QAEXXZ 00426528     mfc90:mfc90.dll
 0002:0000052c       __imp_?GetUserToolBarByIndex@CFrameImpl@@IBEPAVCMFCToolBar@@H@Z 0042652c     mfc90:mfc90.dll
 0002:00000530       __imp_?AddDefaultButtonsToCustomizePane@CFrameImpl@@IAEXPAVCMFCPopupMenu@@I@Z 00426530     mfc90:mfc90.dll
 0002:00000534       __imp_??0CStringList@@QAE@H@Z 00426534     mfc90:mfc90.dll
 0002:00000538       __imp_??1CStringList@@UAE@XZ 00426538     mfc90:mfc90.dll
 0002:0000053c       __imp_?GetRuntimeClass@CRichEditCtrl@@UBEPAUCRuntimeClass@@XZ 0042653c     mfc90:mfc90.dll
 0002:00000540       __imp_??1CRichEditCtrl@@UAE@XZ 00426540     mfc90:mfc90.dll
 0002:00000544       __imp_?GetThisMessageMap@CWnd@@KGPBUAFX_MSGMAP@@XZ 00426544     mfc90:mfc90.dll
 0002:00000548       __imp_?CanPaste@CRichEditCtrl@@QBEHI@Z 00426548     mfc90:mfc90.dll
 0002:0000054c       __imp_?GetStyle@CWnd@@QBEKXZ 0042654c     mfc90:mfc90.dll
 0002:00000550       __imp_?DDX_Text@@YGXPAVCDataExchange@@HAAH@Z 00426550     mfc90:mfc90.dll
 0002:00000554       __imp_??1CMapStringToString@@UAE@XZ 00426554     mfc90:mfc90.dll
 0002:00000558       __imp_?Replace@?$CStringT@DV?$StrTraitMFC_DLL@DV?$ChTraitsCRT@D@ATL@@@@@ATL@@QAEHPBD0@Z 00426558     mfc90:mfc90.dll
 0002:0000055c       __imp_?GetNextAssoc@CMapStringToString@@QBEXAAPAU__POSITION@@AAV?$CStringT@DV?$StrTraitMFC_DLL@DV?$ChTraitsCRT@D@ATL@@@@@ATL@@1@Z 0042655c     mfc90:mfc90.dll
 0002:00000560       __imp_?Lookup@CMapStringToString@@QBEHPBDAAV?$CStringT@DV?$StrTraitMFC_DLL@DV?$ChTraitsCRT@D@ATL@@@@@ATL@@@Z 00426560     mfc90:mfc90.dll
 0002:00000564       __imp_??0CMapStringToString@@QAE@H@Z 00426564     mfc90:mfc90.dll
 0002:00000568       __imp_?GetBufferSetLength@?$CSimpleStringT@D$00@ATL@@QAEPADH@Z 00426568     mfc90:mfc90.dll
 0002:0000056c       __imp_??ACMapStringToString@@QAEAAV?$CStringT@DV?$StrTraitMFC_DLL@DV?$ChTraitsCRT@D@ATL@@@@@ATL@@PBD@Z 0042656c     mfc90:mfc90.dll
 0002:00000570       __imp_??1CComboBox@@UAE@XZ 00426570     mfc90:mfc90.dll
 0002:00000574       __imp_?DDX_CBString@@YGXPAVCDataExchange@@HAAV?$CStringT@DV?$StrTraitMFC_DLL@DV?$ChTraitsCRT@D@ATL@@@@@ATL@@@Z 00426574     mfc90:mfc90.dll
 0002:00000578       __imp_?GetRuntimeClass@CComboBox@@UBEPAUCRuntimeClass@@XZ 00426578     mfc90:mfc90.dll
 0002:0000057c       __imp_?OnChildNotify@CComboBox@@MAEHIIJPAJ@Z 0042657c     mfc90:mfc90.dll
 0002:00000580       __imp_?Create@CComboBox@@UAEHKABUtagRECT@@PAVCWnd@@I@Z 00426580     mfc90:mfc90.dll
 0002:00000584       __imp_?DrawItem@CComboBox@@UAEXPAUtagDRAWITEMSTRUCT@@@Z 00426584     mfc90:mfc90.dll
 0002:00000588       __imp_?MeasureItem@CComboBox@@UAEXPAUtagMEASUREITEMSTRUCT@@@Z 00426588     mfc90:mfc90.dll
 0002:0000058c       __imp_?CompareItem@CComboBox@@UAEHPAUtagCOMPAREITEMSTRUCT@@@Z 0042658c     mfc90:mfc90.dll
 0002:00000590       __imp_?DeleteItem@CComboBox@@UAEXPAUtagDELETEITEMSTRUCT@@@Z 00426590     mfc90:mfc90.dll
 0002:00000594       __imp_?Close@CStdioFile@@UAEXXZ 00426594     mfc90:mfc90.dll
 0002:00000598       __imp_?Flush@CStdioFile@@UAEXXZ 00426598     mfc90:mfc90.dll
 0002:0000059c       __imp_?WriteString@CStdioFile@@UAEXPBD@Z 0042659c     mfc90:mfc90.dll
 0002:000005a0       __imp_??1CStdioFile@@UAE@XZ 004265a0     mfc90:mfc90.dll
 0002:000005a4       __imp_?Open@CStdioFile@@UAEHPBDIPAVCFileException@@@Z 004265a4     mfc90:mfc90.dll
 0002:000005a8       __imp_??0CStdioFile@@QAE@XZ 004265a8     mfc90:mfc90.dll
 0002:000005ac       __imp_?Mid@?$CStringT@DV?$StrTraitMFC_DLL@DV?$ChTraitsCRT@D@ATL@@@@@ATL@@QBE?AV12@HH@Z 004265ac     mfc90:mfc90.dll
 0002:000005b0       __imp_?AddHead@CPtrList@@QAEPAU__POSITION@@PAX@Z 004265b0     mfc90:mfc90.dll
 0002:000005b4       __imp_?RemoveAt@CPtrList@@QAEXPAU__POSITION@@@Z 004265b4     mfc90:mfc90.dll
 0002:000005b8       __imp_?ReadString@CStdioFile@@UAEHAAV?$CStringT@DV?$StrTraitMFC_DLL@DV?$ChTraitsCRT@D@ATL@@@@@ATL@@@Z 004265b8     mfc90:mfc90.dll
 0002:000005bc       __imp_??0COleVariant@@QAE@ABUtagVARIANT@@@Z 004265bc     mfc90:mfc90.dll
 0002:000005c0       __imp_?Insert@?$CStringT@DV?$StrTraitMFC_DLL@DV?$ChTraitsCRT@D@ATL@@@@@ATL@@QAEHHPBD@Z 004265c0     mfc90:mfc90.dll
 0002:000005c4       __imp_?Delete@?$CStringT@DV?$StrTraitMFC_DLL@DV?$ChTraitsCRT@D@ATL@@@@@ATL@@QAEHHH@Z 004265c4     mfc90:mfc90.dll
 0002:000005c8       __imp_?ExitInstance@CWinAppEx@@UAEHXZ 004265c8     mfc90:mfc90.dll
 0002:000005cc       __imp_?LoadStringA@?$CStringT@DV?$StrTraitMFC_DLL@DV?$ChTraitsCRT@D@ATL@@@@@ATL@@QAEHI@Z 004265cc     mfc90:mfc90.dll
 0002:000005d0       __imp_?GetContextMenuManager@CWinAppEx@@QAEPAVCContextMenuManager@@XZ 004265d0     mfc90:mfc90.dll
 0002:000005d4       __imp_?AddMenu@CContextMenuManager@@QAEHPBDI@Z 004265d4     mfc90:mfc90.dll
 0002:000005d8       __imp_?AfxInitRichEdit@@YGHXZ 004265d8     mfc90:mfc90.dll
 0002:000005dc       __imp_?InitInstance@CWinApp@@UAEHXZ 004265dc     mfc90:mfc90.dll
 0002:000005e0       __imp_?AfxOleInit@@YGHXZ   004265e0     mfc90:mfc90.dll
 0002:000005e4       __imp_?AfxMessageBox@@YGHIII@Z 004265e4     mfc90:mfc90.dll
 0002:000005e8       __imp_?AfxEnableControlContainer@@YAXPAVCOccManager@@@Z 004265e8     mfc90:mfc90.dll
 0002:000005ec       __imp_?SetRegistryKey@CWinApp@@IAEXPBD@Z 004265ec     mfc90:mfc90.dll
 0002:000005f0       __imp_?LoadStdProfileSettings@CWinApp@@IAEXI@Z 004265f0     mfc90:mfc90.dll
 0002:000005f4       __imp_?InitContextMenuManager@CWinAppEx@@QAEHXZ 004265f4     mfc90:mfc90.dll
 0002:000005f8       __imp_?InitKeyboardManager@CWinAppEx@@QAEHXZ 004265f8     mfc90:mfc90.dll
 0002:000005fc       __imp_?InitTooltipManager@CWinAppEx@@QAEHXZ 004265fc     mfc90:mfc90.dll
 0002:00000600       __imp_?GetThisClass@CMFCToolTipCtrl@@SGPAUCRuntimeClass@@XZ 00426600     mfc90:mfc90.dll
 0002:00000604       __imp_?GetTooltipManager@CWinAppEx@@QAEPAVCTooltipManager@@XZ 00426604     mfc90:mfc90.dll
 0002:00000608       __imp_?SetTooltipParams@CTooltipManager@@QAEXIPAUCRuntimeClass@@PAVCMFCToolTipInfo@@@Z 00426608     mfc90:mfc90.dll
 0002:0000060c       __imp_??0CCommandLineInfo@@QAE@XZ 0042660c     mfc90:mfc90.dll
 0002:00000610       __imp_?ParseCommandLine@CWinApp@@QAEXAAVCCommandLineInfo@@@Z 00426610     mfc90:mfc90.dll
 0002:00000614       __imp_?ProcessShellCommand@CWinApp@@QAEHAAVCCommandLineInfo@@@Z 00426614     mfc90:mfc90.dll
 0002:00000618       __imp_??1CCommandLineInfo@@UAE@XZ 00426618     mfc90:mfc90.dll
 0002:0000061c       __imp_??1CWinAppEx@@UAE@XZ 0042661c     mfc90:mfc90.dll
 0002:00000620       __imp_?ReloadWindowPlacement@CWinAppEx@@MAEHPAVCFrameWnd@@@Z 00426620     mfc90:mfc90.dll
 0002:00000624       __imp_?StoreWindowPlacement@CWinAppEx@@MAEHABVCRect@@HH@Z 00426624     mfc90:mfc90.dll
 0002:00000628       __imp_?LoadWindowPlacement@CWinAppEx@@MAEHAAVCRect@@AAH1@Z 00426628     mfc90:mfc90.dll
 0002:0000062c       __imp_?OnClosingMainFrame@CWinAppEx@@MAEXPAVCFrameImpl@@@Z 0042662c     mfc90:mfc90.dll
 0002:00000630       __imp_?OnAppContextHelp@CWinAppEx@@UAEXPAVCWnd@@QBK@Z 00426630     mfc90:mfc90.dll
 0002:00000634       __imp_?ShowPopupMenu@CWinAppEx@@UAEHIABVCPoint@@PAVCWnd@@@Z 00426634     mfc90:mfc90.dll
 0002:00000638       __imp_?OnViewDoubleClick@CWinAppEx@@UAEHPAVCWnd@@H@Z 00426638     mfc90:mfc90.dll
 0002:0000063c       __imp_?SaveState@CWinAppEx@@UAEHPBDPAVCFrameImpl@@@Z 0042663c     mfc90:mfc90.dll
 0002:00000640       __imp_?CleanState@CWinAppEx@@UAEHPBD@Z 00426640     mfc90:mfc90.dll
 0002:00000644       __imp_?LoadState@CWinAppEx@@UAEHPBDPAVCFrameImpl@@@Z 00426644     mfc90:mfc90.dll
 0002:00000648       __imp_?LoadSysPolicies@CWinApp@@UAEHXZ 00426648     mfc90:mfc90.dll
 0002:0000064c       __imp_?LoadAppLangResourceDLL@CWinApp@@UAEPAUHINSTANCE__@@XZ 0042664c     mfc90:mfc90.dll
 0002:00000650       __imp_?WinHelpInternal@CWinApp@@UAEXKI@Z 00426650     mfc90:mfc90.dll
 0002:00000654       __imp_?HtmlHelpA@CWinApp@@UAEXKI@Z 00426654     mfc90:mfc90.dll
 0002:00000658       __imp_?WinHelpA@CWinApp@@UAEXKI@Z 00426658     mfc90:mfc90.dll
 0002:0000065c       __imp_?OnDDECommand@CWinApp@@UAEHPAD@Z 0042665c     mfc90:mfc90.dll
 0002:00000660       __imp_?DoWaitCursor@CWinApp@@UAEXH@Z 00426660     mfc90:mfc90.dll
 0002:00000664       __imp_?DoMessageBox@CWinApp@@UAEHPBDII@Z 00426664     mfc90:mfc90.dll
 0002:00000668       __imp_?SaveAllModified@CWinApp@@UAEHXZ 00426668     mfc90:mfc90.dll
 0002:0000066c       __imp_?InitApplication@CWinApp@@UAEHXZ 0042666c     mfc90:mfc90.dll
 0002:00000670       __imp_?AddToRecentFileList@CWinApp@@UAEXPBD@Z 00426670     mfc90:mfc90.dll
 0002:00000674       __imp_?OpenDocumentFile@CWinApp@@UAEPAVCDocument@@PBD@Z 00426674     mfc90:mfc90.dll
 0002:00000678       __imp_?Unregister@CWinApp@@UAEHXZ 00426678     mfc90:mfc90.dll
 0002:0000067c       __imp_?Register@CWinApp@@UAEHXZ 0042667c     mfc90:mfc90.dll
 0002:00000680       __imp_?InitLibId@CWinApp@@UAEXXZ 00426680     mfc90:mfc90.dll
 0002:00000684       __imp_?ProcessWndProcException@CWinApp@@UAEJPAVCException@@PBUtagMSG@@@Z 00426684     mfc90:mfc90.dll
 0002:00000688       __imp_?OnIdle@CWinApp@@UAEHJ@Z 00426688     mfc90:mfc90.dll
 0002:0000068c       __imp_?Run@CWinApp@@UAEHXZ 0042668c     mfc90:mfc90.dll
 0002:00000690       __imp_?GetRuntimeClass@CWinAppEx@@UBEPAUCRuntimeClass@@XZ 00426690     mfc90:mfc90.dll
 0002:00000694       __imp_??0CWinAppEx@@QAE@H@Z 00426694     mfc90:mfc90.dll
 0002:00000698       __imp_?OnFilePrintSetup@CWinApp@@IAEXXZ 00426698     mfc90:mfc90.dll
 0002:0000069c       __imp_?OnFileOpen@CWinApp@@IAEXXZ 0042669c     mfc90:mfc90.dll
 0002:000006a0       __imp_?OnFileNew@CWinApp@@IAEXXZ 004266a0     mfc90:mfc90.dll
 0002:000006a4       __imp_?GetThisMessageMap@CWinApp@@KGPBUAFX_MSGMAP@@XZ 004266a4     mfc90:mfc90.dll
 0002:000006a8       __imp_?GetOFN@CFileDialog@@QBEABUtagOFNA@@XZ 004266a8     mfc90:mfc90.dll
 0002:000006ac       __imp_?AfxGetThread@@YGPAVCWinThread@@XZ 004266ac     mfc90:mfc90.dll
 0002:000006b0       __imp_?AfxGetModuleState@@YGPAVAFX_MODULE_STATE@@XZ 004266b0     mfc90:mfc90.dll
 0002:000006b4       __imp_??2@YAPAXI@Z         004266b4     mfc90:mfc90.dll
 0002:000006b8       __imp_?EnableWindow@CWnd@@QAEHH@Z 004266b8     mfc90:mfc90.dll
 0002:000006bc       __imp_??0CFileDialog@@QAE@HPBD0K0PAVCWnd@@KH@Z 004266bc     mfc90:mfc90.dll
 0002:000006c0       __imp_?GetOFN@CFileDialog@@QAEAAUtagOFNA@@XZ 004266c0     mfc90:mfc90.dll
 0002:000006c4       __imp_?DoModal@CFileDialog@@UAEHXZ 004266c4     mfc90:mfc90.dll
 0002:000006c8       __imp_??1CFileDialog@@UAE@XZ 004266c8     mfc90:mfc90.dll
 0002:000006cc       __imp_?GetNextPathName@CFileDialog@@QBE?AV?$CStringT@DV?$StrTraitMFC_DLL@DV?$ChTraitsCRT@D@ATL@@@@@ATL@@AAPAU__POSITION@@@Z 004266cc     mfc90:mfc90.dll
 0002:000006d0       __imp_??0CInternetSession@@QAE@PBDKK00K@Z 004266d0     mfc90:mfc90.dll
 0002:000006d4       __imp_?GetFtpConnection@CInternetSession@@QAEPAVCFtpConnection@@PBD00GH@Z 004266d4     mfc90:mfc90.dll
 0002:000006d8       __imp_?CreateDirectoryA@CFtpConnection@@QAEHPBD@Z 004266d8     mfc90:mfc90.dll
 0002:000006dc       __imp_?SetCurrentDirectoryA@CFtpConnection@@QAEHPBD@Z 004266dc     mfc90:mfc90.dll
 0002:000006e0       __imp_??0CFtpFileFind@@QAE@PAVCFtpConnection@@K@Z 004266e0     mfc90:mfc90.dll
 0002:000006e4       __imp_?FindFile@CFtpFileFind@@UAEHPBDK@Z 004266e4     mfc90:mfc90.dll
 0002:000006e8       __imp_?FindNextFileA@CFtpFileFind@@UAEHXZ 004266e8     mfc90:mfc90.dll
 0002:000006ec       __imp_?GetFileName@CFileFind@@UBE?AV?$CStringT@DV?$StrTraitMFC_DLL@DV?$ChTraitsCRT@D@ATL@@@@@ATL@@XZ 004266ec     mfc90:mfc90.dll
 0002:000006f0       __imp_??1CFtpFileFind@@UAE@XZ 004266f0     mfc90:mfc90.dll
 0002:000006f4       __imp_?PutFile@CFtpConnection@@QAEHPBD0KK@Z 004266f4     mfc90:mfc90.dll
 0002:000006f8       __imp_?Delete@CWinThread@@UAEXXZ 004266f8     mfc90:mfc90.dll
 0002:000006fc       __imp_?GetMainWnd@CWinThread@@UAEPAVCWnd@@XZ 004266fc     mfc90:mfc90.dll
 0002:00000700       __imp_?ProcessMessageFilter@CWinThread@@UAEHHPAUtagMSG@@@Z 00426700     mfc90:mfc90.dll
 0002:00000704       __imp_?IsIdleMessage@CWinThread@@UAEHPAUtagMSG@@@Z 00426704     mfc90:mfc90.dll
 0002:00000708       __imp_?PumpMessage@CWinThread@@UAEHXZ 00426708     mfc90:mfc90.dll
 0002:0000070c       __imp_?PreTranslateMessage@CWinThread@@UAEHPAUtagMSG@@@Z 0042670c     mfc90:mfc90.dll
 0002:00000710       __imp_?GetInterfaceMap@CCmdTarget@@MBEPBUAFX_INTERFACEMAP@@XZ 00426710     mfc90:mfc90.dll
 0002:00000714       __imp_?OnFinalRelease@CCmdTarget@@UAEXXZ 00426714     mfc90:mfc90.dll
 0002:00000718       __imp_??0CFileFind@@QAE@XZ 00426718     mfc90:mfc90.dll
 0002:0000071c       __imp_?FindFile@CFileFind@@UAEHPBDK@Z 0042671c     mfc90:mfc90.dll
 0002:00000720       __imp_??1CFileFind@@UAE@XZ 00426720     mfc90:mfc90.dll
 0002:00000724       __imp_?ReverseFind@?$CStringT@DV?$StrTraitMFC_DLL@DV?$ChTraitsCRT@D@ATL@@@@@ATL@@QBEHD@Z 00426724     mfc90:mfc90.dll
 0002:00000728       __imp_?Right@?$CStringT@DV?$StrTraitMFC_DLL@DV?$ChTraitsCRT@D@ATL@@@@@ATL@@QBE?AV12@H@Z 00426728     mfc90:mfc90.dll
 0002:0000072c       __imp_?MessageBoxA@CWnd@@QAEHPBD0I@Z 0042672c     mfc90:mfc90.dll
 0002:00000730       __imp_?AfxBeginThread@@YGPAVCWinThread@@P6AIPAX@Z0HIKPAU_SECURITY_ATTRIBUTES@@@Z 00426730     mfc90:mfc90.dll
 0002:00000734       __imp_?DDX_Check@@YGXPAVCDataExchange@@HAAH@Z 00426734     mfc90:mfc90.dll
 0002:00000738       __imp_??A?$CSimpleStringT@D$00@ATL@@QBEDH@Z 00426738     mfc90:mfc90.dll
 0002:0000073c       __imp_?Remove@?$CStringT@DV?$StrTraitMFC_DLL@DV?$ChTraitsCRT@D@ATL@@@@@ATL@@QAEHD@Z 0042673c     mfc90:mfc90.dll
 0002:00000740       __imp_?GetAt@?$CSimpleStringT@D$00@ATL@@QBEDH@Z 00426740     mfc90:mfc90.dll
 0002:00000744       __imp_?GetThisClass@CDialog@@SGPAUCRuntimeClass@@XZ 00426744     mfc90:mfc90.dll
 0002:00000748       __imp_??_U@YAPAXI@Z        00426748     mfc90:mfc90.dll
 0002:0000074c       __imp_?Replace@?$CStringT@DV?$StrTraitMFC_DLL@DV?$ChTraitsCRT@D@ATL@@@@@ATL@@QAEHDD@Z 0042674c     mfc90:mfc90.dll
 0002:00000750       __imp_??Y?$CStringT@DV?$StrTraitMFC_DLL@DV?$ChTraitsCRT@D@ATL@@@@@ATL@@QAEAAV01@ABV?$CSimpleStringT@D$00@1@@Z 00426750     mfc90:mfc90.dll
 0002:00000754       __imp_?Left@?$CStringT@DV?$StrTraitMFC_DLL@DV?$ChTraitsCRT@D@ATL@@@@@ATL@@QBE?AV12@H@Z 00426754     mfc90:mfc90.dll
 0002:00000758       __imp_?GetBuffer@?$CSimpleStringT@D$00@ATL@@QAEPADH@Z 00426758     mfc90:mfc90.dll
 0002:0000075c       __imp_?GetRuntimeClass@CEdit@@UBEPAUCRuntimeClass@@XZ 0042675c     mfc90:mfc90.dll
 0002:00000760       __imp_?OnCtlColor@CWnd@@IAEPAUHBRUSH__@@PAVCDC@@PAV1@I@Z 00426760     mfc90:mfc90.dll
 0002:00000764       __imp_?GetDlgCtrlID@CWnd@@QBEHXZ 00426764     mfc90:mfc90.dll
 0002:00000768       __imp_?SetBkMode@CDC@@QAEHH@Z 00426768     mfc90:mfc90.dll
 0002:0000076c       __imp_?Compare@?$CStringT@DV?$StrTraitMFC_DLL@DV?$ChTraitsCRT@D@ATL@@@@@ATL@@QBEHPBD@Z 0042676c     mfc90:mfc90.dll
 0002:00000770       __imp_?OnOK@CDialog@@MAEXXZ 00426770     mfc90:mfc90.dll
 0002:00000774       __imp_?UpdateData@CWnd@@QAEHH@Z 00426774     mfc90:mfc90.dll
 0002:00000778       __imp_?ShowWindow@CWnd@@QAEHH@Z 00426778     mfc90:mfc90.dll
 0002:0000077c       __imp_?DDX_Text@@YGXPAVCDataExchange@@HAAV?$CStringT@DV?$StrTraitMFC_DLL@DV?$ChTraitsCRT@D@ATL@@@@@ATL@@@Z 0042677c     mfc90:mfc90.dll
 0002:00000780       __imp_?DDV_MaxChars@@YGXPAVCDataExchange@@ABV?$CStringT@DV?$StrTraitMFC_DLL@DV?$ChTraitsCRT@D@ATL@@@@@ATL@@H@Z 00426780     mfc90:mfc90.dll
 0002:00000784       __imp_??4?$CStringT@DV?$StrTraitMFC_DLL@DV?$ChTraitsCRT@D@ATL@@@@@ATL@@QAEAAV01@PBD@Z 00426784     mfc90:mfc90.dll
 0002:00000788       __imp_??1CEdit@@UAE@XZ     00426788     mfc90:mfc90.dll
 0002:0000078c       __imp_?StringLength@?$CSimpleStringT@D$00@ATL@@SAHPBD@Z 0042678c     mfc90:mfc90.dll
 0002:00000790       __imp_?DrawItem@CStatic@@UAEXPAUtagDRAWITEMSTRUCT@@@Z 00426790     mfc90:mfc90.dll
 0002:00000794       __imp_?Create@CStatic@@UAEHPBDKABUtagRECT@@PAVCWnd@@I@Z 00426794     mfc90:mfc90.dll
 0002:00000798       __imp_?GetOccDialogInfo@CWnd@@MAEPAU_AFX_OCC_DIALOG_INFO@@XZ 00426798     mfc90:mfc90.dll
 0002:0000079c       __imp_?SetOccDialogInfo@CWnd@@MAEHPAU_AFX_OCC_DIALOG_INFO@@@Z 0042679c     mfc90:mfc90.dll
 0002:000007a0       __imp_?CheckAutoCenter@CWnd@@UAEHXZ 004267a0     mfc90:mfc90.dll
 0002:000007a4       __imp_?OnChildNotify@CStatic@@MAEHIIJPAJ@Z 004267a4     mfc90:mfc90.dll
 0002:000007a8       __imp_?PreTranslateMessage@CWnd@@UAEHPAUtagMSG@@@Z 004267a8     mfc90:mfc90.dll
 0002:000007ac       __imp_?GetMessageMap@CWnd@@MBEPBUAFX_MSGMAP@@XZ 004267ac     mfc90:mfc90.dll
 0002:000007b0       __imp_?OnCmdMsg@CCmdTarget@@UAEHIHPAXPAUAFX_CMDHANDLERINFO@@@Z 004267b0     mfc90:mfc90.dll
 0002:000007b4       __imp_?GetRuntimeClass@CStatic@@UBEPAUCRuntimeClass@@XZ 004267b4     mfc90:mfc90.dll
 0002:000007b8       __imp_??0CWnd@@QAE@XZ      004267b8     mfc90:mfc90.dll
 0002:000007bc       __imp_?Default@CWnd@@IAEJXZ 004267bc     mfc90:mfc90.dll
 0002:000007c0       __imp_?AfxThrowInvalidArgException@@YGXXZ 004267c0     mfc90:mfc90.dll
 0002:000007c4       __imp_?GetManager@?$CStringT@DV?$StrTraitMFC_DLL@DV?$ChTraitsCRT@D@ATL@@@@@ATL@@QBEPAUIAtlStringMgr@2@XZ 004267c4     mfc90:mfc90.dll
 0002:000007c8       __imp_??0?$CStringT@DV?$StrTraitMFC_DLL@DV?$ChTraitsCRT@D@ATL@@@@@ATL@@QAE@PAUIAtlStringMgr@1@@Z 004267c8     mfc90:mfc90.dll
 0002:000007cc       __imp_?GetLength@?$CSimpleStringT@D$00@ATL@@QBEHXZ 004267cc     mfc90:mfc90.dll
 0002:000007d0       __imp_?Concatenate@?$CSimpleStringT@D$00@ATL@@KAXAAV12@PBDH1H@Z 004267d0     mfc90:mfc90.dll
 0002:000007d4       __imp_?OnCancel@CDialog@@MAEXXZ 004267d4     mfc90:mfc90.dll
 0002:000007d8       __imp_?RemoveAll@CStringList@@QAEXXZ 004267d8     mfc90:mfc90.dll
 0002:000007dc       __imp_?PreTranslateMessage@CDialog@@UAEHPAUtagMSG@@@Z 004267dc     mfc90:mfc90.dll
 0002:000007e0       __imp_??0?$CStringT@DV?$StrTraitMFC_DLL@DV?$ChTraitsCRT@D@ATL@@@@@ATL@@QAE@PBD@Z 004267e0     mfc90:mfc90.dll
 0002:000007e4       __imp_?EndDialog@CDialog@@QAEXH@Z 004267e4     mfc90:mfc90.dll
 0002:000007e8       __imp_?OnCommand@CWnd@@MAEHIJ@Z 004267e8     mfc90:mfc90.dll
 0002:000007ec       __imp_?OnInitDialog@CDialog@@UAEHXZ 004267ec     mfc90:mfc90.dll
 0002:000007f0       __imp_?IsEmpty@?$CSimpleStringT@D$00@ATL@@QBE_NXZ 004267f0     mfc90:mfc90.dll
 0002:000007f4       __imp_?wndTopMost@CWnd@@2V1@B 004267f4     mfc90:mfc90.dll
 0002:000007f8       __imp_?SetWindowPos@CWnd@@QAEHPBV1@HHHHI@Z 004267f8     mfc90:mfc90.dll
 0002:000007fc       __imp_??B?$CSimpleStringT@D$00@ATL@@QBEPBDXZ 004267fc     mfc90:mfc90.dll
 0002:00000800       __imp_?AfxMessageBox@@YGHPBDII@Z 00426800     mfc90:mfc90.dll
 0002:00000804       __imp_?GetDlgItem@CWnd@@QBEPAV1@H@Z 00426804     mfc90:mfc90.dll
 0002:00000808       __imp_?SetFocus@CWnd@@QAEPAV1@XZ 00426808     mfc90:mfc90.dll
 0002:0000080c       __imp_?Format@?$CStringT@DV?$StrTraitMFC_DLL@DV?$ChTraitsCRT@D@ATL@@@@@ATL@@QAAXPBDZZ 0042680c     mfc90:mfc90.dll
 0002:00000810       __imp_?GetWindowTextA@CWnd@@QBEXAAV?$CStringT@DV?$StrTraitMFC_DLL@DV?$ChTraitsCRT@D@ATL@@@@@ATL@@@Z 00426810     mfc90:mfc90.dll
 0002:00000814       __imp_?CompareNoCase@?$CStringT@DV?$StrTraitMFC_DLL@DV?$ChTraitsCRT@D@ATL@@@@@ATL@@QBEHPBD@Z 00426814     mfc90:mfc90.dll
 0002:00000818       __imp_?GetWindowTextLengthA@CWnd@@QBEHXZ 00426818     mfc90:mfc90.dll
 0002:0000081c       __imp_?AddTail@CStringList@@QAEPAU__POSITION@@ABV?$CStringT@DV?$StrTraitMFC_DLL@DV?$ChTraitsCRT@D@ATL@@@@@ATL@@@Z 0042681c     mfc90:mfc90.dll
 0002:00000820       __imp_??Y?$CStringT@DV?$StrTraitMFC_DLL@DV?$ChTraitsCRT@D@ATL@@@@@ATL@@QAEAAV01@PBD@Z 00426820     mfc90:mfc90.dll
 0002:00000824       __imp_?SetSel@CRichEditCtrl@@QAEXJJ@Z 00426824     mfc90:mfc90.dll
 0002:00000828       __imp_?SetWordCharFormat@CRichEditCtrl@@QAEHAAU_charformat@@@Z 00426828     mfc90:mfc90.dll
 0002:0000082c       __imp_?SetWindowTextA@CWnd@@QAEXPBD@Z 0042682c     mfc90:mfc90.dll
 0002:00000830       __imp_?GetThisMessageMap@CDialog@@KGPBUAFX_MSGMAP@@XZ 00426830     mfc90:mfc90.dll
 0002:00000834       __imp_?DDX_Control@@YGXPAVCDataExchange@@HAAVCWnd@@@Z 00426834     mfc90:mfc90.dll
 0002:00000838       __imp_??1CStatic@@UAE@XZ   00426838     mfc90:mfc90.dll
 0002:0000083c       __imp_?PreInitDialog@CDialog@@MAEXXZ 0042683c     mfc90:mfc90.dll
 0002:00000840       __imp_?OnSetFont@CDialog@@UAEXPAVCFont@@@Z 00426840     mfc90:mfc90.dll
 0002:00000844       __imp_?DoModal@CDialog@@UAEHXZ 00426844     mfc90:mfc90.dll
 0002:00000848       __imp_?CreateIndirect@CDialog@@UAEHPBUDLGTEMPLATE@@PAVCWnd@@PAX@Z 00426848     mfc90:mfc90.dll
 0002:0000084c       __imp_?CreateIndirect@CDialog@@UAEHPAXPAVCWnd@@@Z 0042684c     mfc90:mfc90.dll
 0002:00000850       __imp_?Create@CDialog@@UAEHPBDPAVCWnd@@@Z 00426850     mfc90:mfc90.dll
 0002:00000854       __imp_?GetOccDialogInfo@CDialog@@MAEPAU_AFX_OCC_DIALOG_INFO@@XZ 00426854     mfc90:mfc90.dll
 0002:00000858       __imp_?SetOccDialogInfo@CDialog@@MAEHPAU_AFX_OCC_DIALOG_INFO@@@Z 00426858     mfc90:mfc90.dll
 0002:0000085c       __imp_?CreateControlSite@CWnd@@MAEHPAVCOleControlContainer@@PAPAVCOleControlSite@@IABU_GUID@@@Z 0042685c     mfc90:mfc90.dll
 0002:00000860       __imp_?CreateControlContainer@CWnd@@MAEHPAPAVCOleControlContainer@@@Z 00426860     mfc90:mfc90.dll
 0002:00000864       __imp_?IsFrameWnd@CWnd@@UBEHXZ 00426864     mfc90:mfc90.dll
 0002:00000868       __imp_?CheckAutoCenter@CDialog@@UAEHXZ 00426868     mfc90:mfc90.dll
 0002:0000086c       __imp_?OnChildNotify@CWnd@@MAEHIIJPAJ@Z 0042686c     mfc90:mfc90.dll
 0002:00000870       __imp_?PostNcDestroy@CWnd@@MAEXXZ 00426870     mfc90:mfc90.dll
 0002:00000874       __imp_?DefWindowProcA@CWnd@@MAEJIIJ@Z 00426874     mfc90:mfc90.dll
 0002:00000878       __imp_?OnWndMsg@CWnd@@MAEHIIJPAJ@Z 00426878     mfc90:mfc90.dll
 0002:0000087c       __imp_?WindowProc@CWnd@@MAEJIIJ@Z 0042687c     mfc90:mfc90.dll
 0002:00000880       __imp_?OnAmbientProperty@CWnd@@UAEHPAVCOleControlSite@@JPAUtagVARIANT@@@Z 00426880     mfc90:mfc90.dll
 0002:00000884       __imp_?GetSuperWndProcAddr@CWnd@@MAEPAP6GJPAUHWND__@@IIJ@ZXZ 00426884     mfc90:mfc90.dll
 0002:00000888       __imp_?OnNotify@CWnd@@MAEHIJPAJ@Z 00426888     mfc90:mfc90.dll
 0002:0000088c       __imp_?CreateAccessibleProxy@CWnd@@UAEJIJPAJ@Z 0042688c     mfc90:mfc90.dll
 0002:00000890       __imp_?SetProxy@CWnd@@UAEJPAUIAccessibleProxy@@@Z 00426890     mfc90:mfc90.dll
 0002:00000894       __imp_?put_accValue@CWnd@@UAEJUtagVARIANT@@PA_W@Z 00426894     mfc90:mfc90.dll
 0002:00000898       __imp_?put_accName@CWnd@@UAEJUtagVARIANT@@PA_W@Z 00426898     mfc90:mfc90.dll
 0002:0000089c       __imp_?accDoDefaultAction@CWnd@@UAEJUtagVARIANT@@@Z 0042689c     mfc90:mfc90.dll
 0002:000008a0       __imp_?accHitTest@CWnd@@UAEJJJPAUtagVARIANT@@@Z 004268a0     mfc90:mfc90.dll
 0002:000008a4       __imp_?accNavigate@CWnd@@UAEJJUtagVARIANT@@PAU2@@Z 004268a4     mfc90:mfc90.dll
 0002:000008a8       __imp_?accLocation@CWnd@@UAEJPAJ000UtagVARIANT@@@Z 004268a8     mfc90:mfc90.dll
 0002:000008ac       __imp_?accSelect@CWnd@@UAEJJUtagVARIANT@@@Z 004268ac     mfc90:mfc90.dll
 0002:000008b0       __imp_?get_accDefaultAction@CWnd@@UAEJUtagVARIANT@@PAPA_W@Z 004268b0     mfc90:mfc90.dll
 0002:000008b4       __imp_?get_accSelection@CWnd@@UAEJPAUtagVARIANT@@@Z 004268b4     mfc90:mfc90.dll
 0002:000008b8       __imp_?get_accFocus@CWnd@@UAEJPAUtagVARIANT@@@Z 004268b8     mfc90:mfc90.dll
 0002:000008bc       __imp_?get_accKeyboardShortcut@CWnd@@UAEJUtagVARIANT@@PAPA_W@Z 004268bc     mfc90:mfc90.dll
 0002:000008c0       __imp_?get_accHelpTopic@CWnd@@UAEJPAPA_WUtagVARIANT@@PAJ@Z 004268c0     mfc90:mfc90.dll
 0002:000008c4       __imp_?get_accHelp@CWnd@@UAEJUtagVARIANT@@PAPA_W@Z 004268c4     mfc90:mfc90.dll
 0002:000008c8       __imp_?get_accState@CWnd@@UAEJUtagVARIANT@@PAU2@@Z 004268c8     mfc90:mfc90.dll
 0002:000008cc       __imp_?get_accRole@CWnd@@UAEJUtagVARIANT@@PAU2@@Z 004268cc     mfc90:mfc90.dll
 0002:000008d0       __imp_?get_accDescription@CWnd@@UAEJUtagVARIANT@@PAPA_W@Z 004268d0     mfc90:mfc90.dll
 0002:000008d4       __imp_?get_accValue@CWnd@@UAEJUtagVARIANT@@PAPA_W@Z 004268d4     mfc90:mfc90.dll
 0002:000008d8       __imp_?get_accName@CWnd@@UAEJUtagVARIANT@@PAPA_W@Z 004268d8     mfc90:mfc90.dll
 0002:000008dc       __imp_?get_accChild@CWnd@@UAEJUtagVARIANT@@PAPAUIDispatch@@@Z 004268dc     mfc90:mfc90.dll
 0002:000008e0       __imp_?get_accChildCount@CWnd@@UAEJPAJ@Z 004268e0     mfc90:mfc90.dll
 0002:000008e4       __imp_?get_accParent@CWnd@@UAEJPAPAUIDispatch@@@Z 004268e4     mfc90:mfc90.dll
 0002:000008e8       __imp_?EnsureStdObj@CWnd@@UAEJXZ 004268e8     mfc90:mfc90.dll
 0002:000008ec       __imp_?EndModalLoop@CWnd@@UAEXH@Z 004268ec     mfc90:mfc90.dll
 0002:000008f0       __imp_?ContinueModal@CWnd@@UAEHXZ 004268f0     mfc90:mfc90.dll
 0002:000008f4       __imp_?WinHelpInternal@CWnd@@UAEXKI@Z 004268f4     mfc90:mfc90.dll
 0002:000008f8       __imp_?HtmlHelpA@CWnd@@UAEXKI@Z 004268f8     mfc90:mfc90.dll
 0002:000008fc       __imp_?WinHelpA@CWnd@@UAEXKI@Z 004268fc     mfc90:mfc90.dll
 0002:00000900       __imp_?GetScrollBarCtrl@CWnd@@UBEPAVCScrollBar@@H@Z 00426900     mfc90:mfc90.dll
 0002:00000904       __imp_?OnToolHitTest@CWnd@@UBEHVCPoint@@PAUtagTOOLINFOA@@@Z 00426904     mfc90:mfc90.dll
 0002:00000908       __imp_?SetMenu@CWnd@@UAEHPAVCMenu@@@Z 00426908     mfc90:mfc90.dll
 0002:0000090c       __imp_?GetMenu@CWnd@@UBEPAVCMenu@@XZ 0042690c     mfc90:mfc90.dll
 0002:00000910       __imp_?CalcWindowRect@CWnd@@UAEXPAUtagRECT@@I@Z 00426910     mfc90:mfc90.dll
 0002:00000914       __imp_?PreCreateWindow@CWnd@@UAEHAAUtagCREATESTRUCTA@@@Z 00426914     mfc90:mfc90.dll
 0002:00000918       __imp_?DestroyWindow@CWnd@@UAEHXZ 00426918     mfc90:mfc90.dll
 0002:0000091c       __imp_?CreateEx@CWnd@@UAEHKPBD0KHHHHPAUHWND__@@PAUHMENU__@@PAX@Z 0042691c     mfc90:mfc90.dll
 0002:00000920       __imp_?CreateEx@CWnd@@UAEHKPBD0KABUtagRECT@@PAV1@IPAX@Z 00426920     mfc90:mfc90.dll
 0002:00000924       __imp_?Create@CWnd@@UAEHPBD0KABUtagRECT@@PAV1@IPAUCCreateContext@@@Z 00426924     mfc90:mfc90.dll
 0002:00000928       __imp_?PreSubclassWindow@CWnd@@UAEXXZ 00426928     mfc90:mfc90.dll
 0002:0000092c       __imp_?GetConnectionHook@CCmdTarget@@MAEPAUIConnectionPoint@@ABU_GUID@@@Z 0042692c     mfc90:mfc90.dll
 0002:00000930       __imp_?GetExtraConnectionPoints@CCmdTarget@@MAEHPAVCPtrArray@@@Z 00426930     mfc90:mfc90.dll
 0002:00000934       __imp_?GetInterfaceHook@CCmdTarget@@UAEPAUIUnknown@@PBX@Z 00426934     mfc90:mfc90.dll
 0002:00000938       __imp_?OnCreateAggregates@CCmdTarget@@UAEHXZ 00426938     mfc90:mfc90.dll
 0002:0000093c       __imp_?GetEventSinkMap@CCmdTarget@@MBEPBUAFX_EVENTSINKMAP@@XZ 0042693c     mfc90:mfc90.dll
 0002:00000940       __imp_?GetInterfaceMap@CWnd@@MBEPBUAFX_INTERFACEMAP@@XZ 00426940     mfc90:mfc90.dll
 0002:00000944       __imp_?GetConnectionMap@CCmdTarget@@MBEPBUAFX_CONNECTIONMAP@@XZ 00426944     mfc90:mfc90.dll
 0002:00000948       __imp_?GetDispatchMap@CCmdTarget@@MBEPBUAFX_DISPMAP@@XZ 00426948     mfc90:mfc90.dll
 0002:0000094c       __imp_?GetCommandMap@CCmdTarget@@MBEPBUAFX_OLECMDMAP@@XZ 0042694c     mfc90:mfc90.dll
 0002:00000950       __imp_?GetTypeLib@CCmdTarget@@UAEJKPAPAUITypeLib@@@Z 00426950     mfc90:mfc90.dll
 0002:00000954       __imp_?GetTypeLibCache@CCmdTarget@@UAEPAVCTypeLibCache@@XZ 00426954     mfc90:mfc90.dll
 0002:00000958       __imp_?GetTypeInfoCount@CCmdTarget@@UAEIXZ 00426958     mfc90:mfc90.dll
 0002:0000095c       __imp_?GetDispatchIID@CCmdTarget@@UAEHPAU_GUID@@@Z 0042695c     mfc90:mfc90.dll
 0002:00000960       __imp_?IsInvokeAllowed@CCmdTarget@@UAEHJ@Z 00426960     mfc90:mfc90.dll
 0002:00000964       __imp_?OnFinalRelease@CWnd@@UAEXXZ 00426964     mfc90:mfc90.dll
 0002:00000968       __imp_?OnCmdMsg@CDialog@@UAEHIHPAXPAUAFX_CMDHANDLERINFO@@@Z 00426968     mfc90:mfc90.dll
 0002:0000096c       __imp_?GetRuntimeClass@CDialog@@UBEPAUCRuntimeClass@@XZ 0042696c     mfc90:mfc90.dll
 0002:00000970       __imp_??0CDialog@@QAE@IPAVCWnd@@@Z 00426970     mfc90:mfc90.dll
 0002:00000974       __imp_??0?$CStringT@DV?$StrTraitMFC_DLL@DV?$ChTraitsCRT@D@ATL@@@@@ATL@@QAE@XZ 00426974     mfc90:mfc90.dll
 0002:00000978       __imp_??1CDialog@@UAE@XZ   00426978     mfc90:mfc90.dll
 0002:0000097c       __imp_??1?$CStringT@DV?$StrTraitMFC_DLL@DV?$ChTraitsCRT@D@ATL@@@@@ATL@@QAE@XZ 0042697c     mfc90:mfc90.dll
 0002:00000980       __imp_??4?$CStringT@DV?$StrTraitMFC_DLL@DV?$ChTraitsCRT@D@ATL@@@@@ATL@@QAEAAV01@ABV01@@Z 00426980     mfc90:mfc90.dll
 0002:00000984       __imp_??0?$CStringT@DV?$StrTraitMFC_DLL@DV?$ChTraitsCRT@D@ATL@@@@@ATL@@QAE@ABV01@@Z 00426984     mfc90:mfc90.dll
 0002:00000988       __imp_??_V@YAXPAX@Z        00426988     mfc90:mfc90.dll
 0002:0000098c       __imp_?GetRuntimeClass@CCriticalSection@@UBEPAUCRuntimeClass@@XZ 0042698c     mfc90:mfc90.dll
 0002:00000990       __imp_??0CSyncObject@@QAE@PBD@Z 00426990     mfc90:mfc90.dll
 0002:00000994       __imp_?AfxThrowMemoryException@@YGXXZ 00426994     mfc90:mfc90.dll
 0002:00000998       __imp_??1CSyncObject@@UAE@XZ 00426998     mfc90:mfc90.dll
 0002:0000099c       __imp_??0CPtrList@@QAE@H@Z 0042699c     mfc90:mfc90.dll
 0002:000009a0       __imp_?GetRuntimeClass@CPtrList@@UBEPAUCRuntimeClass@@XZ 004269a0     mfc90:mfc90.dll
 0002:000009a4       __imp_??1CPtrList@@UAE@XZ  004269a4     mfc90:mfc90.dll
 0002:000009a8       __imp_??3@YAXPAX@Z         004269a8     mfc90:mfc90.dll
 0002:000009ac       __imp_?OnUpdateFrameTitle@CFrameWndEx@@UAEXH@Z 004269ac     mfc90:mfc90.dll
 0002:000009b0       __imp_?OnHideMenuBar@CFrameWnd@@MAEXXZ 004269b0     mfc90:mfc90.dll
 0002:000009b4       \177mfc90_NULL_THUNK_DATA  004269b4     mfc90:mfc90.dll
 0002:000009b8       __imp__CoInitialize@4      004269b8     ole32:ole32.dll
 0002:000009bc       __imp__CoInitializeSecurity@36 004269bc     ole32:ole32.dll
 0002:000009c0       __imp__CoUninitialize@0    004269c0     ole32:ole32.dll
 0002:000009c4       __imp__CoCreateInstance@20 004269c4     ole32:ole32.dll
 0002:000009c8       \177ole32_NULL_THUNK_DATA  004269c8     ole32:ole32.dll
 0002:000009cc       __imp__ExDetectProtect     004269cc     windisk:windisk.dll
 0002:000009d0       __imp__ExRWDiskAbs         004269d0     windisk:windisk.dll
 0002:000009d4       __imp__ExRWDisk            004269d4     windisk:windisk.dll
 0002:000009d8       \177windisk_NULL_THUNK_DATA 004269d8     windisk:windisk.dll
 0002:000009dc       ___xc_a                    004269dc     msvcrt:cinitexe.obj
 0002:00000a1c       ___xc_z                    00426a1c     msvcrt:cinitexe.obj
 0002:00000a20       ___xi_a                    00426a20     msvcrt:cinitexe.obj
 0002:00000a30       ___xi_z                    00426a30     msvcrt:cinitexe.obj
 0002:00000ae4       ??_7CBootModuleManager@@6B@ 00426ae4     BootModuleManager.obj
 0002:00000aec       ??_7?$CTypedPtrList@VCPtrList@@PAK@@6B@ 00426aec     BootModuleManager.obj
 0002:00000b04       ??_7?$_CTypedPtrList@VCPtrList@@PAK@@6B@ 00426b04     BootModuleManager.obj
 0002:00000b1c       ??_7CCriticalSection@@6B@  00426b1c     BootModuleManager.obj
 0002:00000dc8       ??_7CErrorMessage@@6B@     00426dc8     ChatDlg.obj
 0002:00000dd0       ??_7CErrorTable@@6B@       00426dd0     ChatDlg.obj
 0002:00000dd8       ??_7CInstall@@6B@          00426dd8     ChatDlg.obj
 0002:00000de4       ??_7CChatDlg@@6B@          00426de4     ChatDlg.obj
 0002:00000fa4       ??_7CStatic@@6B@           00426fa4     ChatDlg.obj
 0002:00001174       ??_7CCheckPasswordDlg@@6B@ 00427174     CheckPasswordDlg.obj
 0002:0000134c       ??_7CEdit@@6B@             0042734c     CheckPasswordDlg.obj
 0002:0000199c       ?classCDialogInputname@CDialogInputname@@2UCRuntimeClass@@B 0042799c     DialogInputname.obj
 0002:000019bc       ??_7CDialogInputname@@6B@  004279bc     DialogInputname.obj
 0002:00001f80       ?classCFtpClientDlg@CFtpClientDlg@@2UCRuntimeClass@@B 00427f80     FtpClientDlg.obj
 0002:00001fa4       ??_7CFtpClientDlg@@6B@     00427fa4     FtpClientDlg.obj
 0002:000025d4       ??_7CKiboClientApp@@6B@    004285d4     KiboClient.obj
 0002:000026d4       ??_7CAboutDlg@@6B@         004286d4     KiboClient.obj
 0002:00004790       ?classCMainFrame@CMainFrame@@2UCRuntimeClass@@B 0042a790     MainFrm.obj
 0002:000047bc       ??_7CMainFrame@@6B@        0042a7bc     MainFrm.obj
 0002:00004998       ??_7?$CTypedPtrList@VCPtrList@@PAUtagRECVREQUEST@@@@6B@ 0042a998     MainFrm.obj
 0002:000049b0       ??_7?$_CTypedPtrList@VCPtrList@@PAUtagRECVREQUEST@@@@6B@ 0042a9b0     MainFrm.obj
 0002:000049c8       ??_7CMenu@@6B@             0042a9c8     MainFrm.obj
 0002:000049e4       ??_C@_0L@LBHJMCDF@?$CFs?5?$CI?$CFs?3?$CFd?$CJ?$AA@ 0042a9e4     MainFrm.obj
 0002:000049f0       ??_C@_0O@KHJMBFME@?$CFs?5?$CI?$CFs?3?$CFd?$CJ?6?$CFs?$AA@ 0042a9f0     MainFrm.obj
 0002:00004a00       ??_C@_0BP@OIEOKIDM@Exception?5thrown?5in?5destructor?$AA@ 0042aa00     MainFrm.obj
 0002:00004a20       ??_C@_0EL@GPEBOPMF@H?3?2Program?5Files?2Microsoft?5Visua@ 0042aa20     MainFrm.obj
 0002:00004b04       ??_7CMyRichEdit@@6B@       0042ab04     MyRichEdit.obj
 0002:00004d10       ??_C@_00CNPNBAHC@?$AA@     0042ad10     MyRichEdit.obj
 0002:00004d1c       ??_7CRichEditCtrl@@6B@     0042ad1c     MyRichEdit.obj
 0002:00005058       ?classCPortChannelDlg@CPortChannelDlg@@2UCRuntimeClass@@B 0042b058     PortChannelDlg.obj
 0002:0000507c       ??_7CPortChannelDlg@@6B@   0042b07c     PortChannelDlg.obj
 0002:00005e18       ??_7CPropertyManager@@6B@  0042be18     PropertyManager.obj
 0002:00005e20       ??_7?$CTypedPtrList@VCPtrList@@PAUtagPROPERTY_REQUEST@@@@6B@ 0042be20     PropertyManager.obj
 0002:00005e38       ??_7?$_CTypedPtrList@VCPtrList@@PAUtagPROPERTY_REQUEST@@@@6B@ 0042be38     PropertyManager.obj
 0002:00005f64       ?classCSetDrfaultNICDlg@CSetDrfaultNICDlg@@2UCRuntimeClass@@B 0042bf64     SetDrfaultNICDlg.obj
 0002:00005f84       ??_7CSetDrfaultNICDlg@@6B@ 0042bf84     SetDrfaultNICDlg.obj
 0002:0000612c       ??_7CComboBox@@6B@         0042c12c     SetDrfaultNICDlg.obj
 0002:00006398       ??_C@_01MCMALHOG@a?$AA@    0042c398     comfunc:comfunc.obj
 0002:0000639c       ??_C@_0BE@POPFGFGJ@SeShutdownPrivilege?$AA@ 0042c39c     comfunc:comfunc.obj
 0002:000063b0       ??_C@_0BB@ICFLKOPM@SeDebugPrivilege?$AA@ 0042c3b0     comfunc:comfunc.obj
 0002:000063c4       ??_C@_08PNLNEKOB@kernel32?$AA@ 0042c3c4     comfunc:comfunc.obj
 0002:000063d0       ??_C@_0P@LKABJJMO@IsWow64Process?$AA@ 0042c3d0     comfunc:comfunc.obj
 0002:000063e0       ??_C@_04PFOHOKJK@?5?5?5?5?$AA@ 0042c3e0     comfunc:comfunc.obj
 0002:000063e8       ??_C@_01EEMJAFIK@?6?$AA@   0042c3e8     comfunc:comfunc.obj
 0002:000063ec       ??_C@_0BN@JIAHOFFK@?$CFd?4?$CF02d?4?$CF02d?5?5?$CF02d?3?$CF02d?3?$CF02d?$AA@ 0042c3ec     comfunc:comfunc.obj
 0002:0000640c       ??_C@_0L@NCKBCEGF@runlog?4txt?$AA@ 0042c40c     comfunc:comfunc.obj
 0002:00006418       ??_C@_0BH@OHOHHLFP@Get?5system?5type?5error?$CB?$AA@ 0042c418     comfunc:comfunc.obj
 0002:00006430       ??_C@_0L@NEBNHFIE@Windows?595?$AA@ 0042c430     comfunc:comfunc.obj
 0002:0000643c       ??_C@_0L@GBLDALMJ@Windows?598?$AA@ 0042c43c     comfunc:comfunc.obj
 0002:00006448       ??_C@_0BD@KOHFHFOF@Windows?5Mellinnium?$AA@ 0042c448     comfunc:comfunc.obj
 0002:0000645c       ??_C@_0O@IFKHFILP@Windows?5Vista?$AA@ 0042c45c     comfunc:comfunc.obj
 0002:0000646c       ??_C@_0N@MEKDBOKB@Windows?52000?$AA@ 0042c46c     comfunc:comfunc.obj
 0002:0000647c       ??_C@_0L@IFICELHB@Windows?5XP?$AA@ 0042c47c     comfunc:comfunc.obj
 0002:00006488       ??_C@_0BE@IEOLCCDL@Windows?5Server?52003?$AA@ 0042c488     comfunc:comfunc.obj
 0002:0000649c       ??_C@_0N@EMOGDPPI@Windows?5XP64?$AA@ 0042c49c     comfunc:comfunc.obj
 0002:000064ac       ??_C@_0BO@KOKDPNHB@Comfunc?3?5GetVersionEx?5error2?$CB?$AA@ 0042c4ac     comfunc:comfunc.obj
 0002:000064cc       ??_C@_0P@PHKJNOLH@Windows?5NT?54?40?$AA@ 0042c4cc     comfunc:comfunc.obj
 0002:000064dc       ??_C@_0BA@CHEEJGLI@Windows?5NT?53?451?$AA@ 0042c4dc     comfunc:comfunc.obj
 0002:000064ec       ??_C@_0P@LKDDHMEK@Unknown?5System?$AA@ 0042c4ec     comfunc:comfunc.obj
 0002:000064fc       ??_C@_0BO@KMOFEDCI@Comfunc?3?5GetVersionEx?5error1?$CB?$AA@ 0042c4fc     comfunc:comfunc.obj
 0002:0000651c       ??_C@_09EEDNEKAE@enabledbg?$AA@ 0042c51c     comfunc:comfunc.obj
 0002:00006528       ??_C@_0BA@FDJEPFGB@Software?2Saming?$AA@ 0042c528     comfunc:comfunc.obj
 0002:00006538       ??_C@_0BJ@GKGENCBH@?$CF02X?$CF02X?$CF02X?$CF02X?$CF02X?$CF02X?$AA@ 0042c538     helpful:helpful.obj
 0002:00006554       ??_C@_04LAGKFANA@ssdd?$AA@ 0042c554     commod2:MulticastSocket.obj
 0002:00006560       ??_7?$CTypedPtrList@VCPtrList@@PAUtagUDPRECV@@@@6B@ 0042c560     commod2:MulticastSocket.obj
 0002:00006574       ??_C@_0CL@DJBNJEFG@CMulticastSocket?3?5Failed?5during?5@ 0042c574     commod2:MulticastSocket.obj
 0002:000065a4       ??_7CMulticastSocket@@6B@  0042c5a4     commod2:MulticastSocket.obj
 0002:000065a8       ??_C@_0BB@CBHBLOIH@Para?5flag?5error?$CB?$AA@ 0042c5a8     kibokern:kibokern.obj
 0002:000065bc       ??_C@_0BM@PEOJADO@Para?5sector?5checksum?5error?$CB?$AA@ 0042c5bc     kibokern:kibokern.obj
 0002:000065d8       ??_C@_07NFANNNEC@UNKNOWN?$AA@ 0042c5d8     kibokern:kibokern.obj
 0002:000065e0       ??_C@_04NLFHDAEB@SWAP?$AA@ 0042c5e0     kibokern:kibokern.obj
 0002:000065e8       ??_C@_04CBLCCKIL@EXT2?$AA@ 0042c5e8     kibokern:kibokern.obj
 0002:000065f0       ??_C@_04HPPAIJNK@NTFS?$AA@ 0042c5f0     kibokern:kibokern.obj
 0002:000065f8       ??_C@_05HNJNFBJJ@FAT32?$AA@ 0042c5f8     kibokern:kibokern.obj
 0002:00006600       ??_C@_05BKHFEAPD@FAT16?$AA@ 0042c600     kibokern:kibokern.obj
 0002:00006608       ??_C@_01JOAMLHOP@?9?$AA@   0042c608     kibokern:kibokern.obj
 0002:0000660c       ??_C@_03BOCCJCAP@?$CFC?3?$AA@ 0042c60c     kibokern:kibokern.obj
 0002:00006614       ??_7?$CTypedPtrList@VCPtrList@@PAUSTRUCT_PROTECTITEM@@@@6B@ 0042c614     kibokern:kibokern.obj
 0002:0000662c       ??_7CKiboKern@@6B@         0042c62c     kibokern:kibokern.obj
 0002:00006630       ??_C@_02JOGGLHBA@?2n?$AA@  0042c630     loadres:exloadres.obj
 0002:00006634       ??_C@_0M@DEBJHILM@?2string?4ini?$AA@ 0042c634     loadres:exloadres.obj
 0002:00006640       ??_C@_07GACLGDNA@novalue?$AA@ 0042c640     loadres:exloadres.obj
 0002:00006648       ??_C@_0CC@EOMOIDBP@Resource?5error?3File?5?$CFs?5not?5exist@ 0042c648     loadres:exloadres.obj
 0002:0000666c       ??_C@_08DALEMBDJ@?2bmp?4ini?$AA@ 0042c66c     loadres:exloadres.obj
 0002:00006678       ??_C@_0BG@IADDKNOI@resource?5lib?5is?5bad2?$CB?$AA@ 0042c678     loadres:exloadres.obj
 0002:00006690       ??_C@_03CAKEDOOO@bmp?$AA@  0042c690     loadres:exloadres.obj
 0002:00006694       ??_C@_0BB@JBENNHDF@IDS_PRODUCT_NAME?$AA@ 0042c694     loadres:exloadres.obj
 0002:000066a8       ??_C@_06ICGJLFIM@string?$AA@ 0042c6a8     loadres:exloadres.obj
 0002:000066b0       ??_C@_09BADPAGCD@$product$?$AA@ 0042c6b0     loadres:exloadres.obj
 0002:000066bc       ??_C@_0BG@ICHFBDLB@resource?5lib?5is?5bad1?$CB?$AA@ 0042c6bc     loadres:exloadres.obj
 0002:000066d4       ??_C@_0BE@EOONMDND@Can?8t?5find?5file?5?$CFs?$CB?$AA@ 0042c6d4     loadres:exloadres.obj
 0002:000066e8       ??_C@_06BGHBJFGM@reschk?$AA@ 0042c6e8     loadres:exloadres.obj
 0002:000066f0       ??_C@_0BM@OKCEOKKE@File?5?$CFs?0section?5?$CFs?5too?5big?$CB?$AA@ 0042c6f0     loadres:initwork.obj
 0002:0000670c       ??_C@_0O@BANLFAHC@?$CFCURRENT_DIR?$CF?$AA@ 0042c70c     loadres:initwork.obj
 0002:0000671c       ??_C@_07CLEHDIEJ@replace?$AA@ 0042c71c     loadres:initwork.obj
 0002:00006724       ??_C@_0DK@JCHLPDBB@Resource?5error?3File?5?$CFs?0section?5?$CF@ 0042c724     loadres:initwork.obj
 0002:00006760       ??_C@_0CJ@OCLBFGHK@File?5?$CFs?0section?5?$CFs?0key?5?$CFs?5value?5@ 0042c760     loadres:initwork.obj
 0002:00006790       __sz_dwmapi_dll            0042c790     dwmapi:dwmapi.dll
 0002:0000679c       ??_C@_06JBKGCNBB@Delete?$AA@ 0042c79c     mfcs90:nolib.obj
 0002:000067a4       ??_C@_08KAAPDIAN@NoRemove?$AA@ 0042c7a4     mfcs90:nolib.obj
 0002:000067b0       ??_C@_0M@DBGDLGLL@ForceRemove?$AA@ 0042c7b0     mfcs90:nolib.obj
 0002:000067bc       ??_C@_03LAIAPFCB@Val?$AA@  0042c7bc     mfcs90:nolib.obj
 0002:000067c0       ??_C@_01HMGJMAIH@B?$AA@    0042c7c0     mfcs90:nolib.obj
 0002:000067c4       ??_C@_01CKDDGHAB@D?$AA@    0042c7c4     mfcs90:nolib.obj
 0002:000067c8       ??_C@_01PLPBNMEI@M?$AA@    0042c7c8     mfcs90:nolib.obj
 0002:000067cc       ??_C@_01CPLAODJH@S?$AA@    0042c7cc     mfcs90:nolib.obj
 0002:00006814       ??_7type_info@@6B@         0042c814     msvcrt:ti_inst.obj
 0002:00006820       _IID_IUnknown              0042c820     uuid:unknwn_i.obj
 0002:00006830       ??_7_com_error@@6B@        0042c830     comsuppw:comraise.obj
 0002:00006834       _LIBID_WbemProviders_v1    0042c834     wbemuuid:wbemprov_i.obj
 0002:00006844       _IID_IWbemPropertyProvider 0042c844     wbemuuid:wbemprov_i.obj
 0002:00006854       _IID_IWbemUnboundObjectSink 0042c854     wbemuuid:wbemprov_i.obj
 0002:00006864       _IID_IWbemEventProvider    0042c864     wbemuuid:wbemprov_i.obj
 0002:00006874       _IID_IWbemEventProviderQuerySink 0042c874     wbemuuid:wbemprov_i.obj
 0002:00006884       _IID_IWbemEventProviderSecurity 0042c884     wbemuuid:wbemprov_i.obj
 0002:00006894       _IID_IWbemEventConsumerProvider 0042c894     wbemuuid:wbemprov_i.obj
 0002:000068a4       _IID_IWbemProviderInitSink 0042c8a4     wbemuuid:wbemprov_i.obj
 0002:000068b4       _IID_IWbemProviderInit     0042c8b4     wbemuuid:wbemprov_i.obj
 0002:000068c4       _IID_IWbemHiPerfProvider   0042c8c4     wbemuuid:wbemprov_i.obj
 0002:000068d4       _IID_IWbemDecoupledRegistrar 0042c8d4     wbemuuid:wbemprov_i.obj
 0002:000068e4       _CLSID_WbemAdministrativeLocator 0042c8e4     wbemuuid:wbemprov_i.obj
 0002:000068f4       _CLSID_WbemAuthenticatedLocator 0042c8f4     wbemuuid:wbemprov_i.obj
 0002:00006904       _CLSID_WbemUnauthenticatedLocator 0042c904     wbemuuid:wbemprov_i.obj
 0002:00006914       _CLSID_WbemDecoupledRegistrar 0042c914     wbemuuid:wbemprov_i.obj
 0002:00006924       _CLSID_WbemDecoupledBasicEventProvider 0042c924     wbemuuid:wbemprov_i.obj
 0002:00006934       _IID_IWbemProviderIdentity 0042c934     wbemuuid:wbemprov_i.obj
 0002:00006944       _IID_IWbemDecoupledBasicEventProvider 0042c944     wbemuuid:wbemprov_i.obj
 0002:00006954       _IID_IWbemEventSink        0042c954     wbemuuid:wbemprov_i.obj
 0002:00006964       _LIBID_WbemClient_v1       0042c964     wbemuuid:wbemcli_i.obj
 0002:00006974       _IID_IWbemClassObject      0042c974     wbemuuid:wbemcli_i.obj
 0002:00006984       _IID_IWbemObjectAccess     0042c984     wbemuuid:wbemcli_i.obj
 0002:00006994       _IID_IWbemQualifierSet     0042c994     wbemuuid:wbemcli_i.obj
 0002:000069a4       _IID_IWbemServices         0042c9a4     wbemuuid:wbemcli_i.obj
 0002:000069b4       _IID_IWbemLocator          0042c9b4     wbemuuid:wbemcli_i.obj
 0002:000069c4       _IID_IWbemObjectSink       0042c9c4     wbemuuid:wbemcli_i.obj
 0002:000069d4       _IID_IEnumWbemClassObject  0042c9d4     wbemuuid:wbemcli_i.obj
 0002:000069e4       _IID_IWbemCallResult       0042c9e4     wbemuuid:wbemcli_i.obj
 0002:000069f4       _IID_IWbemContext          0042c9f4     wbemuuid:wbemcli_i.obj
 0002:00006a04       _IID_IUnsecuredApartment   0042ca04     wbemuuid:wbemcli_i.obj
 0002:00006a14       _IID_IWbemUnsecuredApartment 0042ca14     wbemuuid:wbemcli_i.obj
 0002:00006a24       _IID_IWbemStatusCodeText   0042ca24     wbemuuid:wbemcli_i.obj
 0002:00006a34       _IID_IWbemBackupRestore    0042ca34     wbemuuid:wbemcli_i.obj
 0002:00006a44       _IID_IWbemBackupRestoreEx  0042ca44     wbemuuid:wbemcli_i.obj
 0002:00006a54       _IID_IWbemRefresher        0042ca54     wbemuuid:wbemcli_i.obj
 0002:00006a64       _IID_IWbemHiPerfEnum       0042ca64     wbemuuid:wbemcli_i.obj
 0002:00006a74       _IID_IWbemConfigureRefresher 0042ca74     wbemuuid:wbemcli_i.obj
 0002:00006a84       _CLSID_WbemLocator         0042ca84     wbemuuid:wbemcli_i.obj
 0002:00006a94       _CLSID_WbemContext         0042ca94     wbemuuid:wbemcli_i.obj
 0002:00006aa4       _CLSID_UnsecuredApartment  0042caa4     wbemuuid:wbemcli_i.obj
 0002:00006ab4       _CLSID_WbemClassObject     0042cab4     wbemuuid:wbemcli_i.obj
 0002:00006ac4       _CLSID_MofCompiler         0042cac4     wbemuuid:wbemcli_i.obj
 0002:00006ad4       _CLSID_WbemStatusCodeText  0042cad4     wbemuuid:wbemcli_i.obj
 0002:00006ae4       _CLSID_WbemBackupRestore   0042cae4     wbemuuid:wbemcli_i.obj
 0002:00006af4       _CLSID_WbemRefresher       0042caf4     wbemuuid:wbemcli_i.obj
 0002:00006b04       _CLSID_WbemObjectTextSrc   0042cb04     wbemuuid:wbemcli_i.obj
 0002:00006b14       _IID_IWbemShutdown         0042cb14     wbemuuid:wbemcli_i.obj
 0002:00006b24       _IID_IWbemObjectTextSrc    0042cb24     wbemuuid:wbemcli_i.obj
 0002:00006b34       _IID_IMofCompiler          0042cb34     wbemuuid:wbemcli_i.obj
 0002:00006b68       __load_config_used         0042cb68     msvcrt:loadcfg.obj
 0002:00006bfc       ??_R4CBootModuleManager@@6B@ 0042cbfc     BootModuleManager.obj
 0002:00006c10       ??_R3CBootModuleManager@@8 0042cc10     BootModuleManager.obj
 0002:00006c20       ??_R2CBootModuleManager@@8 0042cc20     BootModuleManager.obj
 0002:00006c28       ??_R1A@?0A@EA@CBootModuleManager@@8 0042cc28     BootModuleManager.obj
 0002:00006c44       ??_R4?$CTypedPtrList@VCPtrList@@PAK@@6B@ 0042cc44     BootModuleManager.obj
 0002:00006c58       ??_R3?$CTypedPtrList@VCPtrList@@PAK@@8 0042cc58     BootModuleManager.obj
 0002:00006c68       ??_R2?$CTypedPtrList@VCPtrList@@PAK@@8 0042cc68     BootModuleManager.obj
 0002:00006c7c       ??_R1A@?0A@EA@?$CTypedPtrList@VCPtrList@@PAK@@8 0042cc7c     BootModuleManager.obj
 0002:00006c98       ??_R1A@?0A@EA@?$_CTypedPtrList@VCPtrList@@PAK@@8 0042cc98     BootModuleManager.obj
 0002:00006cb4       ??_R3?$_CTypedPtrList@VCPtrList@@PAK@@8 0042ccb4     BootModuleManager.obj
 0002:00006cc4       ??_R2?$_CTypedPtrList@VCPtrList@@PAK@@8 0042ccc4     BootModuleManager.obj
 0002:00006cd4       ??_R1A@?0A@EA@CPtrList@@8  0042ccd4     BootModuleManager.obj
 0002:00006cf0       ??_R3CPtrList@@8           0042ccf0     BootModuleManager.obj
 0002:00006d00       ??_R2CPtrList@@8           0042cd00     BootModuleManager.obj
 0002:00006d0c       ??_R1A@?0A@EA@CObject@@8   0042cd0c     BootModuleManager.obj
 0002:00006d28       ??_R3CObject@@8            0042cd28     BootModuleManager.obj
 0002:00006d38       ??_R2CObject@@8            0042cd38     BootModuleManager.obj
 0002:00006d40       ??_R4?$_CTypedPtrList@VCPtrList@@PAK@@6B@ 0042cd40     BootModuleManager.obj
 0002:00006d54       ??_R4CCriticalSection@@6B@ 0042cd54     BootModuleManager.obj
 0002:00006d68       ??_R3CCriticalSection@@8   0042cd68     BootModuleManager.obj
 0002:00006d78       ??_R2CCriticalSection@@8   0042cd78     BootModuleManager.obj
 0002:00006d88       ??_R1A@?0A@EA@CCriticalSection@@8 0042cd88     BootModuleManager.obj
 0002:00006da4       ??_R1A@?0A@EA@CSyncObject@@8 0042cda4     BootModuleManager.obj
 0002:00006dc0       ??_R3CSyncObject@@8        0042cdc0     BootModuleManager.obj
 0002:00006dd0       ??_R2CSyncObject@@8        0042cdd0     BootModuleManager.obj
 0002:00006ddc       ??_R4CErrorMessage@@6B@    0042cddc     ChatDlg.obj
 0002:00006df0       ??_R3CErrorMessage@@8      0042cdf0     ChatDlg.obj
 0002:00006e00       ??_R2CErrorMessage@@8      0042ce00     ChatDlg.obj
 0002:00006e08       ??_R1A@?0A@EA@CErrorMessage@@8 0042ce08     ChatDlg.obj
 0002:00006e24       ??_R4CErrorTable@@6B@      0042ce24     ChatDlg.obj
 0002:00006e38       ??_R3CErrorTable@@8        0042ce38     ChatDlg.obj
 0002:00006e48       ??_R2CErrorTable@@8        0042ce48     ChatDlg.obj
 0002:00006e50       ??_R1A@?0A@EA@CErrorTable@@8 0042ce50     ChatDlg.obj
 0002:00006e6c       ??_R4CInstall@@6B@         0042ce6c     ChatDlg.obj
 0002:00006e80       ??_R3CInstall@@8           0042ce80     ChatDlg.obj
 0002:00006e90       ??_R2CInstall@@8           0042ce90     ChatDlg.obj
 0002:00006e98       ??_R1A@?0A@EA@CInstall@@8  0042ce98     ChatDlg.obj
 0002:00006eb4       ??_R4CChatDlg@@6B@         0042ceb4     ChatDlg.obj
 0002:00006ec8       ??_R3CChatDlg@@8           0042cec8     ChatDlg.obj
 0002:00006ed8       ??_R2CChatDlg@@8           0042ced8     ChatDlg.obj
 0002:00006ef0       ??_R1A@?0A@EA@CChatDlg@@8  0042cef0     ChatDlg.obj
 0002:00006f0c       ??_R1A@?0A@EA@CDialog@@8   0042cf0c     ChatDlg.obj
 0002:00006f28       ??_R3CDialog@@8            0042cf28     ChatDlg.obj
 0002:00006f38       ??_R2CDialog@@8            0042cf38     ChatDlg.obj
 0002:00006f4c       ??_R1A@?0A@EA@CWnd@@8      0042cf4c     ChatDlg.obj
 0002:00006f68       ??_R3CWnd@@8               0042cf68     ChatDlg.obj
 0002:00006f78       ??_R2CWnd@@8               0042cf78     ChatDlg.obj
 0002:00006f88       ??_R1A@?0A@EA@CCmdTarget@@8 0042cf88     ChatDlg.obj
 0002:00006fa4       ??_R3CCmdTarget@@8         0042cfa4     ChatDlg.obj
 0002:00006fb4       ??_R2CCmdTarget@@8         0042cfb4     ChatDlg.obj
 0002:00006fc0       ??_R4CStatic@@6B@          0042cfc0     ChatDlg.obj
 0002:00006fd4       ??_R3CStatic@@8            0042cfd4     ChatDlg.obj
 0002:00006fe4       ??_R2CStatic@@8            0042cfe4     ChatDlg.obj
 0002:00006ff8       ??_R1A@?0A@EA@CStatic@@8   0042cff8     ChatDlg.obj
 0002:00007014       ??_R4CCheckPasswordDlg@@6B@ 0042d014     CheckPasswordDlg.obj
 0002:00007028       ??_R3CCheckPasswordDlg@@8  0042d028     CheckPasswordDlg.obj
 0002:00007038       ??_R2CCheckPasswordDlg@@8  0042d038     CheckPasswordDlg.obj
 0002:00007050       ??_R1A@?0A@EA@CCheckPasswordDlg@@8 0042d050     CheckPasswordDlg.obj
 0002:0000706c       ??_R4CEdit@@6B@            0042d06c     CheckPasswordDlg.obj
 0002:00007080       ??_R3CEdit@@8              0042d080     CheckPasswordDlg.obj
 0002:00007090       ??_R2CEdit@@8              0042d090     CheckPasswordDlg.obj
 0002:000070a4       ??_R1A@?0A@EA@CEdit@@8     0042d0a4     CheckPasswordDlg.obj
 0002:000070c0       ??_R4CDialogInputname@@6B@ 0042d0c0     DialogInputname.obj
 0002:000070d4       ??_R3CDialogInputname@@8   0042d0d4     DialogInputname.obj
 0002:000070e4       ??_R2CDialogInputname@@8   0042d0e4     DialogInputname.obj
 0002:000070fc       ??_R1A@?0A@EA@CDialogInputname@@8 0042d0fc     DialogInputname.obj
 0002:00007118       ??_R4CFtpClientDlg@@6B@    0042d118     FtpClientDlg.obj
 0002:0000712c       ??_R3CFtpClientDlg@@8      0042d12c     FtpClientDlg.obj
 0002:0000713c       ??_R2CFtpClientDlg@@8      0042d13c     FtpClientDlg.obj
 0002:00007154       ??_R1A@?0A@EA@CFtpClientDlg@@8 0042d154     FtpClientDlg.obj
 0002:00007170       ??_R1A@?0A@EA@CWinThread@@8 0042d170     FtpClientDlg.obj
 0002:0000718c       ??_R3CWinThread@@8         0042d18c     FtpClientDlg.obj
 0002:0000719c       ??_R2CWinThread@@8         0042d19c     FtpClientDlg.obj
 0002:000071ac       ??_R4CKiboClientApp@@6B@   0042d1ac     KiboClient.obj
 0002:000071c0       ??_R3CKiboClientApp@@8     0042d1c0     KiboClient.obj
 0002:000071d0       ??_R2CKiboClientApp@@8     0042d1d0     KiboClient.obj
 0002:000071ec       ??_R1A@?0A@EA@CKiboClientApp@@8 0042d1ec     KiboClient.obj
 0002:00007208       ??_R1A@?0A@EA@CWinAppEx@@8 0042d208     KiboClient.obj
 0002:00007224       ??_R3CWinAppEx@@8          0042d224     KiboClient.obj
 0002:00007234       ??_R2CWinAppEx@@8          0042d234     KiboClient.obj
 0002:0000724c       ??_R1A@?0A@EA@CWinApp@@8   0042d24c     KiboClient.obj
 0002:00007268       ??_R3CWinApp@@8            0042d268     KiboClient.obj
 0002:00007278       ??_R2CWinApp@@8            0042d278     KiboClient.obj
 0002:0000728c       ??_R4CAboutDlg@@6B@        0042d28c     KiboClient.obj
 0002:000072a0       ??_R3CAboutDlg@@8          0042d2a0     KiboClient.obj
 0002:000072b0       ??_R2CAboutDlg@@8          0042d2b0     KiboClient.obj
 0002:000072c8       ??_R1A@?0A@EA@CAboutDlg@@8 0042d2c8     KiboClient.obj
 0002:000072e4       ??_R4CMainFrame@@6B@       0042d2e4     MainFrm.obj
 0002:000072f8       ??_R3CMainFrame@@8         0042d2f8     MainFrm.obj
 0002:00007308       ??_R2CMainFrame@@8         0042d308     MainFrm.obj
 0002:00007324       ??_R1A@?0A@EA@CMainFrame@@8 0042d324     MainFrm.obj
 0002:00007340       ??_R1A@?0A@EA@CFrameWndEx@@8 0042d340     MainFrm.obj
 0002:0000735c       ??_R3CFrameWndEx@@8        0042d35c     MainFrm.obj
 0002:0000736c       ??_R2CFrameWndEx@@8        0042d36c     MainFrm.obj
 0002:00007384       ??_R1A@?0A@EA@CFrameWnd@@8 0042d384     MainFrm.obj
 0002:000073a0       ??_R3CFrameWnd@@8          0042d3a0     MainFrm.obj
 0002:000073b0       ??_R2CFrameWnd@@8          0042d3b0     MainFrm.obj
 0002:000073c4       ??_R4?$CTypedPtrList@VCPtrList@@PAUtagRECVREQUEST@@@@6B@ 0042d3c4     MainFrm.obj
 0002:000073d8       ??_R3?$CTypedPtrList@VCPtrList@@PAUtagRECVREQUEST@@@@8 0042d3d8     MainFrm.obj
 0002:000073e8       ??_R2?$CTypedPtrList@VCPtrList@@PAUtagRECVREQUEST@@@@8 0042d3e8     MainFrm.obj
 0002:000073fc       ??_R1A@?0A@EA@?$CTypedPtrList@VCPtrList@@PAUtagRECVREQUEST@@@@8 0042d3fc     MainFrm.obj
 0002:00007418       ??_R1A@?0A@EA@?$_CTypedPtrList@VCPtrList@@PAUtagRECVREQUEST@@@@8 0042d418     MainFrm.obj
 0002:00007434       ??_R3?$_CTypedPtrList@VCPtrList@@PAUtagRECVREQUEST@@@@8 0042d434     MainFrm.obj
 0002:00007444       ??_R2?$_CTypedPtrList@VCPtrList@@PAUtagRECVREQUEST@@@@8 0042d444     MainFrm.obj
 0002:00007454       ??_R4?$_CTypedPtrList@VCPtrList@@PAUtagRECVREQUEST@@@@6B@ 0042d454     MainFrm.obj
 0002:00007468       ??_R4CMenu@@6B@            0042d468     MainFrm.obj
 0002:0000747c       ??_R3CMenu@@8              0042d47c     MainFrm.obj
 0002:0000748c       ??_R2CMenu@@8              0042d48c     MainFrm.obj
 0002:00007498       ??_R1A@?0A@EA@CMenu@@8     0042d498     MainFrm.obj
 0002:000074b4       ??_R4CMyRichEdit@@6B@      0042d4b4     MyRichEdit.obj
 0002:000074c8       ??_R3CMyRichEdit@@8        0042d4c8     MyRichEdit.obj
 0002:000074d8       ??_R2CMyRichEdit@@8        0042d4d8     MyRichEdit.obj
 0002:000074f0       ??_R1A@?0A@EA@CMyRichEdit@@8 0042d4f0     MyRichEdit.obj
 0002:0000750c       ??_R1A@?0A@EA@CRichEditCtrl@@8 0042d50c     MyRichEdit.obj
 0002:00007528       ??_R3CRichEditCtrl@@8      0042d528     MyRichEdit.obj
 0002:00007538       ??_R2CRichEditCtrl@@8      0042d538     MyRichEdit.obj
 0002:0000754c       ??_R4CRichEditCtrl@@6B@    0042d54c     MyRichEdit.obj
 0002:00007560       ??_R4CPortChannelDlg@@6B@  0042d560     PortChannelDlg.obj
 0002:00007574       ??_R3CPortChannelDlg@@8    0042d574     PortChannelDlg.obj
 0002:00007584       ??_R2CPortChannelDlg@@8    0042d584     PortChannelDlg.obj
 0002:0000759c       ??_R1A@?0A@EA@CPortChannelDlg@@8 0042d59c     PortChannelDlg.obj
 0002:000075b8       ??_R4CPropertyManager@@6B@ 0042d5b8     PropertyManager.obj
 0002:000075cc       ??_R3CPropertyManager@@8   0042d5cc     PropertyManager.obj
 0002:000075dc       ??_R2CPropertyManager@@8   0042d5dc     PropertyManager.obj
 0002:000075e4       ??_R1A@?0A@EA@CPropertyManager@@8 0042d5e4     PropertyManager.obj
 0002:00007600       ??_R4?$CTypedPtrList@VCPtrList@@PAUtagPROPERTY_REQUEST@@@@6B@ 0042d600     PropertyManager.obj
 0002:00007614       ??_R3?$CTypedPtrList@VCPtrList@@PAUtagPROPERTY_REQUEST@@@@8 0042d614     PropertyManager.obj
 0002:00007624       ??_R2?$CTypedPtrList@VCPtrList@@PAUtagPROPERTY_REQUEST@@@@8 0042d624     PropertyManager.obj
 0002:00007638       ??_R1A@?0A@EA@?$CTypedPtrList@VCPtrList@@PAUtagPROPERTY_REQUEST@@@@8 0042d638     PropertyManager.obj
 0002:00007654       ??_R1A@?0A@EA@?$_CTypedPtrList@VCPtrList@@PAUtagPROPERTY_REQUEST@@@@8 0042d654     PropertyManager.obj
 0002:00007670       ??_R3?$_CTypedPtrList@VCPtrList@@PAUtagPROPERTY_REQUEST@@@@8 0042d670     PropertyManager.obj
 0002:00007680       ??_R2?$_CTypedPtrList@VCPtrList@@PAUtagPROPERTY_REQUEST@@@@8 0042d680     PropertyManager.obj
 0002:00007690       ??_R4?$_CTypedPtrList@VCPtrList@@PAUtagPROPERTY_REQUEST@@@@6B@ 0042d690     PropertyManager.obj
 0002:000076a4       ??_R4CSetDrfaultNICDlg@@6B@ 0042d6a4     SetDrfaultNICDlg.obj
 0002:000076b8       ??_R3CSetDrfaultNICDlg@@8  0042d6b8     SetDrfaultNICDlg.obj
 0002:000076c8       ??_R2CSetDrfaultNICDlg@@8  0042d6c8     SetDrfaultNICDlg.obj
 0002:000076e0       ??_R1A@?0A@EA@CSetDrfaultNICDlg@@8 0042d6e0     SetDrfaultNICDlg.obj
 0002:000076fc       ??_R4CComboBox@@6B@        0042d6fc     SetDrfaultNICDlg.obj
 0002:00007710       ??_R3CComboBox@@8          0042d710     SetDrfaultNICDlg.obj
 0002:00007720       ??_R2CComboBox@@8          0042d720     SetDrfaultNICDlg.obj
 0002:00007734       ??_R1A@?0A@EA@CComboBox@@8 0042d734     SetDrfaultNICDlg.obj
 0002:00007750       ??_R3?$_CTypedPtrList@VCPtrList@@PAUtagUDPRECV@@@@8 0042d750     commod2:MulticastSocket.obj
 0002:00007760       ??_R2?$_CTypedPtrList@VCPtrList@@PAUtagUDPRECV@@@@8 0042d760     commod2:MulticastSocket.obj
 0002:00007770       ??_R1A@?0A@EA@?$_CTypedPtrList@VCPtrList@@PAUtagUDPRECV@@@@8 0042d770     commod2:MulticastSocket.obj
 0002:0000778c       ??_R4?$CTypedPtrList@VCPtrList@@PAUtagUDPRECV@@@@6B@ 0042d78c     commod2:MulticastSocket.obj
 0002:000077a0       ??_R3?$CTypedPtrList@VCPtrList@@PAUtagUDPRECV@@@@8 0042d7a0     commod2:MulticastSocket.obj
 0002:000077b0       ??_R2?$CTypedPtrList@VCPtrList@@PAUtagUDPRECV@@@@8 0042d7b0     commod2:MulticastSocket.obj
 0002:000077c4       ??_R1A@?0A@EA@?$CTypedPtrList@VCPtrList@@PAUtagUDPRECV@@@@8 0042d7c4     commod2:MulticastSocket.obj
 0002:000077e0       ??_R4CMulticastSocket@@6B@ 0042d7e0     commod2:MulticastSocket.obj
 0002:000077f4       ??_R3CMulticastSocket@@8   0042d7f4     commod2:MulticastSocket.obj
 0002:00007804       ??_R2CMulticastSocket@@8   0042d804     commod2:MulticastSocket.obj
 0002:0000780c       ??_R1A@?0A@EA@CMulticastSocket@@8 0042d80c     commod2:MulticastSocket.obj
 0002:00007828       ??_R3?$_CTypedPtrList@VCPtrList@@PAUSTRUCT_PROTECTITEM@@@@8 0042d828     kibokern:kibokern.obj
 0002:00007838       ??_R2?$_CTypedPtrList@VCPtrList@@PAUSTRUCT_PROTECTITEM@@@@8 0042d838     kibokern:kibokern.obj
 0002:00007848       ??_R1A@?0A@EA@?$_CTypedPtrList@VCPtrList@@PAUSTRUCT_PROTECTITEM@@@@8 0042d848     kibokern:kibokern.obj
 0002:00007864       ??_R4?$CTypedPtrList@VCPtrList@@PAUSTRUCT_PROTECTITEM@@@@6B@ 0042d864     kibokern:kibokern.obj
 0002:00007878       ??_R3?$CTypedPtrList@VCPtrList@@PAUSTRUCT_PROTECTITEM@@@@8 0042d878     kibokern:kibokern.obj
 0002:00007888       ??_R2?$CTypedPtrList@VCPtrList@@PAUSTRUCT_PROTECTITEM@@@@8 0042d888     kibokern:kibokern.obj
 0002:0000789c       ??_R1A@?0A@EA@?$CTypedPtrList@VCPtrList@@PAUSTRUCT_PROTECTITEM@@@@8 0042d89c     kibokern:kibokern.obj
 0002:000078b8       ??_R4CKiboKern@@6B@        0042d8b8     kibokern:kibokern.obj
 0002:000078cc       ??_R3CKiboKern@@8          0042d8cc     kibokern:kibokern.obj
 0002:000078dc       ??_R2CKiboKern@@8          0042d8dc     kibokern:kibokern.obj
 0002:000078e4       ??_R1A@?0A@EA@CKiboKern@@8 0042d8e4     kibokern:kibokern.obj
 0002:00007900       ??_R4type_info@@6B@        0042d900     msvcrt:ti_inst.obj
 0002:00007914       ??_R3type_info@@8          0042d914     msvcrt:ti_inst.obj
 0002:00007924       ??_R2type_info@@8          0042d924     msvcrt:ti_inst.obj
 0002:0000792c       ??_R1A@?0A@EA@type_info@@8 0042d92c     msvcrt:ti_inst.obj
 0002:00007950       ___safe_se_handler_table   0042d950     <linker-defined>
 0002:00007b10       ___rtc_iaa                 0042db10     msvcrt:_initsect_.obj
 0002:00007b14       ___rtc_izz                 0042db14     msvcrt:_initsect_.obj
 0002:00007b18       ___rtc_taa                 0042db18     msvcrt:_initsect_.obj
 0002:00007b1c       ___rtc_tzz                 0042db1c     msvcrt:_initsect_.obj
 0002:00009c54       __TI1?AV_com_error@@       0042fc54     comsuppw:comraise.obj
 0002:00009c64       __CTA1?AV_com_error@@      0042fc64     comsuppw:comraise.obj
 0002:00009c6c       __CT??_R0?AV_com_error@@@8??0_com_error@@QAE@ABV0@@Z16 0042fc6c     comsuppw:comraise.obj
 0002:00009c88       __DELAY_IMPORT_DESCRIPTOR_dwmapi_dll 0042fc88     dwmapi:dwmapi.dll
 0002:00009ca8       __NULL_DELAY_IMPORT_DESCRIPTOR 0042fca8     dwmapi:dwmapi.dll
 0002:00009ccc       \177dwmapi_NULL_THUNK_DATA_DLN 0042fccc     dwmapi:dwmapi.dll
 0002:00009cd4       \177dwmapi_NULL_THUNK_DATA_DLB 0042fcd4     dwmapi:dwmapi.dll
 0002:00009cd8       __IMPORT_DESCRIPTOR_windisk 0042fcd8     windisk:windisk.dll
 0002:00009cec       __IMPORT_DESCRIPTOR_diskop 0042fcec     diskop:diskop.dll
 0002:00009d00       __IMPORT_DESCRIPTOR_SAMIO  0042fd00     samio:SAMIO.dll
 0002:00009d14       __IMPORT_DESCRIPTOR_SPIFilter 0042fd14     SPIFilter:SPIFilter.dll
 0002:00009d28       __IMPORT_DESCRIPTOR_mfc90  0042fd28     mfc90:mfc90.dll
 0002:00009d3c       __IMPORT_DESCRIPTOR_MSVCR90 0042fd3c     msvcrt:MSVCR90.dll
 0002:00009d50       __IMPORT_DESCRIPTOR_KERNEL32 0042fd50     kernel32:KERNEL32.dll
 0002:00009d64       __IMPORT_DESCRIPTOR_USER32 0042fd64     user32:USER32.dll
 0002:00009d78       __IMPORT_DESCRIPTOR_ADVAPI32 0042fd78     advapi32:ADVAPI32.dll
 0002:00009d8c       __IMPORT_DESCRIPTOR_SHELL32 0042fd8c     shell32:SHELL32.dll
 0002:00009da0       __IMPORT_DESCRIPTOR_COMCTL32 0042fda0     comctl32:COMCTL32.dll
 0002:00009db4       __IMPORT_DESCRIPTOR_ole32  0042fdb4     ole32:ole32.dll
 0002:00009dc8       __IMPORT_DESCRIPTOR_OLEAUT32 0042fdc8     oleaut32:OLEAUT32.dll
 0002:00009ddc       __IMPORT_DESCRIPTOR_WS2_32 0042fddc     WS2_32:WS2_32.dll
 0002:00009df0       __IMPORT_DESCRIPTOR_VERSION 0042fdf0     Version:VERSION.dll
 0002:00009e04       __IMPORT_DESCRIPTOR_WININET 0042fe04     wininet:WININET.dll
 0002:00009e18       __IMPORT_DESCRIPTOR_UsbControl 0042fe18     UsbControl:UsbControl.dll
 0002:00009e2c       __IMPORT_DESCRIPTOR_SendMessage 0042fe2c     SendMessage:SendMessage.dll
 0002:00009e40       __IMPORT_DESCRIPTOR_LockScreen 0042fe40     LockScreen:LockScreen.dll
 0002:00009e54       __IMPORT_DESCRIPTOR_WTSAPI32 0042fe54     Wtsapi32:WTSAPI32.dll
 0002:00009e68       __IMPORT_DESCRIPTOR_Hook   0042fe68     hook:Hook.dll
 0002:00009e7c       __IMPORT_DESCRIPTOR_HTSAPI 0042fe7c     htsapi:HTSAPI.dll
 0002:00009e90       __IMPORT_DESCRIPTOR_IPHLPAPI 0042fe90     Iphlpapi:IPHLPAPI.DLL
 0002:00009ea4       __NULL_IMPORT_DESCRIPTOR   0042fea4     windisk:windisk.dll
 0003:00000000       ??_R0?AVCBootModuleManager@@@8 00432000     BootModuleManager.obj
 0003:00000024       ??_R0?AV?$CTypedPtrList@VCPtrList@@PAK@@@8 00432024     BootModuleManager.obj
 0003:00000054       ??_R0?AV?$_CTypedPtrList@VCPtrList@@PAK@@@8 00432054     BootModuleManager.obj
 0003:00000084       ??_R0?AVCPtrList@@@8       00432084     BootModuleManager.obj
 0003:0000009c       ??_R0?AVCObject@@@8        0043209c     BootModuleManager.obj
 0003:000000b4       ??_R0?AVCCriticalSection@@@8 004320b4     BootModuleManager.obj
 0003:000000d4       ??_R0?AVCSyncObject@@@8    004320d4     BootModuleManager.obj
 0003:000000f0       ??_R0?AVCErrorMessage@@@8  004320f0     ChatDlg.obj
 0003:0000010c       ??_R0?AVCErrorTable@@@8    0043210c     ChatDlg.obj
 0003:00000128       ??_R0?AVCInstall@@@8       00432128     ChatDlg.obj
 0003:00000140       ??_R0?AVCChatDlg@@@8       00432140     ChatDlg.obj
 0003:00000158       ??_R0?AVCDialog@@@8        00432158     ChatDlg.obj
 0003:00000170       ??_R0?AVCWnd@@@8           00432170     ChatDlg.obj
 0003:00000184       ??_R0?AVCCmdTarget@@@8     00432184     ChatDlg.obj
 0003:000001a0       ??_R0?AVCStatic@@@8        004321a0     ChatDlg.obj
 0003:000001b8       ??_R0?AVCCheckPasswordDlg@@@8 004321b8     CheckPasswordDlg.obj
 0003:000001d8       ??_R0?AVCEdit@@@8          004321d8     CheckPasswordDlg.obj
 0003:000001ec       ??_R0?AVCDialogInputname@@@8 004321ec     DialogInputname.obj
 0003:0000020c       ??_R0?AVCFtpClientDlg@@@8  0043220c     FtpClientDlg.obj
 0003:00000228       ??_R0?AVCWinThread@@@8     00432228     FtpClientDlg.obj
 0003:00000244       ??_R0PAVCInternetException@@@8 00432244     FtpClientDlg.obj
 0003:00000268       ?gbtime@@3PADA             00432268     KiboClient.obj
 0003:0000027c       ?Version@@3PADA            0043227c     KiboClient.obj
 0003:00000290       ??_R0?AVCKiboClientApp@@@8 00432290     KiboClient.obj
 0003:000002b0       ??_R0?AVCWinAppEx@@@8      004322b0     KiboClient.obj
 0003:000002c8       ??_R0?AVCWinApp@@@8        004322c8     KiboClient.obj
 0003:000002e0       ??_R0?AVCAboutDlg@@@8      004322e0     KiboClient.obj
 0003:000002f8       ?g_bFirstSendhd@@3HA       004322f8     MainFrm.obj
 0003:00000508       ??_R0?AVCMainFrame@@@8     00432508     MainFrm.obj
 0003:00000524       ??_R0?AVCFrameWndEx@@@8    00432524     MainFrm.obj
 0003:00000540       ??_R0?AVCFrameWnd@@@8      00432540     MainFrm.obj
 0003:00000558       ??_R0?AV?$CTypedPtrList@VCPtrList@@PAUtagRECVREQUEST@@@@@8 00432558     MainFrm.obj
 0003:00000598       ??_R0?AV?$_CTypedPtrList@VCPtrList@@PAUtagRECVREQUEST@@@@@8 00432598     MainFrm.obj
 0003:000005d8       ??_R0?AVCMenu@@@8          004325d8     MainFrm.obj
 0003:000005ec       ??_R0PAVCException@@@8     004325ec     MainFrm.obj
 0003:00000608       ??_R0?AVCMyRichEdit@@@8    00432608     MyRichEdit.obj
 0003:00000624       ??_R0?AVCRichEditCtrl@@@8  00432624     MyRichEdit.obj
 0003:00000640       ??_R0?AVCPortChannelDlg@@@8 00432640     PortChannelDlg.obj
 0003:00000660       ??_R0?AVCPropertyManager@@@8 00432660     PropertyManager.obj
 0003:00000680       ??_R0?AV?$CTypedPtrList@VCPtrList@@PAUtagPROPERTY_REQUEST@@@@@8 00432680     PropertyManager.obj
 0003:000006c8       ??_R0?AV?$_CTypedPtrList@VCPtrList@@PAUtagPROPERTY_REQUEST@@@@@8 004326c8     PropertyManager.obj
 0003:0000070c       ??_R0?AVCSetDrfaultNICDlg@@@8 0043270c     SetDrfaultNICDlg.obj
 0003:0000072c       ??_R0?AVCComboBox@@@8      0043272c     SetDrfaultNICDlg.obj
 0003:00000748       ??_R0?AV?$_CTypedPtrList@VCPtrList@@PAUtagUDPRECV@@@@@8 00432748     commod2:MulticastSocket.obj
 0003:00000784       ??_R0?AV?$CTypedPtrList@VCPtrList@@PAUtagUDPRECV@@@@@8 00432784     commod2:MulticastSocket.obj
 0003:000007c0       ??_R0?AVCMulticastSocket@@@8 004327c0     commod2:MulticastSocket.obj
 0003:000007e0       ?encrypt_key@@3PADA        004327e0     kibokern:kibokern.obj
 0003:000007f0       ??_R0?AV?$_CTypedPtrList@VCPtrList@@PAUSTRUCT_PROTECTITEM@@@@@8 004327f0     kibokern:kibokern.obj
 0003:00000838       ??_R0?AV?$CTypedPtrList@VCPtrList@@PAUSTRUCT_PROTECTITEM@@@@@8 00432838     kibokern:kibokern.obj
 0003:0000087c       ??_R0?AVCKiboKern@@@8      0043287c     kibokern:kibokern.obj
 0003:00000894       ___security_cookie         00432894     msvcrt:gs_cookie.obj
 0003:00000898       ___security_cookie_complement 00432898     msvcrt:gs_cookie.obj
 0003:0000089c       ??_R0?AVtype_info@@@8      0043289c     msvcrt:ti_inst.obj
 0003:000008c0       ___native_dllmain_reason   004328c0     msvcrt:natstart.obj
 0003:000008c4       ___native_vcclrit_reason   004328c4     msvcrt:natstart.obj
 0003:000008c8       ___globallocalestatus      004328c8     msvcrt:xthdloc.obj
 0003:000008cc       ___defaultmatherr          004328cc     msvcrt:merr.obj
 0003:000008d0       ?__errorPfn@@3P6GXJPAUIErrorInfo@@@ZA 004328d0     comsuppw:comsupp.obj
 0003:000008d8       ?vtMissing@@3V_variant_t@@A 004328d8     comsuppw:comutil.obj
 0003:000008e8       ??_R0?AV_com_error@@@8     004328e8     comsuppw:comraise.obj
 0003:00000910       __imp__DwmEnableComposition@4 00432910     dwmapi:dwmapi.dll
 0003:00000914       \177dwmapi_NULL_THUNK_DATA_DLA 00432914     dwmapi:dwmapi.dll
 0003:00000918       ?lpTranslate@@3PAULANGANDCODEPAGE@@A 00432918     CommonFunc.obj
 0003:0000091c       ?istip@@3HA                0043291c     CommonFunc.obj
 0003:00000920       ?ftpdlg@@3PAVCFtpClientDlg@@A 00432920     FtpClientDlg.obj
 0003:00000924       ?nPort@@3HA                00432924     FtpClientDlg.obj
 0003:00000928       ?szLocDirectory@@3PADA     00432928     FtpClientDlg.obj
 0003:00000a2c       ?szFtpPassword@@3PADA      00432a2c     FtpClientDlg.obj
 0003:00000a40       ?szFtpDirectory@@3PADA     00432a40     FtpClientDlg.obj
 0003:00000b44       ?szFtpUser@@3PADA          00432b44     FtpClientDlg.obj
 0003:00000b58       ?szFtpName@@3PADA          00432b58     FtpClientDlg.obj
 0003:00000c58       ?szAppName@@3PADA          00432c58     FtpClientDlg.obj
 0003:00000d58       ?bFtpOver@@3HA             00432d58     FtpClientDlg.obj
 0003:00000d5c       ?bUpFilename@@3V?$CStringT@DV?$StrTraitMFC_DLL@DV?$ChTraitsCRT@D@ATL@@@@@ATL@@A 00432d5c     FtpClientDlg.obj
 0003:00000d60       ?g_MemorySize@@3PADA       00432d60     KiboClient.obj
 0003:00000d74       ?gVersion@@3V?$CStringT@DV?$StrTraitMFC_DLL@DV?$ChTraitsCRT@D@ATL@@@@@ATL@@A 00432d74     KiboClient.obj
 0003:00000d78       ?m_bootMgr@@3VCBootModuleManager@@A 00432d78     KiboClient.obj
 0003:00001fe8       ?theApp@@3VCKiboClientApp@@A 00433fe8     KiboClient.obj
 0003:000020d8       ?g_pMainFrame@@3PAVCMainFrame@@A 004340d8     MainFrm.obj
 0003:000020dc       ?istipinfo@@3HA            004340dc     MainFrm.obj
 0003:000020e0       ?g_havedlg@@3HA            004340e0     MainFrm.obj
 0003:000020e4       ?bRegFinish@@3HA           004340e4     MainFrm.obj
 0003:000020e8       ?g_bIsLockMsg@@3HA         004340e8     MainFrm.obj
 0003:000020ec       ?g_bIsChatting@@3HA        004340ec     MainFrm.obj
 0003:000020f4       ?m_szMsgList@@3VCStringList@@A 004340f4     MainFrm.obj
 0003:00002110       ?g_sock@@3VCMulticastSocket@@A 00434110     MainFrm.obj
 0003:00002170       ?g_mydisk@@3VCDiskIO@@A    00434170     MainFrm.obj
 0003:00002428       ?g_mykern@@3VCKiboKern@@A  00434428     MainFrm.obj
 0003:00003058       ?g_osvi@@3U_OSVERSIONINFOA@@A 00435058     ProcessHide.obj
 0003:000030ec       ?ZwOpenSection@@3P6GJPAPAXKPAU_OBJECT_ATTRIBUTES@@@ZA 004350ec     ProcessHide.obj
 0003:000030f0       ?RtlInitUnicodeString@@3P6GXPAU_UNICODE_STRING@@PB_W@ZA 004350f0     ProcessHide.obj
 0003:000030f4       ?g_hNtDLL@@3PAUHINSTANCE__@@A 004350f4     ProcessHide.obj
 0003:000030f8       ?g_pMapPhysicalMemory@@3PAXA 004350f8     ProcessHide.obj
 0003:000030fc       ?g_hMPM@@3PAXA             004350fc     ProcessHide.obj
 0003:00003100       ?gIsVisa@@3HA              00435100     PropertyManager.obj
 0003:0000313c       ?NtQuerySystemInformation@@3P6GJIPAXKPAK@ZA 0043513c     comfunc:comfunc.obj
 0003:00003140       ?g_bIsNT@@3HA              00435140     comfunc:comfunc.obj
 0003:00003144       ?g_enabledbg@@3HA          00435144     comfunc:comfunc.obj
 0003:00003148       ?g_CurrentPath@@3V?$CStringT@DV?$StrTraitMFC_DLL@DV?$ChTraitsCRT@D@ATL@@@@@ATL@@A 00435148     comfunc:comfunc.obj
 0003:0000314c       ?g_tempstring@@3V?$CStringT@DV?$StrTraitMFC_DLL@DV?$ChTraitsCRT@D@ATL@@@@@ATL@@A 0043514c     loadres:exloadres.obj
 0003:00003150       ?g_BasicPath@@3V?$CStringT@DV?$StrTraitMFC_DLL@DV?$ChTraitsCRT@D@ATL@@@@@ATL@@A 00435150     loadres:exloadres.obj
 0003:00003154       __hmod__dwmapi_dll         00435154     dwmapi:dwmapi.dll
 0003:00003158       ___puiHead                 00435158     DelayImp:delayhlp.obj
 0003:0000315c       ___pfnDliFailureHook2      0043515c     DelayImp:delayhk1.obj
 0003:00003160       ___pfnDliNotifyHook2       00435160     DelayImp:delayhk2.obj
 0003:00003164       __afxForceEXCLUDE          00435164     mfcs90:nolib.obj
 0003:00003168       __afxForceSTDAFX           00435168     mfcs90:stdafx.obj
 0003:000034b4       __forceCRTManifestRTM      004354b4     msvcrt:crtmanifestrtm.obj
 0003:000034b8       __dowildcard               004354b8     msvcrt:wildcard.obj
 0003:000034bc       __newmode                  004354bc     msvcrt:_newmode.obj
 0003:000034c0       __commode                  004354c0     msvcrt:xncommod.obj
 0003:000034c4       __fmode                    004354c4     msvcrt:xtxtmode.obj
 0003:000034c8       ?_afxInitAppState@@3DA     004354c8     mfcs90:appmodul.obj
 0003:000034cc       __forceMFCManifestRTM      004354cc     mfcs90:mfcmanifestrtm.obj
 0003:000034d0       ___sse2_available          004354d0     <common>
 0003:000034d4       __adjust_fdiv              004354d4     <common>
 0003:000034d8       ___native_startup_state    004354d8     <common>
 0003:000034dc       ___native_startup_lock     004354dc     <common>
 0003:000034e0       ___dyn_tls_init_callback   004354e0     <common>
 0003:000034e4       ___onexitend               004354e4     <common>
 0003:000034e8       ___onexitbegin             004354e8     <common>

 entry point at        0001:00021527

 Static symbols

 0001:000075ee       __catch$?SendFileThread@CMyAppThread@@SAIPAX@Z$0 004085ee f   FtpClientDlg.obj
 0001:00018a5a       __catch$??1CWaitCursor@@QAE@XZ$0 00419a5a f i MainFrm.obj
 0001:0002121c       _pre_cpp_init              0042221c f   msvcrt:crtexew.obj
 0001:00021267       ___tmainCRTStartup         00422267 f   msvcrt:crtexew.obj
 0001:00021446       _pre_c_init                00422446 f   msvcrt:crtexew.obj
 0001:00021a3e       _has_osfxsr_set            00422a3e f   msvcrt:cpu_disp.obj
 0001:00021ea0       __unwindfunclet$??1CBootModuleManager@@UAE@XZ$0 00422ea0 f   BootModuleManager.obj
 0001:00021ea0       __unwindfunclet$??0CBootModuleManager@@QAE@XZ$0 00422ea0 f   BootModuleManager.obj
 0001:00021eab       __unwindfunclet$??0CBootModuleManager@@QAE@XZ$1 00422eab f   BootModuleManager.obj
 0001:00021eab       __unwindfunclet$??1CBootModuleManager@@UAE@XZ$1 00422eab f   BootModuleManager.obj
 0001:00021eb6       __unwindfunclet$??0CBootModuleManager@@QAE@XZ$2 00422eb6 f   BootModuleManager.obj
 0001:00021eb6       __unwindfunclet$??1CBootModuleManager@@UAE@XZ$2 00422eb6 f   BootModuleManager.obj
 0001:00021ec4       __ehhandler$??1CBootModuleManager@@UAE@XZ 00422ec4 f   BootModuleManager.obj
 0001:00021ec4       __ehhandler$??0CBootModuleManager@@QAE@XZ 00422ec4 f   BootModuleManager.obj
 0001:00021ee0       __unwindfunclet$??0CCriticalSection@@QAE@XZ$0 00422ee0 f   BootModuleManager.obj
 0001:00021ee8       __ehhandler$??0CCriticalSection@@QAE@XZ 00422ee8 f   BootModuleManager.obj
 0001:00021f10       __unwindfunclet$??0CChatDlg@@QAE@PAVCWnd@@@Z$0 00422f10 f   ChatDlg.obj
 0001:00021f10       __unwindfunclet$??1CChatDlg@@UAE@XZ$0 00422f10 f   ChatDlg.obj
 0001:00021f18       __unwindfunclet$??1CChatDlg@@UAE@XZ$1 00422f18 f   ChatDlg.obj
 0001:00021f18       __unwindfunclet$??0CChatDlg@@QAE@PAVCWnd@@@Z$1 00422f18 f   ChatDlg.obj
 0001:00021f27       __unwindfunclet$??1CChatDlg@@UAE@XZ$2 00422f27 f   ChatDlg.obj
 0001:00021f27       __unwindfunclet$??0CChatDlg@@QAE@PAVCWnd@@@Z$2 00422f27 f   ChatDlg.obj
 0001:00021f36       __unwindfunclet$??0CChatDlg@@QAE@PAVCWnd@@@Z$3 00422f36 f   ChatDlg.obj
 0001:00021f36       __unwindfunclet$??1CChatDlg@@UAE@XZ$3 00422f36 f   ChatDlg.obj
 0001:00021f44       __unwindfunclet$??1CChatDlg@@UAE@XZ$4 00422f44 f   ChatDlg.obj
 0001:00021f44       __unwindfunclet$??0CChatDlg@@QAE@PAVCWnd@@@Z$4 00422f44 f   ChatDlg.obj
 0001:00021f52       __ehhandler$??0CChatDlg@@QAE@PAVCWnd@@@Z 00422f52 f   ChatDlg.obj
 0001:00021f52       __ehhandler$??1CChatDlg@@UAE@XZ 00422f52 f   ChatDlg.obj
 0001:00021f70       __unwindfunclet$?OnSendButton@CChatDlg@@IAEXXZ$0 00422f70 f   ChatDlg.obj
 0001:00021f79       __unwindfunclet$?OnSendButton@CChatDlg@@IAEXXZ$1 00422f79 f   ChatDlg.obj
 0001:00021f82       __unwindfunclet$?OnSendButton@CChatDlg@@IAEXXZ$2 00422f82 f   ChatDlg.obj
 0001:00021f8b       __unwindfunclet$?OnSendButton@CChatDlg@@IAEXXZ$3 00422f8b f   ChatDlg.obj
 0001:00021f94       __unwindfunclet$?OnSendButton@CChatDlg@@IAEXXZ$4 00422f94 f   ChatDlg.obj
 0001:00021f9d       __unwindfunclet$?OnSendButton@CChatDlg@@IAEXXZ$5 00422f9d f   ChatDlg.obj
 0001:00021fa6       __unwindfunclet$?OnSendButton@CChatDlg@@IAEXXZ$6 00422fa6 f   ChatDlg.obj
 0001:00021faf       __unwindfunclet$?OnSendButton@CChatDlg@@IAEXXZ$7 00422faf f   ChatDlg.obj
 0001:00021fb8       __unwindfunclet$?OnSendButton@CChatDlg@@IAEXXZ$8 00422fb8 f   ChatDlg.obj
 0001:00021fc4       __unwindfunclet$?OnSendButton@CChatDlg@@IAEXXZ$9 00422fc4 f   ChatDlg.obj
 0001:00021fd0       __unwindfunclet$?OnSendButton@CChatDlg@@IAEXXZ$11 00422fd0 f   ChatDlg.obj
 0001:00021fdc       __ehhandler$?OnSendButton@CChatDlg@@IAEXXZ 00422fdc f   ChatDlg.obj
 0001:00022010       __unwindfunclet$?OnInitDialog@CChatDlg@@MAEHXZ$0 00423010 f   ChatDlg.obj
 0001:0002201c       __unwindfunclet$?OnInitDialog@CChatDlg@@MAEHXZ$1 0042301c f   ChatDlg.obj
 0001:00022028       __unwindfunclet$?OnInitDialog@CChatDlg@@MAEHXZ$2 00423028 f   ChatDlg.obj
 0001:00022034       __unwindfunclet$?OnInitDialog@CChatDlg@@MAEHXZ$3 00423034 f   ChatDlg.obj
 0001:00022040       __unwindfunclet$?OnInitDialog@CChatDlg@@MAEHXZ$4 00423040 f   ChatDlg.obj
 0001:0002204c       __unwindfunclet$?OnInitDialog@CChatDlg@@MAEHXZ$5 0042304c f   ChatDlg.obj
 0001:00022055       __unwindfunclet$?OnInitDialog@CChatDlg@@MAEHXZ$6 00423055 f   ChatDlg.obj
 0001:0002205e       __unwindfunclet$?OnInitDialog@CChatDlg@@MAEHXZ$7 0042305e f   ChatDlg.obj
 0001:00022067       __unwindfunclet$?OnInitDialog@CChatDlg@@MAEHXZ$9 00423067 f   ChatDlg.obj
 0001:00022073       __unwindfunclet$?OnInitDialog@CChatDlg@@MAEHXZ$10 00423073 f   ChatDlg.obj
 0001:0002207f       __unwindfunclet$?OnInitDialog@CChatDlg@@MAEHXZ$11 0042307f f   ChatDlg.obj
 0001:0002208b       __unwindfunclet$?OnInitDialog@CChatDlg@@MAEHXZ$12 0042308b f   ChatDlg.obj
 0001:00022097       __unwindfunclet$?OnInitDialog@CChatDlg@@MAEHXZ$13 00423097 f   ChatDlg.obj
 0001:000220a3       __unwindfunclet$?OnInitDialog@CChatDlg@@MAEHXZ$14 004230a3 f   ChatDlg.obj
 0001:000220af       __unwindfunclet$?OnInitDialog@CChatDlg@@MAEHXZ$15 004230af f   ChatDlg.obj
 0001:000220bb       __unwindfunclet$?OnInitDialog@CChatDlg@@MAEHXZ$16 004230bb f   ChatDlg.obj
 0001:000220c7       __unwindfunclet$?OnInitDialog@CChatDlg@@MAEHXZ$17 004230c7 f   ChatDlg.obj
 0001:000220d3       __unwindfunclet$?OnInitDialog@CChatDlg@@MAEHXZ$19 004230d3 f   ChatDlg.obj
 0001:000220df       __unwindfunclet$?OnInitDialog@CChatDlg@@MAEHXZ$20 004230df f   ChatDlg.obj
 0001:000220eb       __unwindfunclet$?OnInitDialog@CChatDlg@@MAEHXZ$21 004230eb f   ChatDlg.obj
 0001:000220f7       __unwindfunclet$?OnInitDialog@CChatDlg@@MAEHXZ$22 004230f7 f   ChatDlg.obj
 0001:00022103       __unwindfunclet$?OnInitDialog@CChatDlg@@MAEHXZ$23 00423103 f   ChatDlg.obj
 0001:0002210f       __unwindfunclet$?OnInitDialog@CChatDlg@@MAEHXZ$24 0042310f f   ChatDlg.obj
 0001:0002211b       __ehhandler$?OnInitDialog@CChatDlg@@MAEHXZ 0042311b f   ChatDlg.obj
 0001:00022150       __unwindfunclet$?OnCommand@CChatDlg@@MAEHIJ@Z$1 00423150 f   ChatDlg.obj
 0001:00022159       __unwindfunclet$?OnCommand@CChatDlg@@MAEHIJ@Z$2 00423159 f   ChatDlg.obj
 0001:00022162       __unwindfunclet$?OnCommand@CChatDlg@@MAEHIJ@Z$3 00423162 f   ChatDlg.obj
 0001:0002216b       __unwindfunclet$?OnCommand@CChatDlg@@MAEHIJ@Z$4 0042316b f   ChatDlg.obj
 0001:00022174       __unwindfunclet$?OnCommand@CChatDlg@@MAEHIJ@Z$5 00423174 f   ChatDlg.obj
 0001:0002217d       __unwindfunclet$?OnCommand@CChatDlg@@MAEHIJ@Z$6 0042317d f   ChatDlg.obj
 0001:00022186       __unwindfunclet$?OnCommand@CChatDlg@@MAEHIJ@Z$7 00423186 f   ChatDlg.obj
 0001:0002218f       __unwindfunclet$?OnCommand@CChatDlg@@MAEHIJ@Z$8 0042318f f   ChatDlg.obj
 0001:00022198       __unwindfunclet$?OnCommand@CChatDlg@@MAEHIJ@Z$9 00423198 f   ChatDlg.obj
 0001:000221a1       __unwindfunclet$?OnCommand@CChatDlg@@MAEHIJ@Z$10 004231a1 f   ChatDlg.obj
 0001:000221aa       __ehhandler$?OnCommand@CChatDlg@@MAEHIJ@Z 004231aa f   ChatDlg.obj
 0001:000221e0       __unwindfunclet$??0CCheckPasswordDlg@@QAE@PAVCWnd@@@Z$0 004231e0 f   CheckPasswordDlg.obj
 0001:000221e8       __unwindfunclet$??0CCheckPasswordDlg@@QAE@PAVCWnd@@@Z$1 004231e8 f   CheckPasswordDlg.obj
 0001:000221f3       __unwindfunclet$??0CCheckPasswordDlg@@QAE@PAVCWnd@@@Z$2 004231f3 f   CheckPasswordDlg.obj
 0001:00022202       __unwindfunclet$??0CCheckPasswordDlg@@QAE@PAVCWnd@@@Z$3 00423202 f   CheckPasswordDlg.obj
 0001:00022211       __ehhandler$??0CCheckPasswordDlg@@QAE@PAVCWnd@@@Z 00423211 f   CheckPasswordDlg.obj
 0001:00022230       __unwindfunclet$??HATL@@YA?AV?$CStringT@DV?$StrTraitMFC_DLL@DV?$ChTraitsCRT@D@ATL@@@@@0@ABV10@PBD@Z$0 00423230 f   CheckPasswordDlg.obj
 0001:00022230       __unwindfunclet$?OnOK@CCheckPasswordDlg@@MAEXXZ$0 00423230 f   CheckPasswordDlg.obj
 0001:00022230       __unwindfunclet$??HATL@@YA?AV?$CStringT@DV?$StrTraitMFC_DLL@DV?$ChTraitsCRT@D@ATL@@@@@0@ABV10@0@Z$0 00423230 f   CheckPasswordDlg.obj
 0001:00022230       __unwindfunclet$??HATL@@YA?AV?$CStringT@DV?$StrTraitMFC_DLL@DV?$ChTraitsCRT@D@ATL@@@@@0@PBDABV10@@Z$0 00423230 f   CheckPasswordDlg.obj
 0001:00022239       __ehhandler$?OnOK@CCheckPasswordDlg@@MAEXXZ 00423239 f   CheckPasswordDlg.obj
 0001:00022239       __ehhandler$??HATL@@YA?AV?$CStringT@DV?$StrTraitMFC_DLL@DV?$ChTraitsCRT@D@ATL@@@@@0@ABV10@0@Z 00423239 f   CheckPasswordDlg.obj
 0001:00022239       __ehhandler$??HATL@@YA?AV?$CStringT@DV?$StrTraitMFC_DLL@DV?$ChTraitsCRT@D@ATL@@@@@0@PBDABV10@@Z 00423239 f   CheckPasswordDlg.obj
 0001:00022239       __ehhandler$??HATL@@YA?AV?$CStringT@DV?$StrTraitMFC_DLL@DV?$ChTraitsCRT@D@ATL@@@@@0@ABV10@PBD@Z 00423239 f   CheckPasswordDlg.obj
 0001:00022260       __unwindfunclet$?IsPhysicalLocalMac@@YAHABV?$CStringT@DV?$StrTraitMFC_DLL@DV?$ChTraitsCRT@D@ATL@@@@@ATL@@@Z$0 00423260 f   CommonFunc.obj
 0001:0002226c       __unwindfunclet$?IsPhysicalLocalMac@@YAHABV?$CStringT@DV?$StrTraitMFC_DLL@DV?$ChTraitsCRT@D@ATL@@@@@ATL@@@Z$1 0042326c f   CommonFunc.obj
 0001:00022278       __ehhandler$?IsPhysicalLocalMac@@YAHABV?$CStringT@DV?$StrTraitMFC_DLL@DV?$ChTraitsCRT@D@ATL@@@@@ATL@@@Z 00423278 f   CommonFunc.obj
 0001:000222a0       __unwindfunclet$?GetLocalComputerInfo@@YAHPAD0@Z$0 004232a0 f   CommonFunc.obj
 0001:000222a9       __unwindfunclet$?GetLocalComputerInfo@@YAHPAD0@Z$1 004232a9 f   CommonFunc.obj
 0001:000222b5       __unwindfunclet$?GetLocalComputerInfo@@YAHPAD0@Z$2 004232b5 f   CommonFunc.obj
 0001:000222c0       __unwindfunclet$?GetLocalComputerInfo@@YAHPAD0@Z$4 004232c0 f   CommonFunc.obj
 0001:000222cc       __unwindfunclet$?GetLocalComputerInfo@@YAHPAD0@Z$5 004232cc f   CommonFunc.obj
 0001:000222d8       __unwindfunclet$?GetLocalComputerInfo@@YAHPAD0@Z$7 004232d8 f   CommonFunc.obj
 0001:000222e4       __unwindfunclet$?GetLocalComputerInfo@@YAHPAD0@Z$8 004232e4 f   CommonFunc.obj
 0001:000222ef       __unwindfunclet$?GetLocalComputerInfo@@YAHPAD0@Z$10 004232ef f   CommonFunc.obj
 0001:000222fb       __unwindfunclet$?GetLocalComputerInfo@@YAHPAD0@Z$12 004232fb f   CommonFunc.obj
 0001:00022307       __unwindfunclet$?GetLocalComputerInfo@@YAHPAD0@Z$13 00423307 f   CommonFunc.obj
 0001:00022312       __unwindfunclet$?GetLocalComputerInfo@@YAHPAD0@Z$15 00423312 f   CommonFunc.obj
 0001:0002231e       __unwindfunclet$?GetLocalComputerInfo@@YAHPAD0@Z$16 0042331e f   CommonFunc.obj
 0001:0002232a       __ehhandler$?GetLocalComputerInfo@@YAHPAD0@Z 0042332a f   CommonFunc.obj
 0001:00022360       __unwindfunclet$?NICLinknumber@@YAHXZ$0 00423360 f   CommonFunc.obj
 0001:00022369       __unwindfunclet$?NICLinknumber@@YAHXZ$1 00423369 f   CommonFunc.obj
 0001:00022375       __ehhandler$?NICLinknumber@@YAHXZ 00423375 f   CommonFunc.obj
 0001:000223a0       __unwindfunclet$?ReadParttionPara@@YAHAAUPartion_para_sector_s@@@Z$0 004233a0 f   CommonFunc.obj
 0001:000223ab       __ehhandler$?ReadParttionPara@@YAHAAUPartion_para_sector_s@@@Z 004233ab f   CommonFunc.obj
 0001:000223e0       __unwindfunclet$?WriteParttionPara@@YAHUPartion_para_sector_s@@H@Z$0 004233e0 f   CommonFunc.obj
 0001:000223eb       __ehhandler$?WriteParttionPara@@YAHUPartion_para_sector_s@@H@Z 004233eb f   CommonFunc.obj
 0001:00022420       __unwindfunclet$?GetfileVersion@@YAHV?$CStringT@DV?$StrTraitMFC_DLL@DV?$ChTraitsCRT@D@ATL@@@@@ATL@@AAV12@@Z$0 00423420 f   CommonFunc.obj
 0001:00022429       __unwindfunclet$?GetfileVersion@@YAHV?$CStringT@DV?$StrTraitMFC_DLL@DV?$ChTraitsCRT@D@ATL@@@@@ATL@@AAV12@@Z$1 00423429 f   CommonFunc.obj
 0001:00022432       __ehhandler$?GetfileVersion@@YAHV?$CStringT@DV?$StrTraitMFC_DLL@DV?$ChTraitsCRT@D@ATL@@@@@ATL@@AAV12@@Z 00423432 f   CommonFunc.obj
 0001:00022450       __unwindfunclet$??0CDialogInputname@@QAE@PAVCWnd@@@Z$0 00423450 f   DialogInputname.obj
 0001:00022450       __unwindfunclet$??1CDialogInputname@@UAE@XZ$0 00423450 f   DialogInputname.obj
 0001:00022458       __unwindfunclet$??1CDialogInputname@@UAE@XZ$1 00423458 f   DialogInputname.obj
 0001:00022458       __unwindfunclet$??0CDialogInputname@@QAE@PAVCWnd@@@Z$1 00423458 f   DialogInputname.obj
 0001:00022464       __unwindfunclet$??1CDialogInputname@@UAE@XZ$2 00423464 f   DialogInputname.obj
 0001:00022464       __unwindfunclet$??0CDialogInputname@@QAE@PAVCWnd@@@Z$2 00423464 f   DialogInputname.obj
 0001:00022470       __ehhandler$??0CDialogInputname@@QAE@PAVCWnd@@@Z 00423470 f   DialogInputname.obj
 0001:00022470       __ehhandler$??1CDialogInputname@@UAE@XZ 00423470 f   DialogInputname.obj
 0001:00022490       __unwindfunclet$?OnInitDialog@CDialogInputname@@MAEHXZ$0 00423490 f   DialogInputname.obj
 0001:00022499       __unwindfunclet$?OnInitDialog@CDialogInputname@@MAEHXZ$1 00423499 f   DialogInputname.obj
 0001:000224a2       __unwindfunclet$?OnInitDialog@CDialogInputname@@MAEHXZ$2 004234a2 f   DialogInputname.obj
 0001:000224ab       __unwindfunclet$?OnInitDialog@CDialogInputname@@MAEHXZ$3 004234ab f   DialogInputname.obj
 0001:000224b4       __ehhandler$?OnInitDialog@CDialogInputname@@MAEHXZ 004234b4 f   DialogInputname.obj
 0001:000224d0       __unwindfunclet$?OnBnClickedOk@CDialogInputname@@QAEXXZ$0 004234d0 f   DialogInputname.obj
 0001:000224d9       __unwindfunclet$?OnBnClickedOk@CDialogInputname@@QAEXXZ$1 004234d9 f   DialogInputname.obj
 0001:000224e2       __unwindfunclet$?OnBnClickedOk@CDialogInputname@@QAEXXZ$3 004234e2 f   DialogInputname.obj
 0001:000224eb       __unwindfunclet$?OnBnClickedOk@CDialogInputname@@QAEXXZ$4 004234eb f   DialogInputname.obj
 0001:000224f4       __unwindfunclet$?OnBnClickedOk@CDialogInputname@@QAEXXZ$5 004234f4 f   DialogInputname.obj
 0001:000224fd       __unwindfunclet$?OnBnClickedOk@CDialogInputname@@QAEXXZ$6 004234fd f   DialogInputname.obj
 0001:00022506       __unwindfunclet$?OnBnClickedOk@CDialogInputname@@QAEXXZ$7 00423506 f   DialogInputname.obj
 0001:0002250f       __unwindfunclet$?OnBnClickedOk@CDialogInputname@@QAEXXZ$8 0042350f f   DialogInputname.obj
 0001:00022518       __unwindfunclet$?OnBnClickedOk@CDialogInputname@@QAEXXZ$9 00423518 f   DialogInputname.obj
 0001:00022521       __unwindfunclet$?OnBnClickedOk@CDialogInputname@@QAEXXZ$10 00423521 f   DialogInputname.obj
 0001:0002252a       __ehhandler$?OnBnClickedOk@CDialogInputname@@QAEXXZ 0042352a f   DialogInputname.obj
 0001:00022550       __unwindfunclet$?IsCNOrEN@CDialogInputname@@QAE_NV?$CStringT@DV?$StrTraitMFC_DLL@DV?$ChTraitsCRT@D@ATL@@@@@ATL@@@Z$0 00423550 f   DialogInputname.obj
 0001:00022559       __unwindfunclet$?IsCNOrEN@CDialogInputname@@QAE_NV?$CStringT@DV?$StrTraitMFC_DLL@DV?$ChTraitsCRT@D@ATL@@@@@ATL@@@Z$1 00423559 f   DialogInputname.obj
 0001:00022562       __ehhandler$?IsCNOrEN@CDialogInputname@@QAE_NV?$CStringT@DV?$StrTraitMFC_DLL@DV?$ChTraitsCRT@D@ATL@@@@@ATL@@@Z 00423562 f   DialogInputname.obj
 0001:00022580       __unwindfunclet$??0CFtpClientDlg@@QAE@PAVCWnd@@@Z$0 00423580 f   FtpClientDlg.obj
 0001:00022588       __unwindfunclet$??0CFtpClientDlg@@QAE@PAVCWnd@@@Z$1 00423588 f   FtpClientDlg.obj
 0001:00022594       __unwindfunclet$??0CFtpClientDlg@@QAE@PAVCWnd@@@Z$2 00423594 f   FtpClientDlg.obj
 0001:000225a3       __ehhandler$??0CFtpClientDlg@@QAE@PAVCWnd@@@Z 004235a3 f   FtpClientDlg.obj
 0001:000225c0       __unwindfunclet$?GetFtpPara@CFtpClientDlg@@QAEXXZ$0 004235c0 f   FtpClientDlg.obj
 0001:000225c9       __ehhandler$?GetFtpPara@CFtpClientDlg@@QAEXXZ 004235c9 f   FtpClientDlg.obj
 0001:000225f0       __unwindfunclet$?OnConnect@CFtpClientDlg@@QAEHXZ$0 004235f0 f   FtpClientDlg.obj
 0001:000225f0       __unwindfunclet$?OnBnClickedCancel@CFtpClientDlg@@QAEXXZ$0 004235f0 f   FtpClientDlg.obj
 0001:000225f9       __unwindfunclet$?OnConnect@CFtpClientDlg@@QAEHXZ$1 004235f9 f   FtpClientDlg.obj
 0001:000225f9       __unwindfunclet$?OnBnClickedCancel@CFtpClientDlg@@QAEXXZ$1 004235f9 f   FtpClientDlg.obj
 0001:00022602       __ehhandler$?OnBnClickedCancel@CFtpClientDlg@@QAEXXZ 00423602 f   FtpClientDlg.obj
 0001:00022602       __ehhandler$?OnConnect@CFtpClientDlg@@QAEHXZ 00423602 f   FtpClientDlg.obj
 0001:00022620       __unwindfunclet$?OnBnClickedOk@CFtpClientDlg@@QAEXXZ$0 00423620 f   FtpClientDlg.obj
 0001:0002262c       __unwindfunclet$?OnBnClickedOk@CFtpClientDlg@@QAEXXZ$1 0042362c f   FtpClientDlg.obj
 0001:00022638       __unwindfunclet$?OnBnClickedOk@CFtpClientDlg@@QAEXXZ$2 00423638 f   FtpClientDlg.obj
 0001:00022644       __unwindfunclet$?OnBnClickedOk@CFtpClientDlg@@QAEXXZ$3 00423644 f   FtpClientDlg.obj
 0001:00022650       __unwindfunclet$?OnBnClickedOk@CFtpClientDlg@@QAEXXZ$4 00423650 f   FtpClientDlg.obj
 0001:00022658       __unwindfunclet$?OnBnClickedOk@CFtpClientDlg@@QAEXXZ$5 00423658 f   FtpClientDlg.obj
 0001:00022664       __unwindfunclet$?OnBnClickedOk@CFtpClientDlg@@QAEXXZ$6 00423664 f   FtpClientDlg.obj
 0001:00022670       __unwindfunclet$?OnBnClickedOk@CFtpClientDlg@@QAEXXZ$8 00423670 f   FtpClientDlg.obj
 0001:0002267c       __unwindfunclet$?OnBnClickedOk@CFtpClientDlg@@QAEXXZ$9 0042367c f   FtpClientDlg.obj
 0001:00022687       __unwindfunclet$?OnBnClickedOk@CFtpClientDlg@@QAEXXZ$10 00423687 f   FtpClientDlg.obj
 0001:00022693       __ehhandler$?OnBnClickedOk@CFtpClientDlg@@QAEXXZ 00423693 f   FtpClientDlg.obj
 0001:000226c0       __unwindfunclet$?FindServFileThread@CMyAppThread@@SAIPAX@Z$0 004236c0 f   FtpClientDlg.obj
 0001:000226c9       __unwindfunclet$?FindServFileThread@CMyAppThread@@SAIPAX@Z$1 004236c9 f   FtpClientDlg.obj
 0001:000226d2       __unwindfunclet$?FindServFileThread@CMyAppThread@@SAIPAX@Z$2 004236d2 f   FtpClientDlg.obj
 0001:000226db       __unwindfunclet$?FindServFileThread@CMyAppThread@@SAIPAX@Z$3 004236db f   FtpClientDlg.obj
 0001:000226e4       __unwindfunclet$?FindServFileThread@CMyAppThread@@SAIPAX@Z$4 004236e4 f   FtpClientDlg.obj
 0001:000226ed       __unwindfunclet$?FindServFileThread@CMyAppThread@@SAIPAX@Z$5 004236ed f   FtpClientDlg.obj
 0001:000226f6       __unwindfunclet$?FindServFileThread@CMyAppThread@@SAIPAX@Z$6 004236f6 f   FtpClientDlg.obj
 0001:000226ff       __unwindfunclet$?FindServFileThread@CMyAppThread@@SAIPAX@Z$7 004236ff f   FtpClientDlg.obj
 0001:00022708       __ehhandler$?FindServFileThread@CMyAppThread@@SAIPAX@Z 00423708 f   FtpClientDlg.obj
 0001:00022730       __unwindfunclet$?SendFileThread@CMyAppThread@@SAIPAX@Z$2 00423730 f   FtpClientDlg.obj
 0001:00022739       __unwindfunclet$?SendFileThread@CMyAppThread@@SAIPAX@Z$3 00423739 f   FtpClientDlg.obj
 0001:00022742       __unwindfunclet$?SendFileThread@CMyAppThread@@SAIPAX@Z$4 00423742 f   FtpClientDlg.obj
 0001:0002274b       __unwindfunclet$?SendFileThread@CMyAppThread@@SAIPAX@Z$5 0042374b f   FtpClientDlg.obj
 0001:00022754       __unwindfunclet$?SendFileThread@CMyAppThread@@SAIPAX@Z$6 00423754 f   FtpClientDlg.obj
 0001:0002275d       __unwindfunclet$?SendFileThread@CMyAppThread@@SAIPAX@Z$7 0042375d f   FtpClientDlg.obj
 0001:00022766       __unwindfunclet$?SendFileThread@CMyAppThread@@SAIPAX@Z$8 00423766 f   FtpClientDlg.obj
 0001:00022770       __unwindfunclet$?SendFileThread@CMyAppThread@@SAIPAX@Z$9 00423770 f   FtpClientDlg.obj
 0001:00022778       __unwindfunclet$?SendFileThread@CMyAppThread@@SAIPAX@Z$10 00423778 f   FtpClientDlg.obj
 0001:00022781       __unwindfunclet$?SendFileThread@CMyAppThread@@SAIPAX@Z$11 00423781 f   FtpClientDlg.obj
 0001:0002278d       __unwindfunclet$?SendFileThread@CMyAppThread@@SAIPAX@Z$12 0042378d f   FtpClientDlg.obj
 0001:00022799       __unwindfunclet$?SendFileThread@CMyAppThread@@SAIPAX@Z$13 00423799 f   FtpClientDlg.obj
 0001:000227a5       __unwindfunclet$?SendFileThread@CMyAppThread@@SAIPAX@Z$14 004237a5 f   FtpClientDlg.obj
 0001:000227b1       __unwindfunclet$?SendFileThread@CMyAppThread@@SAIPAX@Z$16 004237b1 f   FtpClientDlg.obj
 0001:000227ba       __unwindfunclet$?SendFileThread@CMyAppThread@@SAIPAX@Z$17 004237ba f   FtpClientDlg.obj
 0001:000227c6       __unwindfunclet$?SendFileThread@CMyAppThread@@SAIPAX@Z$18 004237c6 f   FtpClientDlg.obj
 0001:000227cf       __unwindfunclet$?SendFileThread@CMyAppThread@@SAIPAX@Z$19 004237cf f   FtpClientDlg.obj
 0001:000227db       __unwindfunclet$?SendFileThread@CMyAppThread@@SAIPAX@Z$21 004237db f   FtpClientDlg.obj
 0001:000227e7       __unwindfunclet$?SendFileThread@CMyAppThread@@SAIPAX@Z$22 004237e7 f   FtpClientDlg.obj
 0001:000227f3       __unwindfunclet$?SendFileThread@CMyAppThread@@SAIPAX@Z$23 004237f3 f   FtpClientDlg.obj
 0001:000227ff       __ehhandler$?SendFileThread@CMyAppThread@@SAIPAX@Z 004237ff f   FtpClientDlg.obj
 0001:00022820       __unwindfunclet$?OnBnClickedBrowse@CFtpClientDlg@@QAEXXZ$0 00423820 f   FtpClientDlg.obj
 0001:0002282c       __unwindfunclet$?OnBnClickedBrowse@CFtpClientDlg@@QAEXXZ$1 0042382c f   FtpClientDlg.obj
 0001:00022838       __unwindfunclet$?OnBnClickedBrowse@CFtpClientDlg@@QAEXXZ$2 00423838 f   FtpClientDlg.obj
 0001:00022843       __unwindfunclet$?OnBnClickedBrowse@CFtpClientDlg@@QAEXXZ$3 00423843 f   FtpClientDlg.obj
 0001:0002284f       __unwindfunclet$?OnBnClickedBrowse@CFtpClientDlg@@QAEXXZ$4 0042384f f   FtpClientDlg.obj
 0001:0002285b       __unwindfunclet$?OnBnClickedBrowse@CFtpClientDlg@@QAEXXZ$5 0042385b f   FtpClientDlg.obj
 0001:00022867       __ehhandler$?OnBnClickedBrowse@CFtpClientDlg@@QAEXXZ 00423867 f   FtpClientDlg.obj
 0001:00022890       __unwindfunclet$?OnFtp@CFtpClientDlg@@QAEJIJ@Z$0 00423890 f   FtpClientDlg.obj
 0001:00022899       __unwindfunclet$?OnFtp@CFtpClientDlg@@QAEJIJ@Z$1 00423899 f   FtpClientDlg.obj
 0001:000228a2       __unwindfunclet$?OnFtp@CFtpClientDlg@@QAEJIJ@Z$2 004238a2 f   FtpClientDlg.obj
 0001:000228ab       __unwindfunclet$?OnFtp@CFtpClientDlg@@QAEJIJ@Z$3 004238ab f   FtpClientDlg.obj
 0001:000228b4       __unwindfunclet$?OnFtp@CFtpClientDlg@@QAEJIJ@Z$4 004238b4 f   FtpClientDlg.obj
 0001:000228bd       __unwindfunclet$?OnFtp@CFtpClientDlg@@QAEJIJ@Z$5 004238bd f   FtpClientDlg.obj
 0001:000228c6       __unwindfunclet$?OnFtp@CFtpClientDlg@@QAEJIJ@Z$6 004238c6 f   FtpClientDlg.obj
 0001:000228cf       __unwindfunclet$?OnFtp@CFtpClientDlg@@QAEJIJ@Z$8 004238cf f   FtpClientDlg.obj
 0001:000228d8       __unwindfunclet$?OnFtp@CFtpClientDlg@@QAEJIJ@Z$9 004238d8 f   FtpClientDlg.obj
 0001:000228e1       __unwindfunclet$?OnFtp@CFtpClientDlg@@QAEJIJ@Z$10 004238e1 f   FtpClientDlg.obj
 0001:000228ea       __ehhandler$?OnFtp@CFtpClientDlg@@QAEJIJ@Z 004238ea f   FtpClientDlg.obj
 0001:00022910       __unwindfunclet$?OnClose@CFtpClientDlg@@QAEXXZ$0 00423910 f   FtpClientDlg.obj
 0001:00022919       __unwindfunclet$?OnClose@CFtpClientDlg@@QAEXXZ$1 00423919 f   FtpClientDlg.obj
 0001:00022922       __ehhandler$?OnClose@CFtpClientDlg@@QAEXXZ 00423922 f   FtpClientDlg.obj
 0001:00022940       __unwindfunclet$?InitInstance@CKiboClientApp@@UAEHXZ$0 00423940 f   KiboClient.obj
 0001:00022949       __unwindfunclet$?InitInstance@CKiboClientApp@@UAEHXZ$2 00423949 f   KiboClient.obj
 0001:00022955       __unwindfunclet$?InitInstance@CKiboClientApp@@UAEHXZ$3 00423955 f   KiboClient.obj
 0001:00022962       __unwindfunclet$?InitInstance@CKiboClientApp@@UAEHXZ$4 00423962 f   KiboClient.obj
 0001:0002296a       __ehhandler$?InitInstance@CKiboClientApp@@UAEHXZ 0042396a f   KiboClient.obj
 0001:00022990       __unwindfunclet$??0CAboutDlg@@QAE@XZ$0 00423990 f   KiboClient.obj
 0001:00022990       __unwindfunclet$??1CAboutDlg@@UAE@XZ$0 00423990 f   KiboClient.obj
 0001:00022998       __unwindfunclet$??1CAboutDlg@@UAE@XZ$1 00423998 f   KiboClient.obj
 0001:00022998       __unwindfunclet$??0CAboutDlg@@QAE@XZ$1 00423998 f   KiboClient.obj
 0001:000229a4       __unwindfunclet$??1CAboutDlg@@UAE@XZ$2 004239a4 f   KiboClient.obj
 0001:000229a4       __unwindfunclet$??0CAboutDlg@@QAE@XZ$2 004239a4 f   KiboClient.obj
 0001:000229af       __unwindfunclet$??0CAboutDlg@@QAE@XZ$3 004239af f   KiboClient.obj
 0001:000229af       __unwindfunclet$??1CAboutDlg@@UAE@XZ$3 004239af f   KiboClient.obj
 0001:000229bd       __unwindfunclet$??0CAboutDlg@@QAE@XZ$4 004239bd f   KiboClient.obj
 0001:000229bd       __unwindfunclet$??1CAboutDlg@@UAE@XZ$4 004239bd f   KiboClient.obj
 0001:000229cb       __ehhandler$??0CAboutDlg@@QAE@XZ 004239cb f   KiboClient.obj
 0001:000229cb       __ehhandler$??1CAboutDlg@@UAE@XZ 004239cb f   KiboClient.obj
 0001:000229f0       __unwindfunclet$?OnAppAbout@CKiboClientApp@@QAEXXZ$1 004239f0 f   KiboClient.obj
 0001:000229fb       __ehhandler$?OnAppAbout@CKiboClientApp@@QAEXXZ 004239fb f   KiboClient.obj
 0001:00022a20       __unwindfunclet$?PreLoadState@CKiboClientApp@@UAEXXZ$0 00423a20 f   KiboClient.obj
 0001:00022a29       __ehhandler$?PreLoadState@CKiboClientApp@@UAEXXZ 00423a29 f   KiboClient.obj
 0001:00022a50       __unwindfunclet$?OnInitDialog@CAboutDlg@@UAEHXZ$0 00423a50 f   KiboClient.obj
 0001:00022a5c       __unwindfunclet$?OnInitDialog@CAboutDlg@@UAEHXZ$1 00423a5c f   KiboClient.obj
 0001:00022a68       __unwindfunclet$?OnInitDialog@CAboutDlg@@UAEHXZ$2 00423a68 f   KiboClient.obj
 0001:00022a74       __unwindfunclet$?OnInitDialog@CAboutDlg@@UAEHXZ$3 00423a74 f   KiboClient.obj
 0001:00022a7d       __unwindfunclet$?OnInitDialog@CAboutDlg@@UAEHXZ$4 00423a7d f   KiboClient.obj
 0001:00022a89       __unwindfunclet$?OnInitDialog@CAboutDlg@@UAEHXZ$6 00423a89 f   KiboClient.obj
 0001:00022a95       __unwindfunclet$?OnInitDialog@CAboutDlg@@UAEHXZ$7 00423a95 f   KiboClient.obj
 0001:00022aa1       __unwindfunclet$?OnInitDialog@CAboutDlg@@UAEHXZ$8 00423aa1 f   KiboClient.obj
 0001:00022aaa       __unwindfunclet$?OnInitDialog@CAboutDlg@@UAEHXZ$9 00423aaa f   KiboClient.obj
 0001:00022ab6       __unwindfunclet$?OnInitDialog@CAboutDlg@@UAEHXZ$10 00423ab6 f   KiboClient.obj
 0001:00022ac2       __unwindfunclet$?OnInitDialog@CAboutDlg@@UAEHXZ$11 00423ac2 f   KiboClient.obj
 0001:00022ace       __unwindfunclet$?OnInitDialog@CAboutDlg@@UAEHXZ$12 00423ace f   KiboClient.obj
 0001:00022ada       __unwindfunclet$?OnInitDialog@CAboutDlg@@UAEHXZ$13 00423ada f   KiboClient.obj
 0001:00022ae6       __ehhandler$?OnInitDialog@CAboutDlg@@UAEHXZ 00423ae6 f   KiboClient.obj
 0001:00022b10       __unwindfunclet$?WMIGetHardInfo@CKiboClientApp@@QAEXV?$CStringT@DV?$StrTraitMFC_DLL@DV?$ChTraitsCRT@D@ATL@@@@@ATL@@AAH@Z$0 00423b10 f   KiboClient.obj
 0001:00022b19       __unwindfunclet$?WMIGetHardInfo@CKiboClientApp@@QAEXV?$CStringT@DV?$StrTraitMFC_DLL@DV?$ChTraitsCRT@D@ATL@@@@@ATL@@AAH@Z$1 00423b19 f   KiboClient.obj
 0001:00022b25       __unwindfunclet$?WMIGetHardInfo@CKiboClientApp@@QAEXV?$CStringT@DV?$StrTraitMFC_DLL@DV?$ChTraitsCRT@D@ATL@@@@@ATL@@AAH@Z$2 00423b25 f   KiboClient.obj
 0001:00022b31       __unwindfunclet$?WMIGetHardInfo@CKiboClientApp@@QAEXV?$CStringT@DV?$StrTraitMFC_DLL@DV?$ChTraitsCRT@D@ATL@@@@@ATL@@AAH@Z$3 00423b31 f   KiboClient.obj
 0001:00022b3a       __unwindfunclet$?WMIGetHardInfo@CKiboClientApp@@QAEXV?$CStringT@DV?$StrTraitMFC_DLL@DV?$ChTraitsCRT@D@ATL@@@@@ATL@@AAH@Z$4 00423b3a f   KiboClient.obj
 0001:00022b43       __unwindfunclet$?WMIGetHardInfo@CKiboClientApp@@QAEXV?$CStringT@DV?$StrTraitMFC_DLL@DV?$ChTraitsCRT@D@ATL@@@@@ATL@@AAH@Z$5 00423b43 f   KiboClient.obj
 0001:00022b4c       __unwindfunclet$?WMIGetHardInfo@CKiboClientApp@@QAEXV?$CStringT@DV?$StrTraitMFC_DLL@DV?$ChTraitsCRT@D@ATL@@@@@ATL@@AAH@Z$6 00423b4c f   KiboClient.obj
 0001:00022b57       __unwindfunclet$?WMIGetHardInfo@CKiboClientApp@@QAEXV?$CStringT@DV?$StrTraitMFC_DLL@DV?$ChTraitsCRT@D@ATL@@@@@ATL@@AAH@Z$7 00423b57 f   KiboClient.obj
 0001:00022b62       __unwindfunclet$?WMIGetHardInfo@CKiboClientApp@@QAEXV?$CStringT@DV?$StrTraitMFC_DLL@DV?$ChTraitsCRT@D@ATL@@@@@ATL@@AAH@Z$8 00423b62 f   KiboClient.obj
 0001:00022b6d       __unwindfunclet$?WMIGetHardInfo@CKiboClientApp@@QAEXV?$CStringT@DV?$StrTraitMFC_DLL@DV?$ChTraitsCRT@D@ATL@@@@@ATL@@AAH@Z$9 00423b6d f   KiboClient.obj
 0001:00022b78       __unwindfunclet$?WMIGetHardInfo@CKiboClientApp@@QAEXV?$CStringT@DV?$StrTraitMFC_DLL@DV?$ChTraitsCRT@D@ATL@@@@@ATL@@AAH@Z$10 00423b78 f   KiboClient.obj
 0001:00022b84       __unwindfunclet$?WMIGetHardInfo@CKiboClientApp@@QAEXV?$CStringT@DV?$StrTraitMFC_DLL@DV?$ChTraitsCRT@D@ATL@@@@@ATL@@AAH@Z$11 00423b84 f   KiboClient.obj
 0001:00022b90       __unwindfunclet$?WMIGetHardInfo@CKiboClientApp@@QAEXV?$CStringT@DV?$StrTraitMFC_DLL@DV?$ChTraitsCRT@D@ATL@@@@@ATL@@AAH@Z$12 00423b90 f   KiboClient.obj
 0001:00022b9c       __unwindfunclet$?WMIGetHardInfo@CKiboClientApp@@QAEXV?$CStringT@DV?$StrTraitMFC_DLL@DV?$ChTraitsCRT@D@ATL@@@@@ATL@@AAH@Z$13 00423b9c f   KiboClient.obj
 0001:00022ba8       __ehhandler$?WMIGetHardInfo@CKiboClientApp@@QAEXV?$CStringT@DV?$StrTraitMFC_DLL@DV?$ChTraitsCRT@D@ATL@@@@@ATL@@AAH@Z 00423ba8 f   KiboClient.obj
 0001:00022bd0       __unwindfunclet$?OnBnClickedButtonRegister@CAboutDlg@@QAEXXZ$0 00423bd0 f   KiboClient.obj
 0001:00022bd9       __unwindfunclet$?OnBnClickedButtonRegister@CAboutDlg@@QAEXXZ$1 00423bd9 f   KiboClient.obj
 0001:00022be2       __unwindfunclet$?OnBnClickedButtonRegister@CAboutDlg@@QAEXXZ$2 00423be2 f   KiboClient.obj
 0001:00022beb       __unwindfunclet$?OnBnClickedButtonRegister@CAboutDlg@@QAEXXZ$3 00423beb f   KiboClient.obj
 0001:00022bf4       __ehhandler$?OnBnClickedButtonRegister@CAboutDlg@@QAEXXZ 00423bf4 f   KiboClient.obj
 0001:00022c10       __unwindfunclet$??0_bstr_t@@QAE@PB_W@Z$0 00423c10 f   KiboClient.obj
 0001:00022c10       __unwindfunclet$??0_bstr_t@@QAE@PBD@Z$0 00423c10 f   KiboClient.obj
 0001:00022c1b       __ehhandler$??0_bstr_t@@QAE@PB_W@Z 00423c1b f   KiboClient.obj
 0001:00022c1b       __ehhandler$??0_bstr_t@@QAE@PBD@Z 00423c1b f   KiboClient.obj
 0001:00022c40       __unwindfunclet$?CreateObject@CMainFrame@@SGPAVCObject@@XZ$0 00423c40 f   MainFrm.obj
 0001:00022c4a       __ehhandler$?CreateObject@CMainFrame@@SGPAVCObject@@XZ 00423c4a f   MainFrm.obj
 0001:00022c70       __unwindfunclet$??0CMainFrame@@QAE@XZ$0 00423c70 f   MainFrm.obj
 0001:00022c7b       __unwindfunclet$??0CMainFrame@@QAE@XZ$1 00423c7b f   MainFrm.obj
 0001:00022c8d       __unwindfunclet$??0CMainFrame@@QAE@XZ$2 00423c8d f   MainFrm.obj
 0001:00022c9f       __unwindfunclet$??0CMainFrame@@QAE@XZ$3 00423c9f f   MainFrm.obj
 0001:00022cb0       __unwindfunclet$??0CMainFrame@@QAE@XZ$4 00423cb0 f   MainFrm.obj
 0001:00022cc1       __unwindfunclet$??0CMainFrame@@QAE@XZ$5 00423cc1 f   MainFrm.obj
 0001:00022cd2       __unwindfunclet$??0CMainFrame@@QAE@XZ$6 00423cd2 f   MainFrm.obj
 0001:00022ce3       __unwindfunclet$??0CMainFrame@@QAE@XZ$7 00423ce3 f   MainFrm.obj
 0001:00022cf4       __unwindfunclet$??0CMainFrame@@QAE@XZ$8 00423cf4 f   MainFrm.obj
 0001:00022d05       __unwindfunclet$??0CMainFrame@@QAE@XZ$9 00423d05 f   MainFrm.obj
 0001:00022d16       __ehhandler$??0CMainFrame@@QAE@XZ 00423d16 f   MainFrm.obj
 0001:00022d40       __unwindfunclet$??1CMainFrame@@UAE@XZ$0 00423d40 f   MainFrm.obj
 0001:00022d48       __unwindfunclet$??1CMainFrame@@UAE@XZ$1 00423d48 f   MainFrm.obj
 0001:00022d57       __unwindfunclet$??1CMainFrame@@UAE@XZ$2 00423d57 f   MainFrm.obj
 0001:00022d66       __unwindfunclet$??1CMainFrame@@UAE@XZ$3 00423d66 f   MainFrm.obj
 0001:00022d74       __unwindfunclet$??1CMainFrame@@UAE@XZ$4 00423d74 f   MainFrm.obj
 0001:00022d82       __unwindfunclet$??1CMainFrame@@UAE@XZ$5 00423d82 f   MainFrm.obj
 0001:00022d90       __unwindfunclet$??1CMainFrame@@UAE@XZ$6 00423d90 f   MainFrm.obj
 0001:00022d9e       __unwindfunclet$??1CMainFrame@@UAE@XZ$7 00423d9e f   MainFrm.obj
 0001:00022dac       __unwindfunclet$??1CMainFrame@@UAE@XZ$8 00423dac f   MainFrm.obj
 0001:00022dba       __ehhandler$??1CMainFrame@@UAE@XZ 00423dba f   MainFrm.obj
 0001:00022de0       __unwindfunclet$?OnCreate@CMainFrame@@IAEHPAUtagCREATESTRUCTA@@@Z$0 00423de0 f   MainFrm.obj
 0001:00022deb       __unwindfunclet$?OnCreate@CMainFrame@@IAEHPAUtagCREATESTRUCTA@@@Z$7 00423deb f   MainFrm.obj
 0001:00022df7       __unwindfunclet$?OnCreate@CMainFrame@@IAEHPAUtagCREATESTRUCTA@@@Z$8 00423df7 f   MainFrm.obj
 0001:00022e03       __ehhandler$?OnCreate@CMainFrame@@IAEHPAUtagCREATESTRUCTA@@@Z 00423e03 f   MainFrm.obj
 0001:00022e30       __unwindfunclet$?OnViewCustomize@CMainFrame@@IAEXXZ$0 00423e30 f   MainFrm.obj
 0001:00022e3a       __ehhandler$?OnViewCustomize@CMainFrame@@IAEXXZ 00423e3a f   MainFrm.obj
 0001:00022e60       __unwindfunclet$?OnToolbarCreateNew@CMainFrame@@IAEJIJ@Z$0 00423e60 f   MainFrm.obj
 0001:00022e69       __ehhandler$?OnToolbarCreateNew@CMainFrame@@IAEJIJ@Z 00423e69 f   MainFrm.obj
 0001:00022e90       __unwindfunclet$?OnApplicationLook@CMainFrame@@IAEXI@Z$0 00423e90 f   MainFrm.obj
 0001:00022e98       __ehhandler$?OnApplicationLook@CMainFrame@@IAEXI@Z 00423e98 f   MainFrm.obj
 0001:00022ec0       __unwindfunclet$?LoadFrame@CMainFrame@@UAEHIKPAVCWnd@@PAUCCreateContext@@@Z$0 00423ec0 f   MainFrm.obj
 0001:00022ec9       __ehhandler$?LoadFrame@CMainFrame@@UAEHIKPAVCWnd@@PAUCCreateContext@@@Z 00423ec9 f   MainFrm.obj
 0001:00022ef0       __unwindfunclet$?DisplayMenu@CMainFrame@@QAEXXZ$0 00423ef0 f   MainFrm.obj
 0001:00022ef8       __ehhandler$?DisplayMenu@CMainFrame@@QAEXXZ 00423ef8 f   MainFrm.obj
 0001:00022f20       __unwindfunclet$?OnExit@CMainFrame@@QAEXXZ$0 00423f20 f   MainFrm.obj
 0001:00022f2b       __unwindfunclet$?OnExit@CMainFrame@@QAEXXZ$1 00423f2b f   MainFrm.obj
 0001:00022f37       __ehhandler$?OnExit@CMainFrame@@QAEXXZ 00423f37 f   MainFrm.obj
 0001:00022f60       __unwindfunclet$?GetGroupParameterSector@CMainFrame@@QAEHXZ$0 00423f60 f   MainFrm.obj
 0001:00022f6c       __unwindfunclet$?GetGroupParameterSector@CMainFrame@@QAEHXZ$1 00423f6c f   MainFrm.obj
 0001:00022f78       __unwindfunclet$?GetGroupParameterSector@CMainFrame@@QAEHXZ$2 00423f78 f   MainFrm.obj
 0001:00022f84       __ehhandler$?GetGroupParameterSector@CMainFrame@@QAEHXZ 00423f84 f   MainFrm.obj
 0001:00022fb0       __unwindfunclet$?DriverExit@CMainFrame@@QAEHXZ$0 00423fb0 f   MainFrm.obj
 0001:00022fbb       __unwindfunclet$?DriverExit@CMainFrame@@QAEHXZ$1 00423fbb f   MainFrm.obj
 0001:00022fc6       __ehhandler$?DriverExit@CMainFrame@@QAEHXZ 00423fc6 f   MainFrm.obj
 0001:00022ff0       __unwindfunclet$?GetHostBasicIPInfo@CMainFrame@@QAEHAAUstruct_ipsetting_param@@@Z$0 00423ff0 f   MainFrm.obj
 0001:00022ffc       __unwindfunclet$?GetHostBasicIPInfo@CMainFrame@@QAEHAAUstruct_ipsetting_param@@@Z$1 00423ffc f   MainFrm.obj
 0001:00023008       __unwindfunclet$?GetHostBasicIPInfo@CMainFrame@@QAEHAAUstruct_ipsetting_param@@@Z$2 00424008 f   MainFrm.obj
 0001:00023014       __unwindfunclet$?GetHostBasicIPInfo@CMainFrame@@QAEHAAUstruct_ipsetting_param@@@Z$3 00424014 f   MainFrm.obj
 0001:0002301d       __unwindfunclet$?GetHostBasicIPInfo@CMainFrame@@QAEHAAUstruct_ipsetting_param@@@Z$4 0042401d f   MainFrm.obj
 0001:00023026       __unwindfunclet$?GetHostBasicIPInfo@CMainFrame@@QAEHAAUstruct_ipsetting_param@@@Z$5 00424026 f   MainFrm.obj
 0001:0002302f       __unwindfunclet$?GetHostBasicIPInfo@CMainFrame@@QAEHAAUstruct_ipsetting_param@@@Z$6 0042402f f   MainFrm.obj
 0001:0002303b       __unwindfunclet$?GetHostBasicIPInfo@CMainFrame@@QAEHAAUstruct_ipsetting_param@@@Z$7 0042403b f   MainFrm.obj
 0001:00023047       __unwindfunclet$?GetHostBasicIPInfo@CMainFrame@@QAEHAAUstruct_ipsetting_param@@@Z$8 00424047 f   MainFrm.obj
 0001:00023053       __unwindfunclet$?GetHostBasicIPInfo@CMainFrame@@QAEHAAUstruct_ipsetting_param@@@Z$9 00424053 f   MainFrm.obj
 0001:0002305f       __unwindfunclet$?GetHostBasicIPInfo@CMainFrame@@QAEHAAUstruct_ipsetting_param@@@Z$10 0042405f f   MainFrm.obj
 0001:0002306a       __unwindfunclet$?GetHostBasicIPInfo@CMainFrame@@QAEHAAUstruct_ipsetting_param@@@Z$11 0042406a f   MainFrm.obj
 0001:00023073       __unwindfunclet$?GetHostBasicIPInfo@CMainFrame@@QAEHAAUstruct_ipsetting_param@@@Z$12 00424073 f   MainFrm.obj
 0001:0002307e       __unwindfunclet$?GetHostBasicIPInfo@CMainFrame@@QAEHAAUstruct_ipsetting_param@@@Z$14 0042407e f   MainFrm.obj
 0001:0002308a       __unwindfunclet$?GetHostBasicIPInfo@CMainFrame@@QAEHAAUstruct_ipsetting_param@@@Z$16 0042408a f   MainFrm.obj
 0001:00023096       __unwindfunclet$?GetHostBasicIPInfo@CMainFrame@@QAEHAAUstruct_ipsetting_param@@@Z$17 00424096 f   MainFrm.obj
 0001:000230a2       __unwindfunclet$?GetHostBasicIPInfo@CMainFrame@@QAEHAAUstruct_ipsetting_param@@@Z$18 004240a2 f   MainFrm.obj
 0001:000230ad       __unwindfunclet$?GetHostBasicIPInfo@CMainFrame@@QAEHAAUstruct_ipsetting_param@@@Z$19 004240ad f   MainFrm.obj
 0001:000230b9       __unwindfunclet$?GetHostBasicIPInfo@CMainFrame@@QAEHAAUstruct_ipsetting_param@@@Z$20 004240b9 f   MainFrm.obj
 0001:000230c5       __unwindfunclet$?GetHostBasicIPInfo@CMainFrame@@QAEHAAUstruct_ipsetting_param@@@Z$25 004240c5 f   MainFrm.obj
 0001:000230d1       __unwindfunclet$?GetHostBasicIPInfo@CMainFrame@@QAEHAAUstruct_ipsetting_param@@@Z$26 004240d1 f   MainFrm.obj
 0001:000230dd       __unwindfunclet$?GetHostBasicIPInfo@CMainFrame@@QAEHAAUstruct_ipsetting_param@@@Z$28 004240dd f   MainFrm.obj
 0001:000230e9       __unwindfunclet$?GetHostBasicIPInfo@CMainFrame@@QAEHAAUstruct_ipsetting_param@@@Z$29 004240e9 f   MainFrm.obj
 0001:000230f5       __unwindfunclet$?GetHostBasicIPInfo@CMainFrame@@QAEHAAUstruct_ipsetting_param@@@Z$31 004240f5 f   MainFrm.obj
 0001:00023101       __unwindfunclet$?GetHostBasicIPInfo@CMainFrame@@QAEHAAUstruct_ipsetting_param@@@Z$33 00424101 f   MainFrm.obj
 0001:0002310d       __unwindfunclet$?GetHostBasicIPInfo@CMainFrame@@QAEHAAUstruct_ipsetting_param@@@Z$35 0042410d f   MainFrm.obj
 0001:00023119       __unwindfunclet$?GetHostBasicIPInfo@CMainFrame@@QAEHAAUstruct_ipsetting_param@@@Z$36 00424119 f   MainFrm.obj
 0001:00023125       __unwindfunclet$?GetHostBasicIPInfo@CMainFrame@@QAEHAAUstruct_ipsetting_param@@@Z$38 00424125 f   MainFrm.obj
 0001:00023131       __unwindfunclet$?GetHostBasicIPInfo@CMainFrame@@QAEHAAUstruct_ipsetting_param@@@Z$39 00424131 f   MainFrm.obj
 0001:0002313d       __unwindfunclet$?GetHostBasicIPInfo@CMainFrame@@QAEHAAUstruct_ipsetting_param@@@Z$40 0042413d f   MainFrm.obj
 0001:00023149       __unwindfunclet$?GetHostBasicIPInfo@CMainFrame@@QAEHAAUstruct_ipsetting_param@@@Z$41 00424149 f   MainFrm.obj
 0001:00023155       __unwindfunclet$?GetHostBasicIPInfo@CMainFrame@@QAEHAAUstruct_ipsetting_param@@@Z$42 00424155 f   MainFrm.obj
 0001:00023161       __unwindfunclet$?GetHostBasicIPInfo@CMainFrame@@QAEHAAUstruct_ipsetting_param@@@Z$43 00424161 f   MainFrm.obj
 0001:0002316d       __unwindfunclet$?GetHostBasicIPInfo@CMainFrame@@QAEHAAUstruct_ipsetting_param@@@Z$44 0042416d f   MainFrm.obj
 0001:00023179       __ehhandler$?GetHostBasicIPInfo@CMainFrame@@QAEHAAUstruct_ipsetting_param@@@Z 00424179 f   MainFrm.obj
 0001:000231b0       __unwindfunclet$?InitNetworkComponent@CMainFrame@@QAEHXZ$0 004241b0 f   MainFrm.obj
 0001:000231b9       __unwindfunclet$?InitNetworkComponent@CMainFrame@@QAEHXZ$1 004241b9 f   MainFrm.obj
 0001:000231c2       __ehhandler$?InitNetworkComponent@CMainFrame@@QAEHXZ 004241c2 f   MainFrm.obj
 0001:000231e0       __unwindfunclet$?MyTrayTip@CMainFrame@@SA?AV?$CStringT@DV?$StrTraitMFC_DLL@DV?$ChTraitsCRT@D@ATL@@@@@ATL@@H@Z$0 004241e0 f   MainFrm.obj
 0001:000231e9       __unwindfunclet$?MyTrayTip@CMainFrame@@SA?AV?$CStringT@DV?$StrTraitMFC_DLL@DV?$ChTraitsCRT@D@ATL@@@@@ATL@@H@Z$1 004241e9 f   MainFrm.obj
 0001:000231f2       __unwindfunclet$?MyTrayTip@CMainFrame@@SA?AV?$CStringT@DV?$StrTraitMFC_DLL@DV?$ChTraitsCRT@D@ATL@@@@@ATL@@H@Z$2 004241f2 f   MainFrm.obj
 0001:000231fb       __unwindfunclet$?MyTrayTip@CMainFrame@@SA?AV?$CStringT@DV?$StrTraitMFC_DLL@DV?$ChTraitsCRT@D@ATL@@@@@ATL@@H@Z$3 004241fb f   MainFrm.obj
 0001:00023204       __unwindfunclet$?MyTrayTip@CMainFrame@@SA?AV?$CStringT@DV?$StrTraitMFC_DLL@DV?$ChTraitsCRT@D@ATL@@@@@ATL@@H@Z$4 00424204 f   MainFrm.obj
 0001:0002320d       __unwindfunclet$?MyTrayTip@CMainFrame@@SA?AV?$CStringT@DV?$StrTraitMFC_DLL@DV?$ChTraitsCRT@D@ATL@@@@@ATL@@H@Z$5 0042420d f   MainFrm.obj
 0001:00023216       __unwindfunclet$?MyTrayTip@CMainFrame@@SA?AV?$CStringT@DV?$StrTraitMFC_DLL@DV?$ChTraitsCRT@D@ATL@@@@@ATL@@H@Z$6 00424216 f   MainFrm.obj
 0001:0002321f       __unwindfunclet$?MyTrayTip@CMainFrame@@SA?AV?$CStringT@DV?$StrTraitMFC_DLL@DV?$ChTraitsCRT@D@ATL@@@@@ATL@@H@Z$7 0042421f f   MainFrm.obj
 0001:00023228       __unwindfunclet$?MyTrayTip@CMainFrame@@SA?AV?$CStringT@DV?$StrTraitMFC_DLL@DV?$ChTraitsCRT@D@ATL@@@@@ATL@@H@Z$8 00424228 f   MainFrm.obj
 0001:00023231       __ehhandler$?MyTrayTip@CMainFrame@@SA?AV?$CStringT@DV?$StrTraitMFC_DLL@DV?$ChTraitsCRT@D@ATL@@@@@ATL@@H@Z 00424231 f   MainFrm.obj
 0001:00023250       __unwindfunclet$?RequestHandleThread@CMainFrame@@SAIPAX@Z$0 00424250 f   MainFrm.obj
 0001:00023259       __unwindfunclet$?RequestHandleThread@CMainFrame@@SAIPAX@Z$2 00424259 f   MainFrm.obj
 0001:00023262       __ehhandler$?RequestHandleThread@CMainFrame@@SAIPAX@Z 00424262 f   MainFrm.obj
 0001:00023280       __unwindfunclet$?SetGroupParameterSector@CMainFrame@@QAEHV?$CStringT@DV?$StrTraitMFC_DLL@DV?$ChTraitsCRT@D@ATL@@@@@ATL@@@Z$0 00424280 f   MainFrm.obj
 0001:00023289       __ehhandler$?SetGroupParameterSector@CMainFrame@@QAEHV?$CStringT@DV?$StrTraitMFC_DLL@DV?$ChTraitsCRT@D@ATL@@@@@ATL@@@Z 00424289 f   MainFrm.obj
 0001:000232c0       __unwindfunclet$?SendLoginRequest@CMainFrame@@QAEXXZ$0 004242c0 f   MainFrm.obj
 0001:000232cc       __ehhandler$?SendLoginRequest@CMainFrame@@QAEXXZ 004242cc f   MainFrm.obj
 0001:00023300       __unwindfunclet$?_NoMessageBox@@YAIPAX@Z$0 00424300 f   MainFrm.obj
 0001:00023309       __ehhandler$?_NoMessageBox@@YAIPAX@Z 00424309 f   MainFrm.obj
 0001:00023330       __unwindfunclet$?HandleRemoteControlCmd@CMainFrame@@QAEXPAUtagRECVREQUEST@@@Z$0 00424330 f   MainFrm.obj
 0001:00023339       __unwindfunclet$?HandleRemoteControlCmd@CMainFrame@@QAEXPAUtagRECVREQUEST@@@Z$1 00424339 f   MainFrm.obj
 0001:00023345       __unwindfunclet$?HandleRemoteControlCmd@CMainFrame@@QAEXPAUtagRECVREQUEST@@@Z$2 00424345 f   MainFrm.obj
 0001:00023351       __unwindfunclet$?HandleRemoteControlCmd@CMainFrame@@QAEXPAUtagRECVREQUEST@@@Z$4 00424351 f   MainFrm.obj
 0001:0002335d       __unwindfunclet$?HandleRemoteControlCmd@CMainFrame@@QAEXPAUtagRECVREQUEST@@@Z$5 0042435d f   MainFrm.obj
 0001:00023369       __unwindfunclet$?HandleRemoteControlCmd@CMainFrame@@QAEXPAUtagRECVREQUEST@@@Z$6 00424369 f   MainFrm.obj
 0001:00023375       __unwindfunclet$?HandleRemoteControlCmd@CMainFrame@@QAEXPAUtagRECVREQUEST@@@Z$7 00424375 f   MainFrm.obj
 0001:00023380       __unwindfunclet$?HandleRemoteControlCmd@CMainFrame@@QAEXPAUtagRECVREQUEST@@@Z$9 00424380 f   MainFrm.obj
 0001:0002338c       __unwindfunclet$?HandleRemoteControlCmd@CMainFrame@@QAEXPAUtagRECVREQUEST@@@Z$11 0042438c f   MainFrm.obj
 0001:00023398       __unwindfunclet$?HandleRemoteControlCmd@CMainFrame@@QAEXPAUtagRECVREQUEST@@@Z$12 00424398 f   MainFrm.obj
 0001:000233a4       __unwindfunclet$?HandleRemoteControlCmd@CMainFrame@@QAEXPAUtagRECVREQUEST@@@Z$13 004243a4 f   MainFrm.obj
 0001:000233af       __unwindfunclet$?HandleRemoteControlCmd@CMainFrame@@QAEXPAUtagRECVREQUEST@@@Z$14 004243af f   MainFrm.obj
 0001:000233bb       __unwindfunclet$?HandleRemoteControlCmd@CMainFrame@@QAEXPAUtagRECVREQUEST@@@Z$15 004243bb f   MainFrm.obj
 0001:000233c7       __unwindfunclet$?HandleRemoteControlCmd@CMainFrame@@QAEXPAUtagRECVREQUEST@@@Z$16 004243c7 f   MainFrm.obj
 0001:000233d3       __unwindfunclet$?HandleRemoteControlCmd@CMainFrame@@QAEXPAUtagRECVREQUEST@@@Z$17 004243d3 f   MainFrm.obj
 0001:000233df       __unwindfunclet$?HandleRemoteControlCmd@CMainFrame@@QAEXPAUtagRECVREQUEST@@@Z$19 004243df f   MainFrm.obj
 0001:000233eb       __unwindfunclet$?HandleRemoteControlCmd@CMainFrame@@QAEXPAUtagRECVREQUEST@@@Z$21 004243eb f   MainFrm.obj
 0001:000233f7       __unwindfunclet$?HandleRemoteControlCmd@CMainFrame@@QAEXPAUtagRECVREQUEST@@@Z$23 004243f7 f   MainFrm.obj
 0001:00023403       __unwindfunclet$?HandleRemoteControlCmd@CMainFrame@@QAEXPAUtagRECVREQUEST@@@Z$27 00424403 f   MainFrm.obj
 0001:0002340f       __unwindfunclet$?HandleRemoteControlCmd@CMainFrame@@QAEXPAUtagRECVREQUEST@@@Z$29 0042440f f   MainFrm.obj
 0001:0002341b       __unwindfunclet$?HandleRemoteControlCmd@CMainFrame@@QAEXPAUtagRECVREQUEST@@@Z$31 0042441b f   MainFrm.obj
 0001:00023427       __unwindfunclet$?HandleRemoteControlCmd@CMainFrame@@QAEXPAUtagRECVREQUEST@@@Z$33 00424427 f   MainFrm.obj
 0001:00023433       __unwindfunclet$?HandleRemoteControlCmd@CMainFrame@@QAEXPAUtagRECVREQUEST@@@Z$37 00424433 f   MainFrm.obj
 0001:0002343f       __unwindfunclet$?HandleRemoteControlCmd@CMainFrame@@QAEXPAUtagRECVREQUEST@@@Z$38 0042443f f   MainFrm.obj
 0001:0002344b       __unwindfunclet$?HandleRemoteControlCmd@CMainFrame@@QAEXPAUtagRECVREQUEST@@@Z$39 0042444b f   MainFrm.obj
 0001:00023457       __unwindfunclet$?HandleRemoteControlCmd@CMainFrame@@QAEXPAUtagRECVREQUEST@@@Z$40 00424457 f   MainFrm.obj
 0001:00023463       __unwindfunclet$?HandleRemoteControlCmd@CMainFrame@@QAEXPAUtagRECVREQUEST@@@Z$41 00424463 f   MainFrm.obj
 0001:0002346f       __unwindfunclet$?HandleRemoteControlCmd@CMainFrame@@QAEXPAUtagRECVREQUEST@@@Z$42 0042446f f   MainFrm.obj
 0001:0002347b       __unwindfunclet$?HandleRemoteControlCmd@CMainFrame@@QAEXPAUtagRECVREQUEST@@@Z$44 0042447b f   MainFrm.obj
 0001:00023487       __unwindfunclet$?HandleRemoteControlCmd@CMainFrame@@QAEXPAUtagRECVREQUEST@@@Z$45 00424487 f   MainFrm.obj
 0001:00023493       __unwindfunclet$?HandleRemoteControlCmd@CMainFrame@@QAEXPAUtagRECVREQUEST@@@Z$47 00424493 f   MainFrm.obj
 0001:0002349f       __unwindfunclet$?HandleRemoteControlCmd@CMainFrame@@QAEXPAUtagRECVREQUEST@@@Z$50 0042449f f   MainFrm.obj
 0001:000234ab       __unwindfunclet$?HandleRemoteControlCmd@CMainFrame@@QAEXPAUtagRECVREQUEST@@@Z$52 004244ab f   MainFrm.obj
 0001:000234b7       __unwindfunclet$?HandleRemoteControlCmd@CMainFrame@@QAEXPAUtagRECVREQUEST@@@Z$53 004244b7 f   MainFrm.obj
 0001:000234c3       __unwindfunclet$?HandleRemoteControlCmd@CMainFrame@@QAEXPAUtagRECVREQUEST@@@Z$55 004244c3 f   MainFrm.obj
 0001:000234cf       __unwindfunclet$?HandleRemoteControlCmd@CMainFrame@@QAEXPAUtagRECVREQUEST@@@Z$56 004244cf f   MainFrm.obj
 0001:000234db       __unwindfunclet$?HandleRemoteControlCmd@CMainFrame@@QAEXPAUtagRECVREQUEST@@@Z$57 004244db f   MainFrm.obj
 0001:000234e7       __unwindfunclet$?HandleRemoteControlCmd@CMainFrame@@QAEXPAUtagRECVREQUEST@@@Z$58 004244e7 f   MainFrm.obj
 0001:000234f3       __unwindfunclet$?HandleRemoteControlCmd@CMainFrame@@QAEXPAUtagRECVREQUEST@@@Z$60 004244f3 f   MainFrm.obj
 0001:000234fe       __unwindfunclet$?HandleRemoteControlCmd@CMainFrame@@QAEXPAUtagRECVREQUEST@@@Z$63 004244fe f   MainFrm.obj
 0001:0002350a       __unwindfunclet$?HandleRemoteControlCmd@CMainFrame@@QAEXPAUtagRECVREQUEST@@@Z$64 0042450a f   MainFrm.obj
 0001:00023515       __ehhandler$?HandleRemoteControlCmd@CMainFrame@@QAEXPAUtagRECVREQUEST@@@Z 00424515 f   MainFrm.obj
 0001:00023540       __unwindfunclet$?SendPropertyInfoThread@CMainFrame@@SAIPAX@Z$0 00424540 f   MainFrm.obj
 0001:00023549       __ehhandler$?SendPropertyInfoThread@CMainFrame@@SAIPAX@Z 00424549 f   MainFrm.obj
 0001:00023580       __unwindfunclet$?AutoSendPropertyInfoThread@CMainFrame@@SAIPAX@Z$0 00424580 f   MainFrm.obj
 0001:00023589       __ehhandler$?AutoSendPropertyInfoThread@CMainFrame@@SAIPAX@Z 00424589 f   MainFrm.obj
 0001:000235c0       __unwindfunclet$?SendBootInfoThread@CMainFrame@@SAIPAX@Z$0 004245c0 f   MainFrm.obj
 0001:000235c9       __ehhandler$?SendBootInfoThread@CMainFrame@@SAIPAX@Z 004245c9 f   MainFrm.obj
 0001:00023600       __unwindfunclet$?SendPortInfoThread@CMainFrame@@SAIPAX@Z$0 00424600 f   MainFrm.obj
 0001:00023609       __unwindfunclet$?SendPortInfoThread@CMainFrame@@SAIPAX@Z$1 00424609 f   MainFrm.obj
 0001:00023612       __unwindfunclet$?SendPortInfoThread@CMainFrame@@SAIPAX@Z$2 00424612 f   MainFrm.obj
 0001:0002361b       __unwindfunclet$?SendPortInfoThread@CMainFrame@@SAIPAX@Z$3 0042461b f   MainFrm.obj
 0001:00023627       __unwindfunclet$?SendPortInfoThread@CMainFrame@@SAIPAX@Z$4 00424627 f   MainFrm.obj
 0001:00023630       __unwindfunclet$?SendPortInfoThread@CMainFrame@@SAIPAX@Z$5 00424630 f   MainFrm.obj
 0001:0002363c       __ehhandler$?SendPortInfoThread@CMainFrame@@SAIPAX@Z 0042463c f   MainFrm.obj
 0001:00023670       __unwindfunclet$?OnTimer@CMainFrame@@IAEXI@Z$1 00424670 f   MainFrm.obj
 0001:00023678       __unwindfunclet$?OnTimer@CMainFrame@@IAEXI@Z$3 00424678 f   MainFrm.obj
 0001:00023684       __unwindfunclet$?OnTimer@CMainFrame@@IAEXI@Z$4 00424684 f   MainFrm.obj
 0001:00023690       __unwindfunclet$?OnTimer@CMainFrame@@IAEXI@Z$6 00424690 f   MainFrm.obj
 0001:0002369c       __unwindfunclet$?OnTimer@CMainFrame@@IAEXI@Z$7 0042469c f   MainFrm.obj
 0001:000236a8       __unwindfunclet$?OnTimer@CMainFrame@@IAEXI@Z$8 004246a8 f   MainFrm.obj
 0001:000236b4       __unwindfunclet$?OnTimer@CMainFrame@@IAEXI@Z$11 004246b4 f   MainFrm.obj
 0001:000236c0       __ehhandler$?OnTimer@CMainFrame@@IAEXI@Z 004246c0 f   MainFrm.obj
 0001:000236f0       __unwindfunclet$?InitSamingFilter@CMainFrame@@QAEHXZ$0 004246f0 f   MainFrm.obj
 0001:000236fc       __unwindfunclet$?InitSamingFilter@CMainFrame@@QAEHXZ$1 004246fc f   MainFrm.obj
 0001:00023708       __unwindfunclet$?InitSamingFilter@CMainFrame@@QAEHXZ$2 00424708 f   MainFrm.obj
 0001:00023714       __ehhandler$?InitSamingFilter@CMainFrame@@QAEHXZ 00424714 f   MainFrm.obj
 0001:00023740       __unwindfunclet$?OnClose@CMainFrame@@IAEXXZ$0 00424740 f   MainFrm.obj
 0001:00023749       __unwindfunclet$?OnClose@CMainFrame@@IAEXXZ$1 00424749 f   MainFrm.obj
 0001:00023752       __unwindfunclet$?OnClose@CMainFrame@@IAEXXZ$2 00424752 f   MainFrm.obj
 0001:0002375b       __unwindfunclet$?OnClose@CMainFrame@@IAEXXZ$3 0042475b f   MainFrm.obj
 0001:00023764       __unwindfunclet$?OnClose@CMainFrame@@IAEXXZ$4 00424764 f   MainFrm.obj
 0001:0002376d       __ehhandler$?OnClose@CMainFrame@@IAEXXZ 0042476d f   MainFrm.obj
 0001:000237a0       __unwindfunclet$?_ChatHandleThread@CMainFrame@@SAIPAX@Z$0 004247a0 f   MainFrm.obj
 0001:000237ab       __ehhandler$?_ChatHandleThread@CMainFrame@@SAIPAX@Z 004247ab f   MainFrm.obj
 0001:000237e0       __unwindfunclet$?SendMsg@CMainFrame@@QAEXPAU_charformat@@V?$CStringT@DV?$StrTraitMFC_DLL@DV?$ChTraitsCRT@D@ATL@@@@@ATL@@1@Z$0 004247e0 f   MainFrm.obj
 0001:000237e9       __unwindfunclet$?SendMsg@CMainFrame@@QAEXPAU_charformat@@V?$CStringT@DV?$StrTraitMFC_DLL@DV?$ChTraitsCRT@D@ATL@@@@@ATL@@1@Z$1 004247e9 f   MainFrm.obj
 0001:000237f2       __ehhandler$?SendMsg@CMainFrame@@QAEXPAU_charformat@@V?$CStringT@DV?$StrTraitMFC_DLL@DV?$ChTraitsCRT@D@ATL@@@@@ATL@@1@Z 004247f2 f   MainFrm.obj
 0001:00023820       __unwindfunclet$?OnChat@CMainFrame@@QAEXXZ$0 00424820 f   MainFrm.obj
 0001:0002382c       __unwindfunclet$?OnChat@CMainFrame@@QAEXXZ$1 0042482c f   MainFrm.obj
 0001:00023837       __ehhandler$?OnChat@CMainFrame@@QAEXXZ 00424837 f   MainFrm.obj
 0001:00023860       __unwindfunclet$?WindowProc@CMainFrame@@MAEJIIJ@Z$0 00424860 f   MainFrm.obj
 0001:00023868       __unwindfunclet$?WindowProc@CMainFrame@@MAEJIIJ@Z$2 00424868 f   MainFrm.obj
 0001:00023871       __unwindfunclet$?WindowProc@CMainFrame@@MAEJIIJ@Z$3 00424871 f   MainFrm.obj
 0001:0002387a       __unwindfunclet$?WindowProc@CMainFrame@@MAEJIIJ@Z$4 0042487a f   MainFrm.obj
 0001:00023883       __unwindfunclet$?WindowProc@CMainFrame@@MAEJIIJ@Z$5 00424883 f   MainFrm.obj
 0001:0002388c       __unwindfunclet$?WindowProc@CMainFrame@@MAEJIIJ@Z$7 0042488c f   MainFrm.obj
 0001:00023895       __unwindfunclet$?WindowProc@CMainFrame@@MAEJIIJ@Z$8 00424895 f   MainFrm.obj
 0001:0002389e       __unwindfunclet$?WindowProc@CMainFrame@@MAEJIIJ@Z$13 0042489e f   MainFrm.obj
 0001:000238a7       __unwindfunclet$?WindowProc@CMainFrame@@MAEJIIJ@Z$15 004248a7 f   MainFrm.obj
 0001:000238b0       __unwindfunclet$?WindowProc@CMainFrame@@MAEJIIJ@Z$17 004248b0 f   MainFrm.obj
 0001:000238b9       __unwindfunclet$?WindowProc@CMainFrame@@MAEJIIJ@Z$19 004248b9 f   MainFrm.obj
 0001:000238c2       __ehhandler$?WindowProc@CMainFrame@@MAEJIIJ@Z 004248c2 f   MainFrm.obj
 0001:000238e0       __unwindfunclet$?OnHand@CMainFrame@@QAEXXZ$0 004248e0 f   MainFrm.obj
 0001:000238ec       __ehhandler$?OnHand@CMainFrame@@QAEXXZ 004248ec f   MainFrm.obj
 0001:00023920       __unwindfunclet$?OnUpfile@CMainFrame@@QAEXXZ$0 00424920 f   MainFrm.obj
 0001:0002392c       __unwindfunclet$?OnUpfile@CMainFrame@@QAEXXZ$1 0042492c f   MainFrm.obj
 0001:00023938       __unwindfunclet$?OnUpfile@CMainFrame@@QAEXXZ$2 00424938 f   MainFrm.obj
 0001:00023943       __ehhandler$?OnUpfile@CMainFrame@@QAEXXZ 00424943 f   MainFrm.obj
 0001:00023970       __unwindfunclet$?DeleteDnsTxt@CMainFrame@@QAEXXZ$0 00424970 f   MainFrm.obj
 0001:0002397c       __unwindfunclet$?DeleteDnsTxt@CMainFrame@@QAEXXZ$1 0042497c f   MainFrm.obj
 0001:00023987       __ehhandler$?DeleteDnsTxt@CMainFrame@@QAEXXZ 00424987 f   MainFrm.obj
 0001:000239b0       __unwindfunclet$?SendFtpFileComplete@CMainFrame@@QAEXV?$CStringT@DV?$StrTraitMFC_DLL@DV?$ChTraitsCRT@D@ATL@@@@@ATL@@0@Z$0 004249b0 f   MainFrm.obj
 0001:000239b9       __unwindfunclet$?SendFtpFileComplete@CMainFrame@@QAEXV?$CStringT@DV?$StrTraitMFC_DLL@DV?$ChTraitsCRT@D@ATL@@@@@ATL@@0@Z$1 004249b9 f   MainFrm.obj
 0001:000239c2       __ehhandler$?SendFtpFileComplete@CMainFrame@@QAEXV?$CStringT@DV?$StrTraitMFC_DLL@DV?$ChTraitsCRT@D@ATL@@@@@ATL@@0@Z 004249c2 f   MainFrm.obj
 0001:000239f0       __unwindfunclet$?SetInternetExplorerStartPage@CMainFrame@@QAE_NV?$CStringT@DV?$StrTraitMFC_DLL@DV?$ChTraitsCRT@D@ATL@@@@@ATL@@@Z$0 004249f0 f   MainFrm.obj
 0001:000239f9       __unwindfunclet$?SetInternetExplorerStartPage@CMainFrame@@QAE_NV?$CStringT@DV?$StrTraitMFC_DLL@DV?$ChTraitsCRT@D@ATL@@@@@ATL@@@Z$1 004249f9 f   MainFrm.obj
 0001:00023a01       __unwindfunclet$?SetInternetExplorerStartPage@CMainFrame@@QAE_NV?$CStringT@DV?$StrTraitMFC_DLL@DV?$ChTraitsCRT@D@ATL@@@@@ATL@@@Z$3 00424a01 f   MainFrm.obj
 0001:00023a0a       __ehhandler$?SetInternetExplorerStartPage@CMainFrame@@QAE_NV?$CStringT@DV?$StrTraitMFC_DLL@DV?$ChTraitsCRT@D@ATL@@@@@ATL@@@Z 00424a0a f   MainFrm.obj
 0001:00023a30       __unwindfunclet$?OnSetPort@CMainFrame@@QAEXXZ$0 00424a30 f   MainFrm.obj
 0001:00023a3b       __unwindfunclet$?OnSetPort@CMainFrame@@QAEXXZ$1 00424a3b f   MainFrm.obj
 0001:00023a47       __unwindfunclet$?OnSetPort@CMainFrame@@QAEXXZ$2 00424a47 f   MainFrm.obj
 0001:00023a52       __unwindfunclet$?OnSetPort@CMainFrame@@QAEXXZ$4 00424a52 f   MainFrm.obj
 0001:00023a5d       __ehhandler$?OnSetPort@CMainFrame@@QAEXXZ 00424a5d f   MainFrm.obj
 0001:00023a80       __unwindfunclet$?OnNetworkSet@CMainFrame@@QAEXXZ$0 00424a80 f   MainFrm.obj
 0001:00023a8b       __unwindfunclet$?OnNetworkSet@CMainFrame@@QAEXXZ$1 00424a8b f   MainFrm.obj
 0001:00023a97       __unwindfunclet$?OnNetworkSet@CMainFrame@@QAEXXZ$2 00424a97 f   MainFrm.obj
 0001:00023aa2       __ehhandler$?OnNetworkSet@CMainFrame@@QAEXXZ 00424aa2 f   MainFrm.obj
 0001:00023ac0       __unwindfunclet$?StartEClassServer@CMainFrame@@QAEXKH@Z$0 00424ac0 f   MainFrm.obj
 0001:00023ac9       __unwindfunclet$?StartEClassServer@CMainFrame@@QAEXKH@Z$1 00424ac9 f   MainFrm.obj
 0001:00023ad2       __unwindfunclet$?StartEClassServer@CMainFrame@@QAEXKH@Z$2 00424ad2 f   MainFrm.obj
 0001:00023adb       __unwindfunclet$?StartEClassServer@CMainFrame@@QAEXKH@Z$3 00424adb f   MainFrm.obj
 0001:00023ae4       __unwindfunclet$?StartEClassServer@CMainFrame@@QAEXKH@Z$4 00424ae4 f   MainFrm.obj
 0001:00023aed       __unwindfunclet$?StartEClassServer@CMainFrame@@QAEXKH@Z$5 00424aed f   MainFrm.obj
 0001:00023af6       __ehhandler$?StartEClassServer@CMainFrame@@QAEXKH@Z 00424af6 f   MainFrm.obj
 0001:00023b20       __unwindfunclet$?StartEClassClient@CMainFrame@@QAEXH@Z$0 00424b20 f   MainFrm.obj
 0001:00023b29       __unwindfunclet$?StartEClassClient@CMainFrame@@QAEXH@Z$1 00424b29 f   MainFrm.obj
 0001:00023b32       __unwindfunclet$?StartEClassClient@CMainFrame@@QAEXH@Z$2 00424b32 f   MainFrm.obj
 0001:00023b3b       __unwindfunclet$?StartEClassClient@CMainFrame@@QAEXH@Z$3 00424b3b f   MainFrm.obj
 0001:00023b44       __unwindfunclet$?StartEClassClient@CMainFrame@@QAEXH@Z$4 00424b44 f   MainFrm.obj
 0001:00023b4d       __unwindfunclet$?StartEClassClient@CMainFrame@@QAEXH@Z$5 00424b4d f   MainFrm.obj
 0001:00023b56       __unwindfunclet$?StartEClassClient@CMainFrame@@QAEXH@Z$6 00424b56 f   MainFrm.obj
 0001:00023b5f       __unwindfunclet$?StartEClassClient@CMainFrame@@QAEXH@Z$7 00424b5f f   MainFrm.obj
 0001:00023b68       __ehhandler$?StartEClassClient@CMainFrame@@QAEXH@Z 00424b68 f   MainFrm.obj
 0001:00023b90       __unwindfunclet$?CloseEClassClient@CMainFrame@@QAEXXZ$0 00424b90 f   MainFrm.obj
 0001:00023b98       __unwindfunclet$?CloseEClassClient@CMainFrame@@QAEXXZ$2 00424b98 f   MainFrm.obj
 0001:00023ba1       __unwindfunclet$?CloseEClassClient@CMainFrame@@QAEXXZ$3 00424ba1 f   MainFrm.obj
 0001:00023baa       __ehhandler$?CloseEClassClient@CMainFrame@@QAEXXZ 00424baa f   MainFrm.obj
 0001:00023bd0       __unwindfunclet$?LockCDRom@CMainFrame@@QAEX_N@Z$0 00424bd0 f   MainFrm.obj
 0001:00023bd8       __ehhandler$?LockCDRom@CMainFrame@@QAEX_N@Z 00424bd8 f   MainFrm.obj
 0001:00023c00       __unwindfunclet$??1CMenu@@UAE@XZ$0 00424c00 f   MainFrm.obj
 0001:00023c08       __ehhandler$??1CMenu@@UAE@XZ 00424c08 f   MainFrm.obj
 0001:00023c30       __unwindfunclet$??1CWaitCursor@@QAE@XZ$2 00424c30 f   MainFrm.obj
 0001:00023c3c       __ehhandler$??1CWaitCursor@@QAE@XZ 00424c3c f   MainFrm.obj
 0001:00023c70       __unwindfunclet$?OnRButtonDown@CMyRichEdit@@QAEXIVCPoint@@@Z$0 00424c70 f   MyRichEdit.obj
 0001:00023c78       __unwindfunclet$?OnRButtonDown@CMyRichEdit@@QAEXIVCPoint@@@Z$1 00424c78 f   MyRichEdit.obj
 0001:00023c81       __unwindfunclet$?OnRButtonDown@CMyRichEdit@@QAEXIVCPoint@@@Z$2 00424c81 f   MyRichEdit.obj
 0001:00023c8a       __unwindfunclet$?OnRButtonDown@CMyRichEdit@@QAEXIVCPoint@@@Z$3 00424c8a f   MyRichEdit.obj
 0001:00023c93       __unwindfunclet$?OnRButtonDown@CMyRichEdit@@QAEXIVCPoint@@@Z$4 00424c93 f   MyRichEdit.obj
 0001:00023c9c       __unwindfunclet$?OnRButtonDown@CMyRichEdit@@QAEXIVCPoint@@@Z$5 00424c9c f   MyRichEdit.obj
 0001:00023ca5       __unwindfunclet$?OnRButtonDown@CMyRichEdit@@QAEXIVCPoint@@@Z$6 00424ca5 f   MyRichEdit.obj
 0001:00023cae       __ehhandler$?OnRButtonDown@CMyRichEdit@@QAEXIVCPoint@@@Z 00424cae f   MyRichEdit.obj
 0001:00023cd0       __unwindfunclet$?SetTitle@CAboutDlg@@QAEXXZ$0 00424cd0 f   PortChannelDlg.obj
 0001:00023cd0       __unwindfunclet$?OnBnClickedOk@CPortChannelDlg@@QAEXXZ$0 00424cd0 f   PortChannelDlg.obj
 0001:00023cd9       __ehhandler$?OnBnClickedOk@CPortChannelDlg@@QAEXXZ 00424cd9 f   PortChannelDlg.obj
 0001:00023cd9       __ehhandler$?SetTitle@CAboutDlg@@QAEXXZ 00424cd9 f   PortChannelDlg.obj
 0001:00023d00       __unwindfunclet$?OnInitDialog@CPortChannelDlg@@UAEHXZ$0 00424d00 f   PortChannelDlg.obj
 0001:00023d00       __unwindfunclet$?InitPortAndCode@CMainFrame@@QAEXXZ$0 00424d00 f   PortChannelDlg.obj
 0001:00023d08       __ehhandler$?InitPortAndCode@CMainFrame@@QAEXXZ 00424d08 f   PortChannelDlg.obj
 0001:00023d08       __ehhandler$?OnInitDialog@CPortChannelDlg@@UAEHXZ 00424d08 f   PortChannelDlg.obj
 0001:00023d30       __unwindfunclet$?OnInitDialog@CFtpClientDlg@@MAEHXZ$0 00424d30 f   PortChannelDlg.obj
 0001:00023d30       __unwindfunclet$?OnInitDialog@CCheckPasswordDlg@@MAEHXZ$0 00424d30 f   PortChannelDlg.obj
 0001:00023d30       __unwindfunclet$?SetTitle@CPortChannelDlg@@QAEXXZ$0 00424d30 f   PortChannelDlg.obj
 0001:00023d39       __unwindfunclet$?OnInitDialog@CFtpClientDlg@@MAEHXZ$1 00424d39 f   PortChannelDlg.obj
 0001:00023d39       __unwindfunclet$?OnInitDialog@CCheckPasswordDlg@@MAEHXZ$1 00424d39 f   PortChannelDlg.obj
 0001:00023d39       __unwindfunclet$?SetTitle@CPortChannelDlg@@QAEXXZ$1 00424d39 f   PortChannelDlg.obj
 0001:00023d42       __unwindfunclet$?SetTitle@CPortChannelDlg@@QAEXXZ$2 00424d42 f   PortChannelDlg.obj
 0001:00023d42       __unwindfunclet$?OnInitDialog@CFtpClientDlg@@MAEHXZ$2 00424d42 f   PortChannelDlg.obj
 0001:00023d42       __unwindfunclet$?OnInitDialog@CCheckPasswordDlg@@MAEHXZ$2 00424d42 f   PortChannelDlg.obj
 0001:00023d4b       __unwindfunclet$?SetTitle@CPortChannelDlg@@QAEXXZ$3 00424d4b f   PortChannelDlg.obj
 0001:00023d4b       __unwindfunclet$?OnInitDialog@CFtpClientDlg@@MAEHXZ$3 00424d4b f   PortChannelDlg.obj
 0001:00023d4b       __unwindfunclet$?OnInitDialog@CCheckPasswordDlg@@MAEHXZ$3 00424d4b f   PortChannelDlg.obj
 0001:00023d54       __unwindfunclet$?SetTitle@CPortChannelDlg@@QAEXXZ$4 00424d54 f   PortChannelDlg.obj
 0001:00023d54       __unwindfunclet$?OnInitDialog@CCheckPasswordDlg@@MAEHXZ$4 00424d54 f   PortChannelDlg.obj
 0001:00023d54       __unwindfunclet$?OnInitDialog@CFtpClientDlg@@MAEHXZ$4 00424d54 f   PortChannelDlg.obj
 0001:00023d5d       __ehhandler$?OnInitDialog@CCheckPasswordDlg@@MAEHXZ 00424d5d f   PortChannelDlg.obj
 0001:00023d5d       __ehhandler$?OnInitDialog@CFtpClientDlg@@MAEHXZ 00424d5d f   PortChannelDlg.obj
 0001:00023d5d       __ehhandler$?SetTitle@CPortChannelDlg@@QAEXXZ 00424d5d f   PortChannelDlg.obj
 0001:00023d80       __unwindfunclet$??1CPropertyManager@@UAE@XZ$0 00424d80 f   PropertyManager.obj
 0001:00023d80       __unwindfunclet$??0CPropertyManager@@QAE@XZ$0 00424d80 f   PropertyManager.obj
 0001:00023d8b       __unwindfunclet$??1CPropertyManager@@UAE@XZ$1 00424d8b f   PropertyManager.obj
 0001:00023d8b       __unwindfunclet$??0CPropertyManager@@QAE@XZ$1 00424d8b f   PropertyManager.obj
 0001:00023d96       __unwindfunclet$??0CPropertyManager@@QAE@XZ$2 00424d96 f   PropertyManager.obj
 0001:00023d96       __unwindfunclet$??1CPropertyManager@@UAE@XZ$2 00424d96 f   PropertyManager.obj
 0001:00023da2       __ehhandler$??1CPropertyManager@@UAE@XZ 00424da2 f   PropertyManager.obj
 0001:00023da2       __ehhandler$??0CPropertyManager@@QAE@XZ 00424da2 f   PropertyManager.obj
 0001:00023dc0       __unwindfunclet$?GetCurrentPropertyInfo@CPropertyManager@@QAEPAUPropertyInfo@@XZ$0 00424dc0 f   PropertyManager.obj
 0001:00023dc9       __ehhandler$?GetCurrentPropertyInfo@CPropertyManager@@QAEPAUPropertyInfo@@XZ 00424dc9 f   PropertyManager.obj
 0001:00023e00       __unwindfunclet$?GetCurrentSoftwareInfo@CPropertyManager@@QAEXXZ$0 00424e00 f   PropertyManager.obj
 0001:00023e0b       __unwindfunclet$?GetCurrentSoftwareInfo@CPropertyManager@@QAEXXZ$1 00424e0b f   PropertyManager.obj
 0001:00023e17       __unwindfunclet$?GetCurrentSoftwareInfo@CPropertyManager@@QAEXXZ$2 00424e17 f   PropertyManager.obj
 0001:00023e23       __unwindfunclet$?GetCurrentSoftwareInfo@CPropertyManager@@QAEXXZ$3 00424e23 f   PropertyManager.obj
 0001:00023e2f       __unwindfunclet$?GetCurrentSoftwareInfo@CPropertyManager@@QAEXXZ$4 00424e2f f   PropertyManager.obj
 0001:00023e3b       __unwindfunclet$?GetCurrentSoftwareInfo@CPropertyManager@@QAEXXZ$5 00424e3b f   PropertyManager.obj
 0001:00023e47       __ehhandler$?GetCurrentSoftwareInfo@CPropertyManager@@QAEXXZ 00424e47 f   PropertyManager.obj
 0001:00023e70       __unwindfunclet$?GethardInfo@CPropertyManager@@QAEHV?$CStringT@DV?$StrTraitMFC_DLL@DV?$ChTraitsCRT@D@ATL@@@@@ATL@@0H@Z$0 00424e70 f   PropertyManager.obj
 0001:00023e79       __unwindfunclet$?GethardInfo@CPropertyManager@@QAEHV?$CStringT@DV?$StrTraitMFC_DLL@DV?$ChTraitsCRT@D@ATL@@@@@ATL@@0H@Z$1 00424e79 f   PropertyManager.obj
 0001:00023e82       __unwindfunclet$?GethardInfo@CPropertyManager@@QAEHV?$CStringT@DV?$StrTraitMFC_DLL@DV?$ChTraitsCRT@D@ATL@@@@@ATL@@0H@Z$2 00424e82 f   PropertyManager.obj
 0001:00023e8b       __unwindfunclet$?GethardInfo@CPropertyManager@@QAEHV?$CStringT@DV?$StrTraitMFC_DLL@DV?$ChTraitsCRT@D@ATL@@@@@ATL@@0H@Z$3 00424e8b f   PropertyManager.obj
 0001:00023e94       __unwindfunclet$?GethardInfo@CPropertyManager@@QAEHV?$CStringT@DV?$StrTraitMFC_DLL@DV?$ChTraitsCRT@D@ATL@@@@@ATL@@0H@Z$4 00424e94 f   PropertyManager.obj
 0001:00023e9d       __unwindfunclet$?GethardInfo@CPropertyManager@@QAEHV?$CStringT@DV?$StrTraitMFC_DLL@DV?$ChTraitsCRT@D@ATL@@@@@ATL@@0H@Z$5 00424e9d f   PropertyManager.obj
 0001:00023ea6       __ehhandler$?GethardInfo@CPropertyManager@@QAEHV?$CStringT@DV?$StrTraitMFC_DLL@DV?$ChTraitsCRT@D@ATL@@@@@ATL@@0H@Z 00424ea6 f   PropertyManager.obj
 0001:00023ed0       __unwindfunclet$?WMIGetHardInfo@CPropertyManager@@QAEXV?$CStringT@DV?$StrTraitMFC_DLL@DV?$ChTraitsCRT@D@ATL@@@@@ATL@@@Z$0 00424ed0 f   PropertyManager.obj
 0001:00023ed9       __unwindfunclet$?WMIGetHardInfo@CPropertyManager@@QAEXV?$CStringT@DV?$StrTraitMFC_DLL@DV?$ChTraitsCRT@D@ATL@@@@@ATL@@@Z$1 00424ed9 f   PropertyManager.obj
 0001:00023ee2       __unwindfunclet$?WMIGetHardInfo@CPropertyManager@@QAEXV?$CStringT@DV?$StrTraitMFC_DLL@DV?$ChTraitsCRT@D@ATL@@@@@ATL@@@Z$2 00424ee2 f   PropertyManager.obj
 0001:00023eeb       __unwindfunclet$?WMIGetHardInfo@CPropertyManager@@QAEXV?$CStringT@DV?$StrTraitMFC_DLL@DV?$ChTraitsCRT@D@ATL@@@@@ATL@@@Z$3 00424eeb f   PropertyManager.obj
 0001:00023ef4       __unwindfunclet$?WMIGetHardInfo@CPropertyManager@@QAEXV?$CStringT@DV?$StrTraitMFC_DLL@DV?$ChTraitsCRT@D@ATL@@@@@ATL@@@Z$4 00424ef4 f   PropertyManager.obj
 0001:00023efd       __unwindfunclet$?WMIGetHardInfo@CPropertyManager@@QAEXV?$CStringT@DV?$StrTraitMFC_DLL@DV?$ChTraitsCRT@D@ATL@@@@@ATL@@@Z$5 00424efd f   PropertyManager.obj
 0001:00023f06       __unwindfunclet$?WMIGetHardInfo@CPropertyManager@@QAEXV?$CStringT@DV?$StrTraitMFC_DLL@DV?$ChTraitsCRT@D@ATL@@@@@ATL@@@Z$6 00424f06 f   PropertyManager.obj
 0001:00023f11       __unwindfunclet$?WMIGetHardInfo@CPropertyManager@@QAEXV?$CStringT@DV?$StrTraitMFC_DLL@DV?$ChTraitsCRT@D@ATL@@@@@ATL@@@Z$7 00424f11 f   PropertyManager.obj
 0001:00023f1c       __unwindfunclet$?WMIGetHardInfo@CPropertyManager@@QAEXV?$CStringT@DV?$StrTraitMFC_DLL@DV?$ChTraitsCRT@D@ATL@@@@@ATL@@@Z$8 00424f1c f   PropertyManager.obj
 0001:00023f27       __unwindfunclet$?WMIGetHardInfo@CPropertyManager@@QAEXV?$CStringT@DV?$StrTraitMFC_DLL@DV?$ChTraitsCRT@D@ATL@@@@@ATL@@@Z$9 00424f27 f   PropertyManager.obj
 0001:00023f32       __unwindfunclet$?WMIGetHardInfo@CPropertyManager@@QAEXV?$CStringT@DV?$StrTraitMFC_DLL@DV?$ChTraitsCRT@D@ATL@@@@@ATL@@@Z$10 00424f32 f   PropertyManager.obj
 0001:00023f3e       __unwindfunclet$?WMIGetHardInfo@CPropertyManager@@QAEXV?$CStringT@DV?$StrTraitMFC_DLL@DV?$ChTraitsCRT@D@ATL@@@@@ATL@@@Z$11 00424f3e f   PropertyManager.obj
 0001:00023f4a       __unwindfunclet$?WMIGetHardInfo@CPropertyManager@@QAEXV?$CStringT@DV?$StrTraitMFC_DLL@DV?$ChTraitsCRT@D@ATL@@@@@ATL@@@Z$12 00424f4a f   PropertyManager.obj
 0001:00023f56       __unwindfunclet$?WMIGetHardInfo@CPropertyManager@@QAEXV?$CStringT@DV?$StrTraitMFC_DLL@DV?$ChTraitsCRT@D@ATL@@@@@ATL@@@Z$13 00424f56 f   PropertyManager.obj
 0001:00023f62       __ehhandler$?WMIGetHardInfo@CPropertyManager@@QAEXV?$CStringT@DV?$StrTraitMFC_DLL@DV?$ChTraitsCRT@D@ATL@@@@@ATL@@@Z 00424f62 f   PropertyManager.obj
 0001:00023f90       __unwindfunclet$??0CSetDrfaultNICDlg@@QAE@PAVCWnd@@@Z$0 00424f90 f   SetDrfaultNICDlg.obj
 0001:00023f98       __unwindfunclet$??0CSetDrfaultNICDlg@@QAE@PAVCWnd@@@Z$1 00424f98 f   SetDrfaultNICDlg.obj
 0001:00023fa3       __unwindfunclet$??0CSetDrfaultNICDlg@@QAE@PAVCWnd@@@Z$2 00424fa3 f   SetDrfaultNICDlg.obj
 0001:00023fb2       __ehhandler$??0CSetDrfaultNICDlg@@QAE@PAVCWnd@@@Z 00424fb2 f   SetDrfaultNICDlg.obj
 0001:00023fd0       __unwindfunclet$??1CSetDrfaultNICDlg@@UAE@XZ$0 00424fd0 f   SetDrfaultNICDlg.obj
 0001:00023fd0       __unwindfunclet$??1CCheckPasswordDlg@@UAE@XZ$0 00424fd0 f   SetDrfaultNICDlg.obj
 0001:00023fd8       __ehhandler$??1CSetDrfaultNICDlg@@UAE@XZ 00424fd8 f   SetDrfaultNICDlg.obj
 0001:00023fd8       __ehhandler$??1CCheckPasswordDlg@@UAE@XZ 00424fd8 f   SetDrfaultNICDlg.obj
 0001:00024000       __unwindfunclet$?OnBnClickedOk@CSetDrfaultNICDlg@@QAEXXZ$0 00425000 f   SetDrfaultNICDlg.obj
 0001:00024008       __unwindfunclet$?OnBnClickedOk@CSetDrfaultNICDlg@@QAEXXZ$2 00425008 f   SetDrfaultNICDlg.obj
 0001:00024011       __ehhandler$?OnBnClickedOk@CSetDrfaultNICDlg@@QAEXXZ 00425011 f   SetDrfaultNICDlg.obj
 0001:00024040       __unwindfunclet$?OnInitDialog@CSetDrfaultNICDlg@@UAEHXZ$0 00425040 f   SetDrfaultNICDlg.obj
 0001:0002404b       __unwindfunclet$?OnInitDialog@CSetDrfaultNICDlg@@UAEHXZ$2 0042504b f   SetDrfaultNICDlg.obj
 0001:00024057       __unwindfunclet$?OnInitDialog@CSetDrfaultNICDlg@@UAEHXZ$4 00425057 f   SetDrfaultNICDlg.obj
 0001:00024063       __ehhandler$?OnInitDialog@CSetDrfaultNICDlg@@UAEHXZ 00425063 f   SetDrfaultNICDlg.obj
 0001:00024090       __unwindfunclet$?GetLocalComputerInfo@CSetDrfaultNICDlg@@QAEHXZ$0 00425090 f   SetDrfaultNICDlg.obj
 0001:0002409c       __ehhandler$?GetLocalComputerInfo@CSetDrfaultNICDlg@@QAEHXZ 0042509c f   SetDrfaultNICDlg.obj
 0001:000240d0       __unwindfunclet$?SetTitle@CSetDrfaultNICDlg@@QAEXXZ$0 004250d0 f   SetDrfaultNICDlg.obj
 0001:000240d9       __unwindfunclet$?SetTitle@CSetDrfaultNICDlg@@QAEXXZ$1 004250d9 f   SetDrfaultNICDlg.obj
 0001:000240e2       __unwindfunclet$?SetTitle@CSetDrfaultNICDlg@@QAEXXZ$2 004250e2 f   SetDrfaultNICDlg.obj
 0001:000240eb       __unwindfunclet$?SetTitle@CSetDrfaultNICDlg@@QAEXXZ$3 004250eb f   SetDrfaultNICDlg.obj
 0001:000240f4       __unwindfunclet$?SetTitle@CSetDrfaultNICDlg@@QAEXXZ$4 004250f4 f   SetDrfaultNICDlg.obj
 0001:000240fd       __unwindfunclet$?SetTitle@CSetDrfaultNICDlg@@QAEXXZ$5 004250fd f   SetDrfaultNICDlg.obj
 0001:00024106       __ehhandler$?SetTitle@CSetDrfaultNICDlg@@QAEXXZ 00425106 f   SetDrfaultNICDlg.obj
 0001:00024130       __unwindfunclet$?GetCurrentPath@@YAHXZ$0 00425130 f   comfunc:comfunc.obj
 0001:0002413c       __ehhandler$?GetCurrentPath@@YAHXZ 0042513c f   comfunc:comfunc.obj
 0001:00024170       __unwindfunclet$?SetKey@CRegistry@@QAEHV?$CStringT@DV?$StrTraitMFC_DLL@DV?$ChTraitsCRT@D@ATL@@@@@ATL@@H@Z$0 00425170 f   comfunc:Registry.obj
 0001:00024179       __ehhandler$?SetKey@CRegistry@@QAEHV?$CStringT@DV?$StrTraitMFC_DLL@DV?$ChTraitsCRT@D@ATL@@@@@ATL@@H@Z 00425179 f   comfunc:Registry.obj
 0001:000241a0       __unwindfunclet$?ReadString@CRegistry@@QAE?AV?$CStringT@DV?$StrTraitMFC_DLL@DV?$ChTraitsCRT@D@ATL@@@@@ATL@@V23@0@Z$0 004251a0 f   comfunc:Registry.obj
 0001:000241a9       __unwindfunclet$?ReadString@CRegistry@@QAE?AV?$CStringT@DV?$StrTraitMFC_DLL@DV?$ChTraitsCRT@D@ATL@@@@@ATL@@V23@0@Z$1 004251a9 f   comfunc:Registry.obj
 0001:000241b2       __ehhandler$?ReadString@CRegistry@@QAE?AV?$CStringT@DV?$StrTraitMFC_DLL@DV?$ChTraitsCRT@D@ATL@@@@@ATL@@V23@0@Z 004251b2 f   comfunc:Registry.obj
 0001:000241e0       __unwindfunclet$?WriteMSZString@CRegistry@@QAEHV?$CStringT@DV?$StrTraitMFC_DLL@DV?$ChTraitsCRT@D@ATL@@@@@ATL@@0@Z$0 004251e0 f   comfunc:Registry.obj
 0001:000241e9       __unwindfunclet$?WriteMSZString@CRegistry@@QAEHV?$CStringT@DV?$StrTraitMFC_DLL@DV?$ChTraitsCRT@D@ATL@@@@@ATL@@0@Z$1 004251e9 f   comfunc:Registry.obj
 0001:000241f2       __ehhandler$?WriteMSZString@CRegistry@@QAEHV?$CStringT@DV?$StrTraitMFC_DLL@DV?$ChTraitsCRT@D@ATL@@@@@ATL@@0@Z 004251f2 f   comfunc:Registry.obj
 0001:00024220       __unwindfunclet$?ReadMSZString@CRegistry@@QAEHV?$CStringT@DV?$StrTraitMFC_DLL@DV?$ChTraitsCRT@D@ATL@@@@@ATL@@PAD@Z$0 00425220 f   comfunc:Registry.obj
 0001:00024229       __ehhandler$?ReadMSZString@CRegistry@@QAEHV?$CStringT@DV?$StrTraitMFC_DLL@DV?$ChTraitsCRT@D@ATL@@@@@ATL@@PAD@Z 00425229 f   comfunc:Registry.obj
 0001:00024260       __unwindfunclet$?Initial@CMulticastSocket@@QAEHPAVCWnd@@V?$CStringT@DV?$StrTraitMFC_DLL@DV?$ChTraitsCRT@D@ATL@@@@@ATL@@GPBDIHH@Z$0 00425260 f   commod2:MulticastSocket.obj
 0001:00024269       __ehhandler$?Initial@CMulticastSocket@@QAEHPAVCWnd@@V?$CStringT@DV?$StrTraitMFC_DLL@DV?$ChTraitsCRT@D@ATL@@@@@ATL@@GPBDIHH@Z 00425269 f   commod2:MulticastSocket.obj
 0001:00024290       __unwindfunclet$??0CMulticastSocket@@QAE@XZ$0 00425290 f   commod2:MulticastSocket.obj
 0001:0002429e       __ehhandler$??0CMulticastSocket@@QAE@XZ 0042529e f   commod2:MulticastSocket.obj
 0001:000242d0       __unwindfunclet$??1CMulticastSocket@@UAE@XZ$0 004252d0 f   commod2:MulticastSocket.obj
 0001:000242db       __ehhandler$??1CMulticastSocket@@UAE@XZ 004252db f   commod2:MulticastSocket.obj
 0001:00024300       __unwindfunclet$?InitKern@CKiboKern@@QAEHXZ$0 00425300 f   kibokern:kibokern.obj
 0001:0002430c       __ehhandler$?InitKern@CKiboKern@@QAEHXZ 0042530c f   kibokern:kibokern.obj
 0001:00024330       __unwindfunclet$??1CKiboKern@@UAE@XZ$0 00425330 f   kibokern:kibokern.obj
 0001:0002433b       __ehhandler$??1CKiboKern@@UAE@XZ 0042533b f   kibokern:kibokern.obj
 0001:00024360       __unwindfunclet$?ExGetResString@@YA?AV?$CStringT@DV?$StrTraitMFC_DLL@DV?$ChTraitsCRT@D@ATL@@@@@ATL@@PAD0@Z$0 00425360 f   loadres:exloadres.obj
 0001:00024369       __unwindfunclet$?ExGetResString@@YA?AV?$CStringT@DV?$StrTraitMFC_DLL@DV?$ChTraitsCRT@D@ATL@@@@@ATL@@PAD0@Z$1 00425369 f   loadres:exloadres.obj
 0001:00024372       __ehhandler$?ExGetResString@@YA?AV?$CStringT@DV?$StrTraitMFC_DLL@DV?$ChTraitsCRT@D@ATL@@@@@ATL@@PAD0@Z 00425372 f   loadres:exloadres.obj
 0001:00024390       __unwindfunclet$?ExGetResBmp@@YA?AV?$CStringT@DV?$StrTraitMFC_DLL@DV?$ChTraitsCRT@D@ATL@@@@@ATL@@PAD0@Z$0 00425390 f   loadres:exloadres.obj
 0001:00024399       __unwindfunclet$?ExGetResBmp@@YA?AV?$CStringT@DV?$StrTraitMFC_DLL@DV?$ChTraitsCRT@D@ATL@@@@@ATL@@PAD0@Z$1 00425399 f   loadres:exloadres.obj
 0001:000243a2       __unwindfunclet$?ExGetResBmp@@YA?AV?$CStringT@DV?$StrTraitMFC_DLL@DV?$ChTraitsCRT@D@ATL@@@@@ATL@@PAD0@Z$2 004253a2 f   loadres:exloadres.obj
 0001:000243aa       __unwindfunclet$?ExGetResBmp@@YA?AV?$CStringT@DV?$StrTraitMFC_DLL@DV?$ChTraitsCRT@D@ATL@@@@@ATL@@PAD0@Z$3 004253aa f   loadres:exloadres.obj
 0001:000243b3       __unwindfunclet$?ExGetResBmp@@YA?AV?$CStringT@DV?$StrTraitMFC_DLL@DV?$ChTraitsCRT@D@ATL@@@@@ATL@@PAD0@Z$4 004253b3 f   loadres:exloadres.obj
 0001:000243cd       __ehhandler$?ExGetResBmp@@YA?AV?$CStringT@DV?$StrTraitMFC_DLL@DV?$ChTraitsCRT@D@ATL@@@@@ATL@@PAD0@Z 004253cd f   loadres:exloadres.obj
 0001:000243f0       __unwindfunclet$?ExCheckAllRes@@YAHPBD@Z$0 004253f0 f   loadres:exloadres.obj
 0001:000243fb       __unwindfunclet$?ExCheckAllRes@@YAHPBD@Z$1 004253fb f   loadres:exloadres.obj
 0001:00024407       __unwindfunclet$?ExCheckAllRes@@YAHPBD@Z$2 00425407 f   loadres:exloadres.obj
 0001:00024413       __unwindfunclet$?ExCheckAllRes@@YAHPBD@Z$3 00425413 f   loadres:exloadres.obj
 0001:0002441f       __unwindfunclet$?ExCheckAllRes@@YAHPBD@Z$4 0042541f f   loadres:exloadres.obj
 0001:0002442a       __unwindfunclet$?ExCheckAllRes@@YAHPBD@Z$5 0042542a f   loadres:exloadres.obj
 0001:00024436       __unwindfunclet$?ExCheckAllRes@@YAHPBD@Z$6 00425436 f   loadres:exloadres.obj
 0001:00024442       __unwindfunclet$?ExCheckAllRes@@YAHPBD@Z$7 00425442 f   loadres:exloadres.obj
 0001:0002444e       __unwindfunclet$?ExCheckAllRes@@YAHPBD@Z$8 0042544e f   loadres:exloadres.obj
 0001:0002445a       __unwindfunclet$?ExCheckAllRes@@YAHPBD@Z$9 0042545a f   loadres:exloadres.obj
 0001:00024466       __unwindfunclet$?ExCheckAllRes@@YAHPBD@Z$10 00425466 f   loadres:exloadres.obj
 0001:00024472       __unwindfunclet$?ExCheckAllRes@@YAHPBD@Z$11 00425472 f   loadres:exloadres.obj
 0001:0002447e       __ehhandler$?ExCheckAllRes@@YAHPBD@Z 0042547e f   loadres:exloadres.obj
 0001:000244a0       __unwindfunclet$?addsection@CIniStruct@@QAEHPAD@Z$0 004254a0 f   loadres:initwork.obj
 0001:000244a9       __ehhandler$?addsection@CIniStruct@@QAEHPAD@Z 004254a9 f   loadres:initwork.obj
 0001:000244d0       __unwindfunclet$?ReadProfileSection@@YAKPBD0AAVCIniStruct@@@Z$0 004254d0 f   loadres:initwork.obj
 0001:000244dc       __ehhandler$?ReadProfileSection@@YAKPBD0AAVCIniStruct@@@Z 004254dc f   loadres:initwork.obj
 0001:00024510       __unwindfunclet$?replacestr@@YAXPAD00@Z$0 00425510 f   loadres:initwork.obj
 0001:00024519       __unwindfunclet$?replacestr@@YAXPAD00@Z$1 00425519 f   loadres:initwork.obj
 0001:00024522       __unwindfunclet$?replacestr@@YAXPAD00@Z$2 00425522 f   loadres:initwork.obj
 0001:0002452b       __unwindfunclet$?replacestr@@YAXPAD00@Z$3 0042552b f   loadres:initwork.obj
 0001:00024534       __unwindfunclet$?replacestr@@YAXPAD00@Z$4 00425534 f   loadres:initwork.obj
 0001:0002453d       __unwindfunclet$?replacestr@@YAXPAD00@Z$5 0042553d f   loadres:initwork.obj
 0001:00024546       __ehhandler$?replacestr@@YAXPAD00@Z 00425546 f   loadres:initwork.obj
 0001:00024570       __unwindfunclet$?ReadIniFileKey@@YAAAV?$CStringT@DV?$StrTraitMFC_DLL@DV?$ChTraitsCRT@D@ATL@@@@@ATL@@PBD0PADAAV12@@Z$0 00425570 f   loadres:initwork.obj
 0001:0002457b       __unwindfunclet$?ReadIniFileKey@@YAAAV?$CStringT@DV?$StrTraitMFC_DLL@DV?$ChTraitsCRT@D@ATL@@@@@ATL@@PBD0PADAAV12@@Z$1 0042557b f   loadres:initwork.obj
 0001:00024587       __unwindfunclet$?ReadIniFileKey@@YAAAV?$CStringT@DV?$StrTraitMFC_DLL@DV?$ChTraitsCRT@D@ATL@@@@@ATL@@PBD0PADAAV12@@Z$2 00425587 f   loadres:initwork.obj
 0001:00024593       __ehhandler$?ReadIniFileKey@@YAAAV?$CStringT@DV?$StrTraitMFC_DLL@DV?$ChTraitsCRT@D@ATL@@@@@ATL@@PBD0PADAAV12@@Z 00425593 f   loadres:initwork.obj
 0001:000245d0       ??__EbUpFilename@@YAXXZ    004255d0 f   FtpClientDlg.obj
 0001:000245f0       ??__Em_bootMgr@@YAXXZ      004255f0 f   KiboClient.obj
 0001:00024610       ??__EgVersion@@YAXXZ       00425610 f   KiboClient.obj
 0001:00024630       ??__EtheApp@@YAXXZ         00425630 f   KiboClient.obj
 0001:00024650       ??__Eg_sock@@YAXXZ         00425650 f   MainFrm.obj
 0001:00024670       ??__Eg_mydisk@@YAXXZ       00425670 f   MainFrm.obj
 0001:000246a0       ??__Eg_mykern@@YAXXZ       004256a0 f   MainFrm.obj
 0001:000246c0       ??__Em_szMsgList@@YAXXZ    004256c0 f   MainFrm.obj
 0001:000246e0       ??__E_afxDefaultAcceleratorDelimiter@@YAXXZ 004256e0 f   stdafx.obj
 0001:00024710       ??__Eg_CurrentPath@@YAXXZ  00425710 f   comfunc:comfunc.obj
 0001:00024730       ??__Eg_tempstring@@YAXXZ   00425730 f   loadres:exloadres.obj
 0001:00024750       ??__Eg_BasicPath@@YAXXZ    00425750 f   loadres:exloadres.obj
 0001:00024770       ??__EvtMissing@@YAXXZ      00425770 f   comsuppw:comutil.obj
 0001:0002477c       ??__E_afxInitAppState@@YAXXZ 0042577c f   mfcs90:appmodul.obj
 0001:00024790       ??__FbUpFilename@@YAXXZ    00425790 f   FtpClientDlg.obj
 0001:000247a0       ??__Fm_bootMgr@@YAXXZ      004257a0 f   KiboClient.obj
 0001:000247b0       ??__FgVersion@@YAXXZ       004257b0 f   KiboClient.obj
 0001:000247c0       ??__FtheApp@@YAXXZ         004257c0 f   KiboClient.obj
 0001:000247d0       ??__Fg_sock@@YAXXZ         004257d0 f   MainFrm.obj
 0001:000247e0       ??__Fg_mydisk@@YAXXZ       004257e0 f   MainFrm.obj
 0001:000247f0       ??__Fg_mykern@@YAXXZ       004257f0 f   MainFrm.obj
 0001:00024800       ??__Fm_szMsgList@@YAXXZ    00425800 f   MainFrm.obj
 0001:00024810       ??__F_afxDefaultAcceleratorDelimiter@@YAXXZ 00425810 f   stdafx.obj
 0001:00024820       ??__Fg_CurrentPath@@YAXXZ  00425820 f   comfunc:comfunc.obj
 0001:00024830       ??__Fg_tempstring@@YAXXZ   00425830 f   loadres:exloadres.obj
 0001:00024840       ??__Fg_BasicPath@@YAXXZ    00425840 f   loadres:exloadres.obj
 0001:00024850       ??__FvtMissing@@YAXXZ      00425850 f   comsuppw:comutil.obj
